:020000040000FA
:040000006FD00400B9
:101000006F009044000000000000000090200020CD
:10101000A4220020A9BDF9F55C23002000000000F7
:10102000000000005C230020902000200000000051
:101030000000000090200020000000009020002010
:101040000000000090200020902000209020002030
:101050009020002090200020B82B0020902000201D
:10106000000000009020002090200020EC230020B1
:1010700090200020C22300209020002090200020FB
:101080009020002090200020902000209020002020
:101090009020002001A04111B7170040985F3AC688
:1010A000945F3247E39CE6FE3245410182800111A4
:1010B00013078008F337078093F787083EC20100C3
:1010C0000100B7170040930570052380B70413068D
:1010D00080FA2380C7040100010083C6B70493F699
:1010E000F60DA385D704238007049246F3A6068055
:1010F0000100010093760502D5CEF336078093F602
:10110000860836C4010001002380B7042380C70489
:1011100001000100B70614007D89558D88C70100C4
:1011200001000100010023800704A246F3A6068007
:101130000100010073370780137787083AC6010062
:1011400001002380B7042380C704010001000100CF
:1011500001003727004093061005A303D7802380A2
:101160000704B247F3A70780010001009307800836
:10117000F3B7078093F787083ECE01000100B71749
:101180000040130770052380E704130780FA2380CB
:10119000E7040100010003C7B70413670708A3852C
:1011A000E70423800704F247F3A70780010001004A
:1011B0000561828093760504BDC6F336078093F6F9
:1011C000860836C8010001002380B7042380C704C5
:1011D00001000100B7061400938606047D89558D31
:1011E00088C7010001000100010023800704C246F6
:1011F000F3A6068001000100733707801377870884
:101200003ACA010001002380B7042380C70401000B
:1012100001003727004093062005A303D7802380D1
:101220000704D24781B773370780137787083ACC12
:10123000010001002380B7042380C70401000100DE
:1012400098471367070C98C723800704E24719BF24
:101250000111814601468145114506CE6D24930753
:101260008008F3B7078093F787083EC601000100A6
:10127000B7170040130770052380E704130780FAAF
:101280002380E7040100010003C767041367170008
:101290002383E70423800704B247F3A707800100F4
:1012A0000100F2400561828041118146014681457D
:1012B0001145912C13078008F337078093F78708AF
:1012C0003EC401000100B7170040130670052380DB
:1012D000C704930680FA2380D70401000100FD555E
:1012E0002396B70223800704A245F3A505800100D9
:1012F000010073370780137787083AC601000100A1
:101300002380C7042380D7040100010003C76704BA
:10131000136717002383E70423800704B247F3A76A
:1013200007800100010001A0BD473305F50201005F
:101330007D1575FD8280411122C426C206C6AA848D
:10134000014463179400B2402244924441018280D8
:1013500005041305803E4204C13F4180DDB7000013
:101360009305000273A04580824573901534924026
:101370002242B2424243D2436244F2440255925561
:101380002256B2564257D2576258F25806499649E9
:10139000264AB64A464BD64B664CF64C065D965DE1
:1013A000265EB65E465FD65F09617300203041114C
:1013B000B7170040985F3AC6945F3247E39CE6FE59
:1013C000324541018280B71700401307000323888C
:1013D000E7028547171700002326F7F47300203033
:1013E000411122C406C6370400201C408297F5BF75
:1013F00037370040834747009146BD8B6389D7004C
:1014000099466394D700834757407300203097165E
:10141000000083C6F6F39387160017160000A30991
:10142000F6F203478700973700009387E75CB6978B
:101430002380E700B7E70400BC4F0946894517152C
:1014400000000345C5E98297C9B723030480154707
:101450002303E48001002302A48082808307648048
:10146000E3CE07FE23030480828083076480E3CEFB
:1014700007FE03454480828083076480E3CE07FE35
:101480002302A4808280411126C44AC24EC006C6EF
:101490001377F50BAD47AA892E8995446306F700AB
:1014A00019456537653F8D444E854537FD59FD1417
:1014B00063983401B240A2441249824941018280BA
:1014C000135509011375F50F453F2209CDB70111D9
:1014D00026CC06CEB704080051371545BD37713705
:1014E00069372AC6A53F32459377150089EB136506
:1014F00015001375F50FF240E24405618280FD147A
:10150000E9FC0145CDBF397126DC4ADA4ED852D606
:1015100056D45AD25ED006DE62CE66CCB7E700E083
:101520007D5783AA070022C603AA470023A0E71815
:1015300023A2E718B7170040130770052380E704BC
:10154000130780FA2380E70483C74704930B75FFD2
:10155000B684E20793FBFB0F8546AA892E8B32895E
:1015600037240040E187015763FA76016308D5000C
:101570008946130700026313D5000157D98F93F7EB
:10158000F70FB71C00402382FC0411472303E480BB
:101590001305F00F5D3D094CD135636D7C11B70526
:1015A0000700DA9537870700795563F2E504B387BA
:1015B0009500636EF702370B0800A94733EB65010E
:1015C0006399F90689E48144513D26850DA0DA85A9
:1015D0000945553D05090345F9FFFD14050B693D16
:1015E00081C49377FB0FFDF7DD3569FD7D55B71796
:1015F0000040130770052380E704130780FA238057
:10160000E70403C74704418B2382E704F250B7E79E
:1016100000E023A0571123A24711E254324452594B
:10162000C259325AA25A125B825B724CE24C21615F
:101630008280A5476395F90685691309F00FB30603
:101640009900B3742B01B6941349F9FFB374990050
:10165000856B33796901416B9387F9FFB3F72701F4
:1016600099E363FC340193D94900C147E3E637FFAE
:1016700099BF0569C1697D19D9B71305800D6388C4
:101680006901130500026384790113051008CA85F6
:10169000DD3B353D21DD4E99B3843441D9B7DA8540
:1016A0002D45D533CA94E30099F205097D3BA30F7C
:1016B000A9FED5BF9387F9FF93F7F70F6361FC0C81
:1016C00083C71C0413073008631FF704370708009B
:1016D000636BEB04B3079B00B706100063F5D704F8
:1016E000334BEB0089476393F9068980D549E38C36
:1016F00004ECDA850945413B11090327C9FF9147ED
:101700002320E48003076480E34E07FE2303348133
:10171000FD17EDFBFD14110B81C49377FB0FE9FF5F
:101720007D3371F5E1B5B717004003C75704B7071C
:1017300008001377070219E3B78707007955E378A4
:10174000FBEA33079B00E3FFE7F855B58547E382E3
:10175000F9F2DA852D45053B9389F4FFE38504E62C
:10176000293393F7390091EB83260480032709007E
:1017700093074900E39AE6E43E89CE84F1BFB5477A
:101780006396F9001305900BC93135BDB1471305B8
:10179000B00AE38BF9FE99476391F904B705080095
:1017A000B365BB002D45C53181448D4BA1497539C9
:1017B00063967401832704802320F9008504E3984D
:1017C00034FF8327048013172B016355070023126E
:1017D000F900D5BB2322F900FDB39D476399F902B7
:1017E00081451305B0044531BD442320090023225F
:1017F0000900FD599D3993F77400CA9703C7070084
:10180000FD14398D2380A700E39634FF6DBBA147FB
:101810006392F9046D398144630D0B008D47930485
:10182000C0036308FB009304000563048B01930469
:1018300040041375C507E30895D81945393139397E
:101840000545213126850D3909453D314931E31CD6
:1018500005D669BB91476399F90013056006F53613
:10186000F53E130590090DB7E38F09D4F154A9BBD8
:10187000BD660147173600001306C644938606A6C8
:1018800085458347060093F7F70F91C382800507CC
:10189000E3F9E6FE973700002386B742DDB77D16F1
:1018A0006206618693178601E18763D407000145CC
:1018B0008280931726003307F500AE9718439C43A8
:1018C00063E7E7007D16E37FF7FC7D5582800545E1
:1018D0008280FD15E205E18513978501618793F705
:1018E000F50F63480700FD15139725002A97584305
:1018F00065D7138517006205618582803308B502BC
:101900001C4283A80600B335B502C29733B5070160
:10191000AE98469585486367B5006394A50063E378
:10192000070181480C43C6950CC388C21CC2828043
:1019300081471397870161876343B70082801397BC
:1019400027002A97232007008507E5B7814701472D
:1019500093968701E18663C5B60013351700828030
:1019600093962700AA9694428507558FD5B793D7AB
:1019700055408A07AA979C4305453315B5007D8DD0
:10198000828017F3FFDFE702C33B2A84993705C53E
:10199000931725003E940327C4FF814711EB7D1563
:1019A00016053E954205418517F3FFDF6700A33B0F
:1019B00005838507E5B70145C5BF814713978701B3
:1019C00061876343C700828013972700B386E500D1
:1019D00094422A97850714C3D5B77D16620661869F
:1019E000014793178601E18763D507001335170078
:1019F000828093172600B306F500AE9794429C436D
:101A00007D16B58F5D8FF1BF8A05AA950147636387
:101A1000B500828083A6C5FFF11593D71600D98F34
:101A20009CC11397F601E5B72A8301480147014598
:101A30006343D7008280B387050183A80700B307FB
:101A400006019C43C697AA976384F80033B5170133
:101A50000507B3080301620723A0F8006187110896
:101A6000C1BF2A8301478147014563C3D7008280F4
:101A70003388E50083280800330EE600032E0E00AD
:101A80003388A8403308C8416384080133B508018E
:101A90008507B308E300E20723A00801E1871107E7
:101AA000E9B717F3FFDFE702C3290111B286B28459
:101AB0002E86AA850A8575372A84A6850A857935F2
:101AC00033348000060413351500018D056117F3CA
:101AD000FFDF6700432917F3FFDFE702032441110B
:101AE000AA89AE8A328BB68402C202C402C60144FD
:101AF000131C8401135C8C4163499C02939B14006A
:101B0000FD1B0549138CF4FFF15C33048901620469
:101B10006184634D740592478E04CE9423AEF4FE27
:101B2000410117F3FFDF6700C32213192400B30B31
:101B30002B01014A93172A00D69783A50B008843EF
:101B40007800340050005D3B050A93178A01E18755
:101B5000F11BE351FCFE92474E9905042320F90046
:101B6000A2473EC2B24702C63EC459B7131A890102
:101B7000135A8A41131D240093178A01E18763CF0A
:101B8000970092470A044E941CC0A2470509137996
:101B9000F90F3EC2B24702C63EC485BFB3079A03DF
:101BA00013152A0056950841780034005000050AA4
:101BB000EA97DA978C439933C1B70000197106C2CE
:101BC00012C416C61AC81ECA22CC26CE2AD02ED2BD
:101BD00032D436D63AD83EDA42DC46DECAC0CEC26D
:101BE000D2C4D6C6DAC8DECAE2CCE6CEEAD0EED29D
:101BF000F2D4F6D6FAD8FEDA97050000938505727E
:101C00008841E700050092402242B2424243D2435B
:101C10006244F244025592552256B2564257D25768
:101C20006258F25806499649264AB64A464BD64B60
:101C3000664CF64C065D965D265EB65E465FD65FE8
:101C40000961730020300000972100209381813BBF
:101C500017510020130101BB17F5FFFF1305C53A0B
:101C6000970500209385053A171600201306C6FD38
:101C700063FAC5008322050023A0550011059105D4
:101C8000E3EAC5FE17A501001305C54E9715002010
:101C90009385C5FB171600201306C66563FAC500B9
:101CA0008322050023A0550011059105E3EAC5FE36
:101CB0001715002013050564974500209385854C72
:101CC0006377B500232005001105E36DB5FEFD42E5
:101CD000739002BC8D4273904280B72200009382C1
:101CE000828873900230970200209382A23193E29F
:101CF00032007390523097420000938222F073902A
:101D000012346FC0E42F73002030397101436EC666
:101D100019A0397141536AC866CA62CC5ECE19A057
:101D2000397101535AD056D252D44ED64AD826DAF7
:101D300022DC06DE33016140828241114AC026C2A4
:101D400022C406C68282B24D4101024D924C224C01
:101D5000B24B4101024B924A224AB2494101024927
:101D600092442244B240410182803D432A876373FA
:101D7000C3029377F700BDEFADE5937606FF3D8A8A
:101D8000BA960CC34CC30CC74CC74107E36BD7FED4
:101D900011E28280B306C3408A069702000096963D
:101DA0006780A6002307B700A306B7002306B70085
:101DB000A305B7002305B700A304B7002304B700A9
:101DC000A303B7002303B700A302B7002302B700A1
:101DD000A301B7002301B700A300B7002300B70099
:101DE000828093F5F50F93968500D58D9396050126
:101DF000D58D61B79396270097020000969686824C
:101E0000E78086FA9680C1171D8F3E96E374C3F86B
:101E1000A5B73367B500FD530D8B79E7B7877F7F93
:101E20009387F7F710419441B372F6003363F600DD
:101E3000BE92B3E262006397720C6318D6065041FB
:101E4000D441B372F6003363F600BE92B3E262008F
:101E50006398720A631BD60410459445B372F6006A
:101E60003363F600BE92B3E262006391720A631EAE
:101E7000D6025045D445B372F6003363F600BE92E5
:101E8000B3E26200639A72086311D6021049944962
:101E9000B372F6003363F600BE92B3E2620063935E
:101EA00072085105D105E30FD6F613170601939773
:101EB0000601631CF7001357060193D7060133058B
:101EC000F7409375F50F91E982804183C183330513
:101ED000F7409375F50F91E182801377F70F93F731
:101EE000F70F3305F74082800346050083C60500DF
:101EF000050585056313D60065FA3305D640828053
:101F000011059105E312D6FE014582802105A10548
:101F1000E31CD6FC014582803105B105E316D6FCF1
:101F2000014582804105C105E310D6FC0145828050
:101F3000B717004003C777051377E70FA38BE704B4
:101F4000130700F8A38DE7043D47238CE70413072C
:101F50005003A38CE70403C7A7051377D70F238D7E
:101F6000E7048280B717004003C7E7020D894111DB
:101F70001377C70F498F93068008F3B6068093F650
:101F8000860836C601000100930670052380D70439
:101F9000930680FA2380D704010001002387E7021B
:101FA00023800704B247F3A7078001000100410125
:101FB000828041112A83014E930E407E130F001937
:101FC000930F400663E56E12930800191303400651
:101FD000B3781503854E0D4FA14F337365020D89FC
:101FE0001335150063EFBE121308F6FF7946729899
:101FF0004208135808013307C70213D61700BE075B
:1020000032976146B3F6C60213068070B386C602E5
:102010003697A166F58F42075D8FB716004083C7DC
:10202000F60293F70708A303F1000346710083C784
:10203000F60293F70708E394C7FE83477100B716CB
:10204000004093F7F70F6388071293078008F3B7F0
:10205000078093F787083EC401000100B7170040CE
:10206000930670052380D704930680FA2380D70453
:102070000100010023AA070383C6170393E606089D
:10208000A388D70223800704A247F3A70780010093
:1020900001001166B71700407D16D45BC85F9385B9
:1020A0004703A98EF18EF5FA93068008F3B60680F1
:1020B00093F6860836C6010001009306700523805A
:1020C000D704930680FA2380D7040100010098C149
:1020D00003C7170313670704A388E70223800704D5
:1020E000B247F3A7078001000100410182807D1300
:1020F0003368E3039308E016630E08003368F303C4
:102100009308D016630808009378330093B818003A
:102110009388D81633081E01131E0801135E0E01A2
:1021200055B56393E50305486386080001486303DA
:1021300003002A8871087298FD15131E0801C20554
:10214000135E0E01C18179BD13F8150063F4BF0061
:102150007908D5B713381800E5BF83C7F60293F79F
:102160000708A303F1000346710083C7F60293F743
:102170000708E394C7FE8347710093F7F70FF1DF79
:10218000E9B531714AD966CB06DF22DD26DB4ED7B1
:1021900052D556D35AD15ECF62CD6AC96EC7AA8CCA
:1021A00002D8EF00901C2A8993078008F3B70780B4
:1021B00093F787083EDA01000100B71700401307C4
:1021C00070052380E704130780FA2380E7040100E9
:1021D000010003C7F7021377770FA387E70203C74E
:1021E000F70213678700A387E70223800704D2570B
:1021F000F3A70780010001000545AD33130780C137
:102200003347E902116A93070AE893065002BD6951
:10221000930BA004814A014B1304800893047005BA
:102220007D1AB347F9023307D7023EC0FD873ECC83
:10223000938709A69309803E3347F7023AC27D8708
:102240003AC4334739038549B399990193D9394041
:10225000B306D702B30B7703B3C6F602B3CBFB02C8
:1022600036C6FD8636C893D6FB4136CEB7460F003C
:10227000938606243349D9028566938606FAB39677
:102280009601B389E902130760553309D902930611
:102290000010B389E9023349D902B3C9F902931690
:1022A000390036CA37190040FD8636D0930D09042F
:1022B00093D7F9413ED2F336048093F6860836DC94
:1022C00001000100930770052380FD00930680FA4A
:1022D0002380DD00010001008346390593F6860F57
:1022E000A309D9048346390593E61600A309D90446
:1022F00023800D00E256F3A6068001000100130CB6
:1023000080FA116DF336048093F6860836DE0100FC
:102310000100930770052380FD0023808D010100DB
:10232000010083463905216693E60602A309D90414
:1023300083560905B3E6A6012318D9048356090577
:10234000D18E2318D90423800D00F256F3A60680FF
:10235000010001008346390593F60602638A0618D8
:1023600003463905218A6DDE0818EF001004733624
:10237000048013768608B2C20100010023809D000C
:1023800023808D0101000100B717004003C6370507
:102390001376F60DA389C70403C637051366060234
:1023A000A389C704835609052166B3E6A60123184D
:1023B000D90483560905D18E2318D90423800D0032
:1023C0009646F3A60680010001008346390593F680
:1023D00006026386061483463905A18AEDFE97003E
:1023E0000020E78040CBAA8636D497000020E78003
:1023F00080CAA256E30AD5FE835609054255B3E6C4
:10240000A6012318D904C12783463905A18AEDDE28
:10241000035609058346290582473376CA00B30669
:10242000DA0293D5F641B296B388F640E24733B864
:10243000C6002E983308F840A247B3B616013308F9
:10244000D84063C70701631DF800924763FA17017C
:10245000C247634DF80E63950701B24763E8F80E73
:10246000894663E7660FF2469315180013D3F80107
:102470005E8613951800B365B30042D646D4EF606C
:10248000A1353258050B137BFB0F63470001631224
:102490000838A258638F083613081500B336A80011
:1024A000B69513D6F5013298B336C800AE961358D8
:1024B0001800FE06B3E6060173360480137686081C
:1024C000B2C60100010023809D0023808D01010020
:1024D00001000356C902B296C206C1822316D90270
:1024E00023800D00B646F3A606800100010019BD49
:1024F000F336048093F68608B6C0010001002380FD
:102500009D0023808D01010001008346390593E67B
:102510000602A309D90423800D00864605BDF336C3
:10252000048093F68608B6C40100010023809D0054
:1025300023808D01010001008346390593E60602E0
:10254000A309D90423800D00A646A5BDE30D0BF019
:10255000F336048093F68608B6C80100010093069E
:1025600080FA23809D002380DD0001000100834666
:10257000390593F5FC0F93F6860FA309D90483461A
:102580003905CD8EA309D90423800D00C646F3A6D4
:10259000068001000100130580FA03463905930601
:1025A00039051D8A631496297336048013768608CC
:1025B000B2CC01000100130680FA23809D00238025
:1025C000CD000100010003C606001376F60D23803E
:1025D000C60003C60600136606022380C6008356A3
:1025E00009051166D18E2318D90483560905216681
:1025F000D18E2318D90423800D00E646F3A6068069
:1026000001000100130680FA8346390593F606029D
:102610006388062483463905130C3905A18AFDDA3F
:1026200008186123F336048093F68608B6D00100BB
:102630000100930680FA23809D002380DD000100C5
:10264000010083460C00116693F6F60D2300DC00B2
:1026500083460C0093E606022300DC00835609053E
:10266000D18E2318D904835609052166D18E2318EB
:10267000D90423800D008656F3A6068001000100D0
:10268000130680FA8346390593F606026385062011
:1026900083463905A18AEDFE97000020E780A09FC0
:1026A0002A8C97000020E780009FE30C85FF83566B
:1026B000090511664255D18E2318D9042923834672
:1026C000390513063905A18AFDDAF336048093F63D
:1026D0008608B6D401000100930680FA23809D008D
:1026E0002380DD00010001008346060093F6F60D0D
:1026F0002300D60023800D00A656F3A60680010015
:1027000001008356090503462905D247B376DA004E
:102710003306CA021305800C9355F6413696330DE5
:10272000F6408257333CD6002E9C3336A601330C3C
:10273000FC40330CCC403308850392564E86B335AB
:10274000A5033305A503C295EF6001096346800127
:10275000631E0C16630C0D16130615003335A60008
:102760002E959356F5013696B335D600AA959396D5
:10277000F50105828585D18E6346B000639D051AFB
:10278000638B061A0356C90215823305D600333609
:10279000C500B2956348B000639105241306F00F9D
:1027A000637DA622894663F3561593078008F3B725
:1027B000078093F78708BED6010001003717004055
:1027C000930770052300F704930780FA2300F704AA
:1027D000010001008356C70289678117D58FC207A0
:1027E000C1832316F70223000704B657F3A7078017
:1027F00001000100FA506A54DA544A59BA592A5A67
:102800009A5A0A5BFA4B6A4CDA4C4A4DBA4D296126
:1028100082801308F5FF3335A800FD152E95135659
:10282000F5013298B336C800AA9651B1F336048048
:1028300093F68608B6CA0100010023809D0023801C
:10284000AD000100010083463905CD8EA309D904EE
:1028500023800D00D646F3A606800100010035BB9B
:10286000F336048093F68608B6CE0100010023807B
:102870009D002380CD00010001008346390593E6C9
:102880000602A309D90423800D00F646F3A60680AC
:102890000100010095BBF336048093F68608B6D29A
:1028A0000100010023809D002380CD000100010074
:1028B0008346390593E60602A309D90423800D0057
:1028C0009656F3A60680010001006DBB9306F5FF46
:1028D00033B5A600FD152E959355F501AE96B3B50B
:1028E000B600AA951396F501858269B5F336048082
:1028F00093F68608B6D801000100930680FA23807B
:102900009D002380DD00010001008356C902056699
:10291000011693F6F60FD18EC206C1822316D90294
:1029200023800D00C656F3A6068001000100850A2B
:1029300093FAFA0F49B233E6B60045C20356C9020C
:102940003305D0403338A000B305B040B38505410E
:1029500015826345B000D1E16371A608894663F032
:10296000560593078008F3B7078093F78708BEDA08
:1029700001000100B7170040130770052380E7042A
:10298000130780FA2380E7040100010003D7C70280
:102990007D8B2396E70223800704D65781BDF3364B
:1029A000048093F68608B6DC01000100930680FAE5
:1029B00023809D002380DD00010001008356C902B1
:1029C0000566011693F6F60FD18EC206C182231654
:1029D000D90223800D00E656B9B793078008F3B7F4
:1029E000078093F78708BEDE01000100371700401B
:1029F000930770052300F704930780FA2300F70478
:102A0000010001000356C70293975600B297C20710
:102A1000C1832316F70223000704F657C1BB914771
:102A200063EEB70217870100130787AB8A05BA95D3
:102A30009C41BA978287B717004003A7470B1345FD
:102A4000F5FF698F23AAE70A03A7070B698F23A85D
:102A5000E70A03A7070A798D23A0A70A8280B71780
:102A6000004083A6470B1347F5FFF98E23AAD70A28
:102A700083A6070B558D23A8A70A83A6070A758F7F
:102A800023A0E70A8280B717004003A7470B498FAE
:102A900023AAE70A03A7070B1345F5FF45BFB7179E
:102AA000004083A6470B1347F5FF758F23AAE70A5B
:102AB00003A7070A598D4DB7B717004003A7470B67
:102AC000498FEDB7914763EEB702178701001307EF
:102AD00067A28A05BA959C41BA978287B7170040CA
:102AE00003A7470D1345F5FF698F23AAE70C03A73A
:102AF000070D698F23A8E70C03A7070C798D23A086
:102B0000A70C8280B717004083A6470D1347F5FF37
:102B1000F98E23AAD70C83A6070D558D23A8A70CE1
:102B200083A6070C758F23A0E70C8280B71700409F
:102B300003A7470D498F23AAE70C03A7070D1345E9
:102B4000F5FF45BFB717004083A6470D1347F5FFB4
:102B5000758F23AAE70C03A7070C598D4DB7B7173C
:102B6000004003A7470D498FEDB7B71700408847CE
:102B7000420541819377050491EB9377F501375531
:102B8000E801130505803345F50282809377050C33
:102B9000130700046397E7009377F50137459C1C02
:102BA000CDB72165130505D0828037E700E01C43CF
:102BB0005443A183E206D58F1CC1FD572320F7188B
:102BC0002322F718828013178500B7E700E023A0BF
:102BD000E710618123A2A7108280B7F700E0884741
:102BE000CC478280814737370040A14663C4C70085
:102BF000328582800345B740E38EA6FE3385F5001B
:102C00000345050085072304A740CDB7970700209B
:102C10009387476A9C43173700201307A7563E95B2
:102C2000636EE500174700201307C79D6368A70080
:102C3000170700202320A7683E858280FD57EDBF3F
:102C4000411122C406C62A840D372947B307E5027D
:102C5000B2408D83B3D7870222449507B3D7E702EA
:102C600037370040C207C1832316F7004101828035
:102C7000716541111305052006C6D937B7370040E5
:102C8000130770F82381E7000D47A381E7001307BE
:102C90000004A380E70005472387E700B240410115
:102CA000828037370040834727001A0593F7F703E0
:102CB000C98F93F7F70F2301F7008280B7370040E1
:102CC00003C7170019C9D98DA380B70003C7070030
:102CD000136787002380E700828093C5F5FFF98D95
:102CE000A380B7008280B73700402147B736004045
:102CF00091E1828003C6B700E30CC7FE05050346D9
:102D0000F5FFFD15C2052384C600C181D5B7411169
:102D100022C406C62A84913D2947B307E502B24082
:102D20008D83B3D7870222449507B3D7E70237379D
:102D30000040C207C1832316F740410182807165BC
:102D400041111305052006C6D937B73700401307D0
:102D500070F82381E7400D47A381E7401307000483
:102D6000A380E74005472387E740B24041018280C6
:102D7000CC41411106C6328503C6150083C5050046
:102D800022064D8E42068D654186138875A2630C1E
:102D90000611634BC804138845A26300060D634AFD
:102DA000C800938535A26301B60823900600294622
:102DB0004DA0138855A26305060D938565A2E31601
:102DC000B6FE8D451D4663E6E5081146198E63F390
:102DD000C7003E86B7E704002390C600FC479795DE
:102DE0000100938525339DA0138895A263030611E6
:102DF000634E060D1388A5A263000613938505A5EF
:102E0000E315B6FA99451D4663E5E504198E63F3AB
:102E1000C7003E86B7E704002390C600FC4797052D
:102E200000209385A5491DA09D451D4663E3E5024D
:102E30002146198E63F3C7003E86B7E70400FC47BE
:102E40002390C600970500209385C54ABA958297BE
:102E50000146B240328541018280AD451D46E3EA1C
:102E6000E5FE3146198E63F3C7003E86B7E70400DE
:102E70002390C600FC47977501009385A56AF9B7B2
:102E8000B1451D46E3E7E5FC3546198E63F3C700FF
:102E90003E86B7E704002390C600FC479775010003
:102EA0009385456965B78D451D46E3E4E5FA11460E
:102EB000198E63F3C7003E86B7E704002390C6006F
:102EC000FC47979501009385A52549B78D451D467B
:102ED000E3E1E5F81146198E63F3C7003E86B7E7D4
:102EE00004002390C600FC479795010093850525B3
:102EF000B1BFA5451D46E3EEE5F42946198E63F3FF
:102F0000C7003E86B7E704002390C600FC479775CC
:102F10000100938565601DBFB5451D46E3EBE5F2F5
:102F20003946198E63F3C7003E86B7E70400239045
:102F3000C600FC47977501009385055D01BFB7E7A3
:102F4000040003A3071397060020938626D9414661
:102F5000A54517050020130565CF02832D4559EFC0
:102F600003C5050009476317E50803A8450041119B
:102F700006C6034718003285034608002207416849
:102F8000518F930828FE6308170363E9E8000518CA
:102F9000630307052390060029451DA8130648FE74
:102FA000630BC7021518E31707FF15463E87637BBF
:102FB000F602154705A83E8691C30546B7E704000B
:102FC000FC472390C6004206CC45418282970145CA
:102FD000B240410182801306700F3E876374F60091
:102FE0001307700FB7E704002390E600FC471316A1
:102FF0000701D9BF23900600054582808280416782
:1030000079176304E504411122C406C685472A8462
:10301000639FF500B7E7040022852244B24003A372
:103020008713970500209385A52D410102838947C9
:103030006399F500B7E7040083A7070B85458297DE
:1030400071D9B2402244410182808280797122D4B8
:1030500052CC2E842A8A977501009385E54F177507
:1030600001001305255106D63AC626D24AD0B684A9
:1030700032894ECEEF509141A68517750100130598
:103080006550EF50B1402945EF509144834784008B
:1030900093F70702E1E78349040089470545324772
:1030A0006396F908544083C7160083C60600A2073A
:1030B000D58FC166138616FE638CC7028D16638F8B
:1030C000D7068D669386269029456391D706B7E784
:1030D0000400A285225403A34714B250F249A686E5
:1030E0004A86925402595285624A85474561028355
:1030F0002D450DEF9307700F354563E99702B7E74C
:103100000400FC4748441306700FCA858297814922
:10311000970700209387871F9C43014581CB9C43E1
:1031200091C74E852686CA8582970145B2502254A2
:1031300092540259F249624A456182802D457DF7D9
:103140009307700F3545E3E397FEB7E70400FC47AC
:1031500048441306700FCA8582975DBF2145F9B7B1
:10316000411122C437E404008327841326C2AA84B1
:10317000416506C697050020938585187D158297C1
:103180008327C40A170500001305A5E785888297E1
:1031900095C0032304132244B240924497060020B2
:1031A000938686C54146C545170500201305C5B35E
:1031B00041010283B2402244924401454101828090
:1031C00019C59707002023A3A71401458280454510
:1031D00082801147636AA70A977601009386863634
:1031E0000A0536951841411106C63697AE87B28555
:1031F00002871307700F6145639DE700B7E704007E
:10320000FC471306700F170500201305E51682977B
:103210000145B2404101828005476145E39BE7FEDD
:10322000B7E70400FC470546170500201305050D08
:10323000F9BF1307700F6145E39DE7FCB7E7040092
:10324000FC471306700F1705002013056522C1B750
:103250001307700F6145E39EE7FAB7E70400FC47E8
:103260001306700F17050020130505304DB71547DD
:103270006145E390E7FAB7E70400FC4715461705F8
:1032800000201305250861B709458280411126C237
:10329000B7E4040083A7C41322C44AC006C62E8420
:1032A000970500209385C5052A898297058905C55C
:1032B00097070020938747A383D7A70BA28503A373
:1032C000440D2310F4002244B24092444A8502493E
:1032D000014641010283B2402244924402494945D9
:1032E000410182809707002023840702970700206E
:1032F00023A20702B717004003A7070CB706C0FFB9
:10330000FD16758F23A0E70C03A7070DB706400035
:10331000558F23A8E70C03A7070C3D9B23A0E70CC0
:1033200003A7070D1367070123A8E70C8280B717CF
:10333000004003A5470C83A7470C5981134515008E
:10334000C18B058999E3136525009707002083C782
:1033500027FC6380A70297070020238BA7FA11C9D7
:1033600097070020938707FB03A30700630303006D
:103370000283828011456FE0DFE0411193962500C2
:10338000AA852D4506C697F0FF1FE780C017B240FB
:10339000014541018280011122CC06CE3714004044
:1033A00026CA4AC84EC652C483447405034AB405AB
:1033B0008349840503499405EFE09FB78347A4053B
:1033C00093F4F40F137AFA0F93E71700230DF40424
:1033D00093F9F90F1379F90FB717004003C7A70541
:1033E000058B6DFF03D5C705A38D4705238C3705D6
:1033F000A38C2705A38B9704F2406244D244424930
:10340000B249224A0561828041119397050122C485
:1034100006C626C2C1872E8463DC0700B7E4040019
:10342000FC54829719C1BC5482972165218D3DA01F
:1034300093F7150013C5150095E393F7250085C78D
:10344000FD35B7E70400BC4F1306000A8945170590
:1034500000200345A5EC829713452400B240224486
:103460009244410182809397250163D50702B7E416
:10347000040083A7C41E8297F53DBC4C37F60200BA
:10348000130606E0896517050020034525E98297A4
:10349000096569BF939715010145E3D107FC1775CD
:1034A00001001305E514EF503113B7E70400BC4FDA
:1034B00013060064916517050020034525E68297F1
:1034C0001165ADB72D71232A9110FD74E98C232C61
:1034D000811023282111232631112A84AE893289B3
:1034E000930600100A86A6852D45232E111097F00D
:1034F000FF1FE780400113154401B7E70400FC47B4
:1035000051810A0513962900CA850A958297A685D6
:1035100085660146254597F0FF1FE780C0FE0A86B5
:10352000A68593060010294597F0FF1FE780A0FDB0
:103530008320C11103248111832441110329011126
:103540008329C11015618280B7F7070003C70701FF
:10355000411106C622C426C24AC0A547631AF70015
:103560009537B2402244924402490145410182808C
:1035700013942500AA843289A286AA85014625458E
:1035800097F0FF1FE78020F8A2864A86A685294586
:1035900097F0FF1FE78020F7E9B71D71A2CC37E451
:1035A00004005C5C485886CE4946977501009385B7
:1035B000A5FF829701E91775010013052500EF505B
:1035C000B10101A0B7F600E0795798CAFD57DCCAEF
:1035D0000567B7E700E023A0E7101306F00290C2EA
:1035E00023A0E71801000100370700201847130641
:1035F000000481459706002023A0E6D24157A38A04
:10360000E7403C440808829797170020938787DE9D
:103610003EC8856713870760231AE1001D673ACC0F
:1036200037070105130707103ACE9387B7D313075F
:10363000B00F2310E1022312F102054797F7FFFFB5
:103640009387E7592301E1023ED8170700001307CB
:1036500007D397070000938747D4B7F50700BAC28E
:103660003EDC17070000130767EE970700009387FB
:10367000A7D081463000E1051945BAC43EDE97F077
:10368000FF1FE78040E818088147994630003E96C2
:103690000346060085070507A30BC700E398D7FE7E
:1036A000C24791C70357410185676373F70001A0C3
:1036B000B7E7040083A7470A08088297AA8501C9CB
:1036C000177501001305C5F0EF50415C01A0F640ED
:1036D000664425618280411126C2B7E4040083A7B5
:1036E000040806C622C417050000130525D28297D8
:1036F00017040020130484C22300A4003128DD36FF
:1037000003450400224403A38405B24092441306F7
:103710000032896541010283797106D622D41307EC
:103720008008F337078093F787083EC20100010045
:10373000B7170040930570052380B704130680FA7D
:103740002380C7040100010083C6F70293F6A60F89
:10375000A387D702238007049246F3A606800100C0
:10376000010073370780137787083AC4010001000E
:103770002380B7042380C7040100010003C7F702B8
:1037800013672700A387E70223800704A247F3A754
:103790000780010001000545EFE0CFFCE13E014755
:1037A00081468147054685451305407EEFE07F80D1
:1037B00037E404003C446800514681458297B707CE
:1037C000C0A83EC8B787E803938707D03ECA97F7DB
:1037D000FF1F9387C7BD3EC67C5868008297B250D2
:1037E00022544561828041119775010093850550EF
:1037F00017750100130505D806C6EF502149177546
:10380000010013052569EF506148B2402945410187
:103810006F50014C4111977501009385654E1775E6
:103820000100130525D506C6EF5041461775010066
:1038300013050565EF508145B240294541016F50A0
:103840002149411122C406C6834705002A849DC32D
:10385000977501009385855017750100130585D173
:10386000EF50C1424C40177501001305E576EF504B
:10387000E1411DA058411DE7977501009385054E54
:1038800017750100130505CFEF5041401775010072
:1038900013050576EF50813F2244B240294541018E
:1038A0006F500143A1679386D7036311D7029775C1
:1038B00001009385A54A177501001305A5CBEF50AC
:1038C000E13C177501001305A573E9B7ED0797757E
:1038D00001009385A548177501001305A5C9631953
:1038E000F700EF50A13A177501001305A5725DB7F7
:1038F000EF50C1394C40177501001305A57385BF02
:103900004111977501009385E54017750100130576
:1039100065C606C6EF508137B240294541016F5058
:10392000213B797122D426D24AD02E842A8981451E
:10393000B2844800714606D6EFE02FC397F7FF1F09
:103940009387076BDC4783D70700231421012313D8
:10395000F100EF20B0019547A305F1009307401F48
:103960003EC6FD572305A100230AF100EF205012A7
:103970002686A2854800EF205002B250225492546D
:10398000025945618280970700202392079C970780
:103990000020238D079AB7E70400BC47411106C6F3
:1039A000414681451385413D8297EF103067EF1006
:1039B00090440145EF30401403C7C1259307F00A36
:1039C000631BF7009307F00889451385C125239EE3
:1039D000F124EF30C03EEF30A04E814537050400A2
:1039E0009707002023A0079697070020239A0794A3
:1039F000970700202387079497070020239F0792AB
:103A000097070020239A079297070020239907928F
:103A100097070020239A0792EF20C0360145EF3028
:103A2000C040977501009385653117750100130536
:103A300065B4EF50A125177501001305E565EF503A
:103A4000E124B240294541016F508128411122C42F
:103A500006C626C293F715002E84638D070C814697
:103A600017F6FF1F13064656854517050020035518
:103A7000658CEF80700905C5977501009385C52C8D
:103A800017750100130505AFEF50412017750100B0
:103A9000130545CEEF50811F2945EF5061239775DF
:103AA00001009385652A177501001305A5ACEF5039
:103AB000E11D17750100130525CDEF50211D294586
:103AC000EF50012117F5FF1F130585525C4505478F
:103AD0002390E700EFF0A019977501009385C526A4
:103AE00017750100130505A9EF50411A177501005C
:103AF0001305C5CAEF5081192945EF50611D930781
:103B000010F8238EF1249707002083D76782A38EB5
:103B1000F1241385C125A1839145238FF124A38F1F
:103B20000124EF30C02913451400B24022449244CE
:103B30004101828093F72500D1CB1707002003575E
:103B4000278051C397F6FF1F9386C67F94429777CD
:103B500001009387675617F6FF1F0346867E81454F
:103B60001385413DEF409007AA8431CD9775010040
:103B700093854524177501001305C59FEF5001116A
:103B8000A685177501001305E5C2EF5021102945E0
:103B9000EF50011497F7FF1F2394077A930710F84B
:103BA000238EF12497F7FF1F83D78778A38EF12404
:103BB000A183238FF12491458D471385C125A38FC0
:103BC000F124EF30C01F1345240085B793F745005B
:103BD000B1CF977501009385E51D17750100130599
:103BE0006599EF50A10A17750100130565BEEF50E6
:103BF000E1092945EF50C10D930720F8238EF124E8
:103C000097F7FF1F83D76773A38EF124A183238FB8
:103C1000F1248547A38FF124EF2080671385C12508
:103C20009145EF30C0191345440001B793F7850063
:103C30008DCF977501009385E51717750100130562
:103C40006593EF50A104177501001305A5B9EF5056
:103C5000E1032945EF50C10797F7FF1F2392076E35
:103C6000EF40B00413458400C9B593F70501A5C31F
:103C7000854517F5FF1F0355456CEF00714E97758D
:103C8000010093852513177501001305A58EEF40DC
:103C9000F17F17750100130525B6EF40317F2945E7
:103CA000EF500103930730F8238EF12497F7FF1F9D
:103CB00083D7A768A38EF1241385C125A1838D45E1
:103CC000238FF124EF30A00F13450401B9BD93F702
:103CD0000502B5C3977501009385C50D17750100E1
:103CE00013054589EF40917A17750100130505B357
:103CF000EF40D1792945EF40B17D930740F8238EFD
:103D0000F12497F7FF1F83D72763A38EF124A183A4
:103D1000238FF1248547A38FF12497F7FF1F239D5D
:103D20000760EF20E0561385C1259145EF3020094B
:103D300013450402DDBB93F70504CDC79775010059
:103D400093854507177501001305C582EF4011746F
:103D500017750100130505AEEF4051732945EF407B
:103D6000317783C7C1251307700A6388E7041307F7
:103D7000800A6386E7061307600A6397E7029307E2
:103D800060F8238EF12497F7FF1F83D7475BA38E3C
:103D9000F124A183238FF1248547A383F126B14524
:103DA0001385C125EF30A001EF20804E1345040498
:103DB00097F7FF1F239507588DBB930770F8238E45
:103DC000F12497F7FF1F83D78757A38EF124A18390
:103DD000238FF1248547A380F1269945D1B7930716
:103DE00080F8F1BF93F705080145E38007D4977584
:103DF0000100938525FC176501001305A577EF40A9
:103E0000F16817750100130565A4EF403168294575
:103E1000EF40116C9307A0F8238EF12497F7FF1F52
:103E200083D78752A38EF124A183238FF124854762
:103E3000A38FF12497F7FF1F23980750EF204045E9
:103E40001385C1259145EF20907713450408F1B9FA
:103E5000411122C497750100938585F12A84176565
:103E600001001305257106C6EF4051624C401775DD
:103E700001001305E513EF4071612945EF405165DD
:103E8000034704009307F00F6319F70297750100C9
:103E9000938505EE176501001305C56DEF40115FB1
:103EA0004C40177501001305A511EF40315E224407
:103EB000B240294541016F40B161B2402244410105
:103EC000828085CD411122C4176501001305856AE2
:103ED0002E84977501009385A5E406C6EF40115B1B
:103EE000A285177501001305E518EF40315A2244E9
:103EF000B240294541016F40B15D8280411122C429
:103F000026C22E84AA8497750100938525E2176541
:103F100001001305256606C6EF40515717750100CD
:103F200013050516EF4091562945EF40715A9775D4
:103F300001009385A5DF97F7FF1F239D973E176527
:103F4000010013052563854497F7FF1F2392873EE1
:103F500097F7FF1F239F973C97F7FF1F2399873EF3
:103F6000EF40D15297F5FF1F83D5653E17750100CD
:103F700013058511EF4091512945EF40715597F791
:103F8000FF1F2385973CEF1000672285EF20D03676
:103F90000545EF20906997F7FF1F93876705DC477A
:103FA00003D70700C167FD176312F7022244B7E782
:103FB0000400B240924403A3870517F5FF1F034591
:103FC00065361306000A854541010283B24022444A
:103FD000924441018280011122CC37E404005C5CF0
:103FE00006CE26CA3546977501009385E5EB177511
:103FF000010013052578829701E917650100130573
:10400000E55BEF40715D01A097F7FF1F9387476560
:104010003EC4B7F507008567938707C0814617F64A
:10402000FF1F13066630E10519453EC697E0FF1FE6
:10403000E780604D7C44194697F5FF1F9385C52E98
:10404000138581368297340017F6FF1F1306C62D9D
:10405000977501009385C52F177501001305C530AD
:10406000EF404010AA8415C997750100938585D348
:104070001765010013050550EF405141A6851775DE
:104080000100130565E3EF4071402945EF405144BD
:10409000F2406244D24405618280EFA02027177568
:1040A0000100130565D8EF30802BEF706015EF002D
:1040B000F13317F5FF1F130565F0EF00D1201775D9
:1040C0000100130565D7EF003134AA84EF303006C4
:1040D000EFC04059EF209153EF405022EF30706510
:1040E000EFE03036977501009385C5CB1765010069
:1040F0001305454889C8EF407139A6851775010039
:104100001305C5DD49B7EF40713817750100130578
:1041100025DFEF40B1372945EF40913BEFE0D01864
:10412000EFB000436305050E854537050400EF1029
:104130007045977501009385E5C617650100130565
:104140006543EF40B134177501001305E5DCEF401E
:10415000F1332945EF40D13797F7FF1F938787D970
:1041600083D7070017F7FF1F2313F71E854717F79D
:10417000FF1F230DF71CEF106065EF10C04717F508
:10418000FF1F0355C51CEF20301797F7FF1F83C78C
:10419000D71BB9EFA303010083274417130671004F
:1041A000854513055030829797750100938585BF2B
:1041B000176501001305053CEF40512D17750100EF
:1041C0001305C5D7EF40912C2945EF407130977505
:1041D0000100938525BD176501001305A539EF4042
:1041E000F12A17750100130565DBEF40312A71BD17
:1041F00097750100938505BB176501001305853789
:10420000EF40D128177501001305C5D665BF977516
:104210000100938525B9176501001305A535EF4009
:10422000F12617750100130525E7EF4031262945D2
:10423000EF40112A0145EF20503F51BF411122C4E8
:1042400037E404008327041A06C68297EF209013F0
:104250008327040817F5FFFF1305857F829797F7DB
:10426000FF1F2381A70C17F5FF1F130565D8EF204B
:10427000002F2244B2404101B9BB411122C49146F2
:104280002A84138601349D652D4506C697E0FF1FDD
:10429000E7806027B7F7070003C70701A547631347
:1042A000F70001A09306001001469D65254597E0A3
:1042B000FF1FE7804025238081342244B24091468D
:1042C000138601349D652945410117E3FF1F6700EF
:1042D0008323B7E704001171FC47CED79389C1252A
:1042E000A2DDCAD986DFA6DB2E8432892E86AA8576
:1042F0004E85829783C70900130780029387E707DB
:1043000093F7F70F636AF774176701001307872E97
:104310008A07BA979C43BA9782878D4797750100A1
:10432000938585AA176501001305C524630BF40066
:10433000EF40D115176501001305C567EF40111552
:10434000FDA2EF40B1141765010013052568EF4089
:10435000F1132945EF40D117930720F811469385B3
:10436000C1254A85238EF124A38F0124EFF06FDB52
:104370002A840DC597750100938505A51765010071
:104380001305451FEF409110A28517650100130525
:10439000A567EF40B10F2945EF40911397750100D4
:1043A000938585A2176501001305C51CEF40110E0A
:1043B0001765010013058566EF40510D2945EF4053
:1043C00031114165930730FA05469385C1257D1566
:1043D000238EF124EFF0EFD42A840DC597750100E8
:1043E0009385859E176501001305C518EF40110AD6
:1043F000A2851765010013052561EF4031092945A4
:10440000EF40110DB7E70400BC4F0566130606C860
:10441000A14517F5FF1F0345E5F08297FE506E5446
:10442000DE544E59BE591161828091476301F402F6
:10443000977501009385459917650100130585134C
:10444000EF40D1041765010013058560C5BDB7E7CE
:104450000400FC4F914517F5FF1F0345A5EC82971B
:104460009775010093854596176501001305851022
:10447000EF40D101176501001305455FEF401101C1
:104480002945EF40F104EF10B0609145E1A2854766
:104490006301F40297750100938505931765010088
:1044A0001305450DEF40817E176501001305855DFD
:1044B00071B597F7FF1F239227E9B7E70400056658
:1044C000BC4F130606C8C145A9B78D476301F40266
:1044D000977501009385458F1765010013058509C0
:1044E000EF40C17A176501001305855B81BD930715
:1044F00040F811469385C1254A85238EF124A38F68
:104500000124EFF00FC22A84E30A05F09775010039
:104510009385858B176501001305C505EF4001776D
:10452000A285176501001305254EEF402176294528
:10453000EF40017AE5B59147E31CF4F8B7E70400D2
:10454000FC4F9305000217F5FF1F0345A5DD829779
:10455000977501009385458717650100130585014F
:10456000EF40C172176501001305055501BF89476A
:1045700063E1870297750100938505851765010042
:10458000130545FFEF4081701765010013050554C1
:1045900075B383C4E12583C7D12597750100938541
:1045A000A582A204176501001305C5FCDD8CEF4050
:1045B000E16DA2851765010013058552EF40016D7D
:1045C000C2042945EF40C170C1849305D4FF93967E
:1045D0000401C1824A8693F5F50F1385F125EF108A
:1045E000E07DE35D90E2930750F8238EF12483C7CA
:1045F000390022869385C12585074A85A38FF1243A
:10460000EFF02FB22A84E30B05E097650100938554
:10461000A57B176501001305E5F5EF402167A2852D
:1046200017750100130505A409B7894763E18702DF
:10463000976501009385457917650100130585F39A
:10464000EF40C164176501001305454BC5B9EF1074
:104650003044A2851385C125EF206076C1B38D4714
:104660006301F402976501009385057617650100E3
:10467000130545F0EF408161176501001305C54939
:1046800075B9B76602000146B7750200054597E0A7
:10469000FF1FE78040E7930760F8238EF124A38F84
:1046A00001249307002623A0F126E57793870721AD
:1046B0002392F1263146A383A1269385C1254A85FD
:1046C00023830126EFF0EFA52A84E30905D497653B
:1046D00001009385656F176501001305A5E9EF409B
:1046E000E15AA28517650100130585443DBDB14718
:1046F0006301F402976501009385056D176501005C
:10470000130545E7EF40815817650100130505447F
:1047100035B1B7E70400FC4F9305000417F5FF1F00
:10472000034545C08297EF10B036B14525B7914794
:1047300063E18702976501009385056917650100AC
:10474000130545E3EF408154176501001305C5418A
:10475000F5B683C4012683C7F125A204DD8C8E043F
:10476000B77702006D14BE942286A68517650100F6
:104770001305C540EF408151B7E70400FC4722868E
:10478000938511262800829793160401C182300078
:10479000A685094597E0FF1FE780E0D62A8419C562
:1047A000176501001305453FEF400163930770F85B
:1047B00019469385C1254A85238EF124A38081263D
:1047C000EFF02F962A84E30B05C4976501009385CB
:1047D000A55F176501001305E5D9EF40214BA285C0
:1047E000176501001305453C89B399476301F4102F
:1047F000976501009385455D17650100130585D711
:10480000EF40C148176501001305853B05BE914780
:1048100063E18702976501009385055B17650100D9
:10482000130545D5EF408146176501001305C53ACC
:1048300031B683C4012683C7F125A204DD8C8E0422
:10484000B77702006D14BE942286A6851765010015
:104850001305C539EF408143B7E70400FC472286C2
:10486000938511262800829793160401C182300097
:10487000A6850D4597E0FF1FE780E0C82A8419C58B
:104880001765010013054538EF400155930780F87F
:1048900019469385C1254A85238EF124A38081265C
:1048A000EFF02F882A84E30B05B697650100938506
:1048B000A551176501001305E5CBEF40213DA28509
:1048C00017650100130585358DB199476301F40221
:1048D000976501009385454F17650100130585C94C
:1048E000EF40C13A176501001305C53481BCB7E735
:1048F0000400FC4F9305000417F5FF1F034585A234
:104900008297EF10F0189945B1B38D476301F40217
:10491000976501009385454B17650100130585C513
:10492000EF40C136176501001305453201BC17651C
:1049300001001305A532EF40214A1305C01297E08C
:10494000FF1FE780409F0145EFE02FA60D45EFF0E8
:10495000DF92294597E0FF1FE780E09D97E0FF1F6A
:10496000E780008F65BC99476301F40297650100F9
:1049700093858545176501001305C5BFEF400131DB
:10498000176501001305452E55BA03C7112683C7C5
:10499000012622075D8F9166BA96C2061166C18212
:1049A0001306F6EF8D476363D60297E7FF1F9387E1
:1049B00027649C4B03C6F1259386C70039C603D6EE
:1049C00007005DCA8907E39CD7FE89471307A0F853
:1049D00011469385C1254A85238EE124A38FF124B6
:1049E000EFE03FF42A84E30B05A29765010093856D
:1049F000A53D176501001305E5B7EF402129A28504
:104A000017650100130585270DB603D6070063025D
:104A1000E60A8907E39BF6FE8D474DBF9147630287
:104A2000F402976501009385253A17650100130587
:104A300065B4EF40A125176501001305A5256FF0AA
:104A4000FF8FB7E70400FC4F9305000817F5FF1F21
:104A50000345458D829705BC976501009385C53652
:104A600017650100130505B1EF40412217650100EC
:104A70001305C5236FF09F8C2390E70017E5FF1FF8
:104A800013050557EFE04020976501009385C53376
:104A900017650100130505AEEF40411F17650100C2
:104AA0001305C521EF40811E2945EF406122814752
:104AB00031BF2390070017E5FF1F13056553EFE093
:104AC000A01C97650100938525301765010013052B
:104AD00065AAEF40A11B176501001305A51FD9B7F3
:104AE000411122C406C6834705002A849DC39765E9
:104AF000010093852529176501001305A5A7EF403F
:104B0000E1184C40176501001305055CEF400118E2
:104B100075A05841B707CF009387777D6313F706D9
:104B2000976501009385052617650100130585A487
:104B3000EF40C1151C448356E4008355C40003C6EE
:104B40000700176501001305A559EF4021142945F9
:104B5000EF4001180357E40097E7FF1F83D7277F33
:104B60006307F7008355C4000844EFE0CF9703566E
:104B7000E4008355C40008442244B24041016FF070
:104B80004FF5B707CC009387777D631FF7029765D2
:104B900001009385251F176501001305A59DEF40B2
:104BA000E10E1C448356E4008355C40003C607008D
:104BB000176501001305C552EF40410D2244B24074
:104BC000294541016F40C110B707CE009387777D1B
:104BD0006302F702976501009385C51A1765010006
:104BE00013054599EF40810A4C40176501001305F4
:104BF000654429BFB2402244410182805171CAD12B
:104C000037E904008327C904A2D52E8686D7A6D308
:104C10002E84AA851385C125829783C7C1251307D2
:104C2000700A638DE70C636CF7001307600A6382F8
:104C3000E704BE502E549E540E596D6182801307B6
:104C4000800A6382E7121307900AE394E7FE8D4718
:104C5000630BF416976501009385C518176501006D
:104C600013054591EF408102176501001305C5AD9D
:104C700015A08D476306F40297650100938585169C
:104C8000176501001305058FEF404100176501000E
:104C90001305C5A4EF30917F2945EF40610351BF53
:104CA000854717650100130525A517E7FF1F230793
:104CB000F768EF406112B7750200B766020001465F
:104CC000054597E0FF1FE7800084930760F8238E77
:104CD000F124A38F01249307002623A0F126E57772
:104CE000938707212392F126B14523830126A383CD
:104CF000A1261385C125EF20800C25BF914763E1D4
:104D00008702976501009385E50D1765010013057E
:104D10006586EF30B177176501001305E59F9DBFEC
:104D200083C4012683C7F125A204DD8C8327C9042F
:104D30006D14228693851126280082978E0493167F
:104D40000401B7750200C1823000A695094597D0CD
:104D5000FF1FE780407B930770F8238EF12499456D
:104D6000A380A12679B7914763E187029765010087
:104D700093854507175501001305C57FEF30117165
:104D8000176501001305C59A31B783C4012683C78F
:104D9000F125A204DD8C8327C9046D142286938536
:104DA0001126280082978E0493160401B77502001D
:104DB000C1823000A6950D4597D0FF1FE780A074F3
:104DC000930780F859BF1765010013052599EF4037
:104DD000A1001305C01297D0FF1FE780C055014501
:104DE000EFD0BFDC0D45EFF04FC9294597D0FF1F2D
:104DF000E780605497D0FF1FE78080451DBDB7E76F
:104E000004004111FC4726C29384C1252E8606C6A4
:104E100022C44AC02E842A89AA852685829797654E
:104E200001009385E5FD175501001305A574EF30CA
:104E3000F16583C5C125176501001305A5A2EF30F3
:104E4000F1642945EF30D16883C704004147938757
:104E5000070693F7F70F6365F74817670100130715
:104E6000A7838A07BA979C43BA9782879D476303B3
:104E7000F402976501009385A5F817550100130505
:104E8000656FEF30B160176501001305259EEF30A7
:104E9000F15FD1A283C7D125ADCF83D7012603D738
:104EA000E125C207D98F17E7FF1F232DF74883C7D6
:104EB0006400976501009385A5F41755010013055B
:104EC000656B17E7FF1F230EF746EF30315C97E75E
:104ED000FF1F938727478C4317E6FF1F034666464D
:104EE000176501001305459AEF30515A2945EF30F7
:104EF000315EA38E01242244B240924402499307BA
:104F000000F8238EF1249D451385C12541016F10C2
:104F1000106BEF302065239FA124935705012A844D
:104F20002380F126935785010145A380F126EF30B8
:104F300020642381A12697650100938565EC1755B0
:104F4000010013052563EF30715403C62126A285A5
:104F5000176501001305C59441BFCD476301F402F5
:104F6000976501009385C5E9175501001305856014
:104F7000EF30D151176501001305059409BF37E4DF
:104F800004007C4441469385D1251385413D829799
:104F90001385413DEF00E07CB92D83C7E12603C7AF
:104FA000D126A20703238405D98F17E7FF1F2319F2
:104FB000F7381306000A89452244B2409244024958
:104FC00017E5FF1F03450536410102838D47630145
:104FD000F402976501009385A5E2175501001305BA
:104FE0006559EF30B14A176501001305A59C45B519
:104FF00003C4E12583C7D12597650100938545E06A
:105000002204175501001305E5565D8CEF30114859
:10501000A285176501001305A58BEF30314729459F
:10502000EF30114B0D469385C1252285EFE07F8F30
:10503000AA8415C997650100938585DC1755010081
:1050400013054553EF309144A685176501001305FC
:105050006589EF30B1432244B24092440249294568
:1050600041016F30F14697E7FF1F2398872CB7E780
:105070000400116603A38705130606E891452DBFBA
:105080008D476301F40297650100938565D7175535
:1050900001001305254EEF30713F17650100130520
:1050A00025A0F5B303C4E12583C7D1259765010089
:1050B000938505D52204175501001305A54B5D8C7A
:1050C000EF30D13CA285176501001305E582EF3072
:1050D000F13B2945EF30D13F0D469385C12522850F
:1050E000EFE03F84AA840DC197650100938545D107
:1050F0001755010013050548EF305139A68517658E
:1051000001001305A580B1B797E7FF1F23968722FB
:10511000B7E70400116603A38705130606E89305A5
:10512000000259BD894763E18702976501009385B5
:1051300025CD175501001305E543EF3031351765CF
:1051400001001305A598A1B383C4E12583C7D12528
:10515000976501009385C5CAA20417550100130580
:105160006541DD8CEF309132A6851755010013059E
:10517000657BEF30B1312945EF309135228693853B
:10518000C1252685EFE0EFF92A84630A05169765A5
:1051900001009385E5C6175501001305A53DEF30C5
:1051A000F12EA28517550100130505795DB58547D8
:1051B00063F78714834519002244B24092440249A0
:1051C000B335B00097E7FF1F238AB71617550100C4
:1051D0001305C57741016F30712BA2852244B2407F
:1051E00092444A85024941016FF05FA199476301EA
:1051F000F402976501009385A5C0175501001305BA
:105200006537EF30B128176501001305E5A541B1F9
:1052100003C4E12583C7D12597650100938545BE69
:105220002204175501001305E5345D8CEF3011267B
:10523000A285175501001305E572EF303125294588
:10524000EF30112919469385C1252285EFE06FEDD6
:10525000AA840DC197650100938585BA1755010091
:1052600013054531EF309122A6851755010013052E
:105270006570C5B397E7FF1F2398870CB7E7040055
:10528000116603A38705130606E8930500082DB3EE
:105290008547976501009385A5B61755010013054D
:1052A000652D6309F400EF30711E175501001305D9
:1052B000A56DF1BEEF30911D175501001305456E28
:1052C000EF30D11C2945EF30B1202244B240924446
:1052D000024997E7FF1F2395070641016F30E01C45
:1052E000976501009385C5B1175501001305852801
:1052F000EF30D119176501001305459B49BEB24037
:1053000022449244024941018280411106C622C4CE
:10531000EFE02FE19377F50F95CB2A849765010095
:10532000938585AF175501001305C524EF3011167D
:105330009375F40F176501001305C5D2EF301115F1
:105340002244B240294541016F309118B2402244B5
:105350004101828001114EC6B28917E6FF1F035634
:10536000E6F726CA4AC806CE22CCAA842E8925236F
:1053700097E7FF1F83C787FDA9CB03C4440083C7FA
:105380003400176501001305E5D922045D8CEF3068
:10539000F10F4A86A68522858D3F638F090297E724
:1053A000FF1F83C787FA8DCB6308090297E7FF1FAA
:1053B00083C7C7F895E36244F240B249CA8526859F
:1053C0004249D24405616F10901F17650100130513
:1053D000E5D5EF307120D1B7F2406244D244424962
:1053E000B2490561828083475500834545001765B2
:1053F00001001305E5D1A207DD8D6F303109176576
:1054000001001305E5CF6F30311D8D4763F2B70AF8
:10541000011126CA06CE22CC0344350097E4FF1FB3
:1054200083C4B4F297650100938505D1B33780003A
:1054300017E7FF1FA30BF7F009C4976501009385D9
:1054400065D017650100130565D0EF30310497E78B
:10545000FF1F83C797EF63839700252C97E7FF1FF4
:1054600083C7B7EE9DC385472306F100B7E7040065
:1054700083A747177000854513055030829717653D
:1054800001001305A5CDEF3031159967938757EECD
:105490002316F100680085479145A3078100230783
:1054A000F100EF10D011F2406244D24405618280D5
:1054B0008280894763F2B708011122CC06CE26CA42
:1054C0008344250085472A846398F404914763F058
:1054D000B704034545008347340022055D8D97E7F7
:1054E000FF1F239DA7DE3D219967938767EE231455
:1054F000F1008347340023059100A305F1008347A1
:105500004400954528002306F100EF10500BF240AF
:105510006244D24405618280FDF89967938767EE03
:105520002314F10097E7FF1F83D747DBA305F100A2
:1055300023050100A183F1B782800111996722CC74
:10554000D51717E4FF1F130464E02314F100834709
:10555000040026CA97E4FF1F938464DF2305F1004B
:1055600083D7040028009545A305F100A18306CE4A
:105570002306F100EF10B00403D6040083450400B5
:1055800017650100130505BFEF304170F24062441A
:10559000D244056182809D677971D9172316F10085
:1055A00097E7FF1F83C787DA06D62307F1009DCB55
:1055B000B7E70400FC4741469385413D1305F100E0
:1055C00082976800CD45EF10807F97E5FF1F83C568
:1055D000E5D7176501001305E5BCEF30216BB2502C
:1055E00045618280B7E70400BC4741468145130509
:1055F000F1008297F9B7B76702036971938757AAD9
:105600003EC48567938717A02316F10097E7FF1F15
:105610009387C7D383C7070023248112A307010000
:105620002307F10097E7FF1F938767D283D707000F
:1056300037E40400232611122318F10097E7FF1F17
:105640009387C7C983D70700414648082319F1004B
:105650007C449385413D8297F1452800ED2A231231
:10566000A1027C442C002810794682973C44130503
:1056700061041306900D8145829730109305700FD9
:105680000145EFD01FB58320C1120324811255615B
:105690008280B7C7A55A01119387C7333EC497E7E5
:1056A000FF1F83C797CA3EC6B7F7070003C70701A6
:1056B00006CE22CCA5476313F70001A01164930521
:1056C00004F0930600100146254597D0FF1FE780A0
:1056D00080E33000930504F0A146294597D0FF1FD1
:1056E000E78060E297E5FF1F83C535C617650100B7
:1056F000130505BCEF308159F24062440561828098
:1057000001119165A1463000938505F02D4506CE27
:1057100097D0FF1FE78020DF2247B7C7A55A93879E
:10572000C7336312F702B24517650100130585AB55
:10573000B335B00097E7FF1FA389B7C0EF3001551D
:10574000F240056182808547854517650100130594
:10575000A5AB17E7FF1FA30AF7BEEF302153153F94
:10576000C5B7B7C7A55A79719387F7353EC6B7E76E
:105770000400FC47AA8506D622D441460808829731
:10578000B7F7070003C70701A5476313F70001A098
:105790001164930504E8930600100146254597D04F
:1057A000FF1FE78040D67000930504E8D1462945E5
:1057B00097D0FF1FE78020D517650100130505B3BB
:1057C000EF308161B25022544561828079719165D8
:1057D000D1467000938505E82D4506D697D0FF1F6A
:1057E000E78060D23247B7C7A55A9387F735176568
:1057F0000100130565A9631EF700B7E70400FC4725
:105800001385413D41460C08829717650100130539
:10581000A5A5EF30615CB25045618280B7F7070003
:1058200003C70701A5476313F70001A09165411164
:10583000930600100146938505E8254506C697D0D6
:10584000FF1FE78040CCB240176501001305C597E4
:1058500041016F306158C16769768146FD170506C1
:105860001397060141836364B7003E858280330746
:10587000D50003470700B98F214713F81700858328
:1058800063050800B18FC207C1837D171377F70F37
:105890006DF78506F1B725CD25478546637AB706AE
:1058A000411122C406C626C20347150083460500DF
:1058B00031682207558F931687002183558F420741
:1058C00041831308C8552A848546631C0703034790
:1058D000250011486377E802130857006393050316
:1058E00093043700A301C50021822302C500A685C9
:1058F0009D37B30794002380A7002181A380A700D0
:105900008146B240224492443685410182808546D8
:1059100036858280B7C7A55A01119387E7343EC404
:105920002AC6B7F7070003C7070106CE22CC26CA4E
:10593000A5476313F70001A091642A84938504EEC0
:10594000930600100146254597D0FF1FE780A0BBB6
:105950003000A146938504EE294597D0FF1FE780CC
:1059600080BAA2851765010013058596EF300132D4
:10597000EFF07FC8F2406244D24405618280011199
:105980009165A1463000938505EE2D4506CE97D052
:10599000FF1FE78040B72247B7C7A55A9387E73470
:1059A0006314F702B245176501001305E58797E711
:1059B000FF1F2395B792C205C181EF30212DEFF073
:1059C0009FC3F24005618280D147D1451765010030
:1059D0001305858717E7FF1F2312F790EF30012B80
:1059E00017E5FF1F0355858F3537E1BF011126CA23
:1059F00006CE22CC93F71500AE848DCBAD6737175A
:105A000000409387A7AA1CC3B7E70400BC4F130646
:105A10000019854517E5FF1F0345258C829713C59F
:105A20001400F2406244D2440561828093F725005D
:105A300063830712976501009385458F2D464800C3
:105A4000EF30611997E5FF1F83C55590854793C4D3
:105A5000240063E1B70489CD97E7FF1F83C7E78E72
:105A600085C38545170500201305C5F8EF102035BF
:105A70001395040197E7FF1FA38A078C418155B74F
:105A800041650546970500209385C5F67D15EFF025
:105A9000DF87F9BF170400200344C4F597070020EF
:105AA00083C757F522045D8CAD679387B7556306AE
:105AB000F40863E68702A9679387A7556306F4088D
:105AC00097E7FF1F83C767888DE741652E867D15A1
:105AD00097050020938505F2EFF03F83B9A0B167E9
:105AE0009387C755630EF400B5679387D755E319BD
:105AF000F4FC170500201305E5EFEF10402C35A04E
:105B00000546170500201305E5EEEFF0BF8497E783
:105B1000FF1F83C7A78391EB4800EF302134931513
:105B20000501C1814800EFD00F9CA28517550100E7
:105B30001305C57DEF30811525BF1705002013051E
:105B400065EBEFF05F8AD5B717050020130585EAEE
:105B5000EFF0FF8AD9BF93F745000145E38307ECD7
:105B6000175501001305C57BEF300127EF100037F3
:105B700013C544007DB5411122C437E404005C5CC8
:105B800006C6354697550100938505321765010015
:105B9000130545BE829701E9175501001305C57924
:105BA000EF30812301A08327041C82972A840545B6
:105BB000EF802075EF10C168EF100147EF70B0293A
:105BC0002285B2402244410182801567B717004008
:105BD0001307575598C3D8439D66558FD8C3D843EC
:105BE000FD76758FD8C3D8431367F70FD8C33567D1
:105BF0001307C7CC98C3828041111305800406C6E1
:105C000022C426C24AC097C0FF1FE780404A85458C
:105C10007D55EFC0DFE085457D55EFC0BFEA371405
:105C200000408327840A8D451305002093E7072051
:105C30002324F40AEFC0BFDEB7E40400EFD02F90B6
:105C4000C8581309840C1304C40CEF30E11817650D
:105C50000100130525B2EF3021188327C4FF8545C5
:105C6000414593E70708232EF4FEEFC0BFE58D45BD
:105C700013050008EFC01FE5EFC09FFF0145EFD0FF
:105C80004F8285450545894717D7FF1F2302F76CCB
:105C9000EFD0CF8237070004B7E700E023A0E7107A
:105CA000EFD0BF8FEFD03FA3F935EFF07FA5EFF036
:105CB0001FCDEFE0AFD88D450D65EFC0BFE01705F4
:105CC0000020130525E385671CC58967232025016E
:105CD00040C12326250100C95CC983A7841E829781
:105CE00083A7040817050000130585D0829797D76E
:105CF000FF1F2384A75EBC4C130600648545829772
:105D0000E93597C0FF1FE780A06D01458280B7F796
:105D1000070003C70701A547AE866316F7009397F0
:105D2000450191C301A0AA850146254517C3FF1F60
:105D30006700637D4111B2862E86AA852D4506C671
:105D400097C0FF1FE780207CB2400145410182805F
:105D50009307000463E6C7021D71A2CC2A840808D9
:105D600086CE32C6EF203167B2461008A28529459B
:105D700097C0FF1FE7802079F64066442561828046
:105D800039558280411126C2AE848D4522C406C693
:105D90002A84EFC03FD3B717004099C803A5C70CAA
:105DA000418D23A6A70CB240224492444101828037
:105DB00003A5870C418D23A4A70CF5B783470500E5
:105DC00003471500A207D98FC2076177C187130760
:105DD00027206397E70083452500370504005DB75A
:105DE000828097D7FF1F9387E75618429C4383D63C
:105DF00045000345070083C5C70003564600639668
:105E0000A50083D5E700638DD502011106CE238658
:105E1000A7002397D700B705CF00DC4B9385757D8E
:105E200005077D162EC2230001003AC42316C100C7
:105E30002317D10099C30A858297F24005618280B9
:105E40008280DC4DDC4B81CFB7E70400904503A393
:105E50008705914517D5FF1F0345055002838280B2
:105E60006D713C083EC6B707E500232291103EC87D
:105E7000AA843C083285232611103ECA23248110AF
:105E8000232021112E89EF2090672A849755010045
:105E90009385C552174501001305C56DEF20115FAD
:105EA000A2851755010013056561EF20315E294574
:105EB000EF201162B705CB009385757D6800EF1068
:105EC000A043A2856800EF20305901478146700049
:105ED000CA852685EF10C06215C52A849755010032
:105EE0009385C54D174501001305C568EF20115A6C
:105EF000A285175501001305255DEF20315929456D
:105F0000EF20115D8320C1100324811083244110F0
:105F1000032901105161828097D7FF1F9387874320
:105F200018429C43797122D406D60348070083C8DF
:105F300007012A8483D6450003554600639608016D
:105F400083D82701638DD802238807010507239989
:105F5000D7003708CC00DC4B1308787D3ACC130708
:105F6000F5FF42CA23080100231EE100231FD100D0
:105F700099C7080832C62EC482973246A2452285A8
:105F8000C535B2502254456182806D713C083EC0D7
:105F9000B707E5003EC23C083EC423261110232467
:105FA00081102322911023170100231801002319C7
:105FB0000100231A0100231B010097D7FF1F83D77D
:105FC000270799E3C167FD172316F10097D7FF1F35
:105FD00083D7270691EB97D7FF1F9387A7379C435B
:105FE0009C43DC4783D7070017D4FF1F13044404E6
:105FF000584C2317F10083574400484B2318F100F5
:1060000005ED97550100938565421745010013057D
:106010006556EF20B1471755010013056542EF2083
:10602000F1462945EF20D14A8320C1100324811075
:10603000832441105161828097D7FF1F83C7B7FF28
:1060400089EBB7E70400BC5782975C4C23AA070092
:10605000E1BFFD1797D6FF1FA38FF6FC035607017C
:10606000834704014C470A85230BF100EF20F03CE5
:1060700097D7FF1F9387072E9C430147814688438C
:106080000A866C00EF10C047AA841DC9975501000D
:106090009385C539174501001305C54DEF20113F04
:1060A000A685175501001305653AEF20313E2945B5
:1060B000EF201142584CB7E70400BC57484B69B772
:1060C00097D7FF1F83C737F7F5D7B7E70400BC4F53
:1060D0001044854517D5FF1F034505288297A9B7AA
:1060E0005C4EDC4BA9CBA1C9411122C4174501006C
:1060F000130545482E84975501009385653106C6E2
:10610000EF20D138A2851755010013056536EF2021
:10611000F1372945EF20D13BB7E704002244B240D4
:1061200003A3870517D5FF1F034505231306400664
:106130009145410102838280411122C417D4FF1F7F
:10614000130404ED1C4C06C689C7DC4399C34C48B4
:106150008297584CB7E70400BC57484B82975C4C79
:10616000B240224423AA07004101828017D7FF1FB3
:106170001307E716834707009306F00B850793F78D
:10618000F70F63E9F60097D6FF1F238AF61403453D
:1061900007008280930700F8FDB7835745006386A8
:1061A000070E01114AC817D9FF1F130969E852C425
:1061B000032AC90106CE22CC03274A0126CA4EC6AD
:1061C00056C2F15721EF1307D00DFD576368C7047E
:1061D000B7E9040083A709072A841305860042054E
:1061E0004181B284AE8A8297232AAA000325C9017D
:1061F0005C499DEF975501009385851F1745010068
:1062000013054537EF209128175501001305852EFA
:10621000EF20D1272945EF20B12BDD57F240624412
:10622000D2444249B249224A924A3E85056182805F
:1062300093874400B705CF002319F5009385757D3A
:106240003105EF10600B0325C9018345640031055A
:10625000EF2090200325C9012686D6853105EF2041
:10626000D01D7146A2854A85EF20F116504419CA07
:1062700083A78905854517D5FF1F0345E50D82973F
:10628000814769BFEFF07FD0E5BFFD573E85828033
:10629000411126C297D4FF1F938484D9D84C22C4BD
:1062A00037E404003C54484B06C68297DC4C032379
:1062B000C4052244B240924423AA070017D5FF1F09
:1062C00003458509854541010283411126C297D4C2
:1062D000FF1F938424089C4006C622C44AC0C9CB31
:1062E000DC43D9C75CC12300B5002A84975501005F
:1062F0009385450B174501001305C527EF2011199C
:106300002945EF20F11C9C4023A4070023A207008D
:1063100097D7FF1F9387C7CFDC4FDC4B81C7295529
:10632000EFF09FE197D7FF1F938787D0DC4FDC4BBF
:1063300091C3B93F37E904008327C905894517D5BB
:10634000FF1F0345650182978327C905914517D52E
:10635000FF1F0345650082979C4003A34701630923
:10636000030022852244B240924402494101028343
:10637000B240224492440249410182800111328597
:1063800006CE22CC26CA2E84EF207017AA849755F9
:10639000010093856504174501001305A51DEF2035
:1063A000F10E030784000356640083554400A6865B
:1063B000175501001305C50DEF20510D2945EF209C
:1063C000311197D7FF1F83C707C563989700014511
:1063D000EFF09FD681450A85CD3DF2406244D2441C
:1063E000056182806D7123248110232611102322E0
:1063F000911093F745002E84638507123C083EC038
:10640000B707E5003EC23C083EC42317010023182D
:10641000010023190100231A0100231B010097D753
:10642000FF1F83D7E7BE99E3C167FD172316F1006D
:1064300097D7FF1F83D7E7BD91EB97D7FF1F9387B0
:1064400067F19C439C43DC4783D7070017D7FF1FA6
:10645000130707BC2317F100544F83574700231835
:10646000F100DC4A95EF97550100938525FB174510
:10647000010013052510EF207101175501001305C8
:1064800025FCEF20B1002945EF209104134544007D
:106490008320C11003248110832441105161828024
:1064A00097D7FF1F83C737B72555ADCBFD1717D635
:1064B000FF1FA302F6B603D6060183470701CC46A9
:1064C0000A85230BF100EF20407797D7FF1F9387B2
:1064D00067E89C4317D7FF1F130787B39766010030
:1064E000938686C888430A866C00EF106001AA84F0
:1064F00051DD97550100938565F21745010013059D
:106500006507EF20A178A68517550100130505F44E
:10651000EF20C1772945EF20A17B2685EFF0DFC171
:10652000B5B793F725009DC3B7E70400BC474146C4
:106530008145280882972555EFF01FC0280893054C
:10654000F00FEFF09FD81345240099B793F715008B
:1065500001459DDFEFF07FA31345140015BF5C4D8F
:10656000411106C688C317D7FF1F2325F7DEB7E7FB
:10657000040083A70708170500001305E5E68297C6
:10658000B24097D7FF1F2389A7DC014541018280D4
:1065900001119307700F2316F10006CE97D7FF1F46
:1065A00083C757DC8DE7B7E7040083A7870D17D6AD
:1065B000FF1F034626D36C0017D5FF1F0355C5DA0E
:1065C00082973335A00097D7FF1FA38DA7D8F2403D
:1065D0000561828041119397050122C406C626C237
:1065E000C1872E8463D40702B7E40400FC5417D596
:1065F000FF1F034525CF829719C1BC54829721659F
:10660000218DB240224492444101828093F71500CB
:106610008DC7B7E7040083A7471A17D6FF1F1306D5
:1066200026A397F5FF1F9385E55117D5FF1F034557
:1066300065CB829713451400E9B793F7250099CFEE
:10664000B7E70400BC4F13060064894517D5FF1F48
:10665000034545C982971345240065B793F7850024
:106660009DC7B7E7040003A8871A1307401F97D7F1
:10667000FF1F83C727C7814613064006994517D5D4
:10668000FF1F035565CE0298134584009DBF93F705
:1066900045000145BDD7B7E4040083A7041817D50A
:1066A000FF1F035565CC8297BC4C130600649145CF
:1066B00017D5FF1F034505C382971345440091B7C3
:1066C00097D7FF1F83D747CA6396A70217D7FF1F25
:1066D000231DB7C817D7FF1F231AC7C817D7FF1F17
:1066E0002317D7C82E8617550100130565F6BE85FA
:1066F0006F20C15917550100130505F76F20C16DB3
:1067000003574500011106CE22CC97D7FF1F83D730
:10671000A7C517550100130525F56310F706C167D6
:10672000F91717D7FF1F2321F7C437E4040097D7C1
:10673000FF1F23AD07C27C4C894517D5FF1F0345BA
:1067400065BA82977C4C914517D5FF1F034585B9E3
:10675000829797D7FF1F83C757BF95C78547A30762
:10676000F100832744171306F100854513055030C7
:106770008297175501001305A5E4EF20E165F2406B
:1067800062440561828097D7FF1F83C727BC1755D6
:1067900001001305A5E7F5F38547A307F10083275B
:1067A00044171306F100854513055030829717559D
:1067B0000100130525E3D1B77D15954763E0A71ABE
:1067C00017570100130787DC0A053A951C41011190
:1067D00022CC06CE26CABA972E848287175501008E
:1067E000130505E9EF20415F0DA203C72500994776
:1067F000631DF7002E85EFF0BFF083456400175549
:1068000001001305E5E7EF20614897D7FF1F238EAE
:1068100007B217550100130565E8E9B703C725005E
:1068200095476317F702C16717D7FF1F0357C7B311
:10683000F91703D5A5006307F702B7E7040083A79C
:10684000C717829717550100130545E6EF20C15879
:10685000854717D7FF1F230AF7AE17550100130509
:1068600065E749B797D7FF1F2390A7B083D7E50007
:10687000B7E40400096617D7FF1F2318F7AE83D7C4
:1068800005011306069017D5FF1F0345A5A517D7C9
:10689000FF1F231DF7AC83D72501A14517D7FF1F85
:1068A0002317F7ACBC4C8297BC4C1306006491458F
:1068B00017D5FF1F034505A382970356E4008355B0
:1068C000A400175501001305A5DFEF20213C49B7AF
:1068D000175501001305C5E031B783C52500914761
:1068E000639AF5028547175501001305E5E0A307F4
:1068F000F100EF20614EB7E7040083A747171306A6
:10690000F1008545130550308297F2406244D2442D
:10691000056182809947639EF5002285EFF05FDE76
:106920008345640017550100130585D5EF20013616
:10693000E9BF9547639FF500834714001755010091
:10694000130585DBE39007EA17550100130585DC85
:1069500051BD17550100130565DCC9BF82806D71FB
:10696000232481102326111023229110328401CD7B
:1069700089476306F5028320C11003248110832414
:10698000411051618280175501001305E5D9AE848D
:10699000EF208144A2852685EFE06FC6E9BFB7E707
:1069A0000400FC472800829717550100130585D87D
:1069B000EF2081428347810039C01307000B638EAB
:1069C000E7001387A7051377F70F8D4663E9E60203
:1069D000A2852800EFE08FA279BF8547E3FD87F805
:1069E0008345910017450100130545F6B335B00006
:1069F00097D7FF1F2384B794EF204129ADBF0347EA
:106A00009100A207D98F35671307D755638DE70625
:106A10006366F7022D671307B7556381E706316791
:106A20001307C7556386E70429671307A7556392C1
:106A3000E702A2852800EFE09F9C35BF39679306E7
:106A4000E7656383D70663E9F6001307E7556388B4
:106A5000E704A285280089B73D679306F755638A46
:106A6000D7041307F766E396E7FEEFE0DFB221B73E
:106A70000146A2852800EFE0FF8DF5BDA285280024
:106A8000EFE07F96CDBD8947E3F787EE9305E4FFFE
:106A9000C205C1811305A100EFC0EFA4E9BDA28525
:106AA0002800EFE09F96C1BDA2852800EFE07FA0FF
:106AB000D9B5EFE09FA8C1B5411122C417C4FF1F8B
:106AC0001304C45AAA86175601001306A6AD2285E0
:106AD000C14506C6EF2041310357440097C7FF1F49
:106AE0009387C7592393E700035764002394E70073
:106AF000B240224441018280011106CE22CC6D3F7A
:106B000037E404008327841417C6FF1F13060656B4
:106B1000D54501458297832784179305F100130516
:106B2000503082978347F100A1C7A3070100832754
:106B300044171306F10085451305503082978327CB
:106B4000441717C6FF1F13066653CD451305703053
:106B500082978547A307F100832744171306F100A6
:106B60008545130550308297F2406244056182806A
:106B70008327441717C6FF1F13064650CD4513053C
:106B80007030D5B7130101DE232C812037E40400D7
:106B900083270408232E1120232A91202328212132
:106BA0002326312117050000130505A3829717C975
:106BB000FF1F13092973994785442300A90023184F
:106BC000F100975501009385E5A693074006174508
:106BD00001001305259A2314F1102304910097C98D
:106BE000FF1F9389C976EF20610A83D509001755E5
:106BF00001001305E59BEF2061092945EF20410DB8
:106C000003D50900EFF05FEB83274417300085457B
:106C10001305503082978327441717C6FF1F1306AA
:106C2000E645CD451305703082978327441717C674
:106C3000FF1F1306A642B5451305603082978327D0
:106C4000441710088945130510318297832744178C
:106C50003002894513052031829783274415930517
:106C600000050D45829783274415930500051145BE
:106C70008297A30191002302910023049100232411
:106C80000110230801008327841630029145130563
:106C900070408297832784161306310085451305BB
:106CA00000408297832784165000854513051040C5
:106CB0008297832784161008854513052040829704
:106CC000832784163000854513055040829783271B
:106CD00004157D558297832744137D5582977D55F2
:106CE000EFC00FC88327440C8297EFC04FA58327BE
:106CF000841417C6FF1F13066637D54501458297D2
:106D000089471306700F814508082302F100EFB090
:106D1000CF858D471306700F814528022308F100A7
:106D2000EFB0AF8491472304F11097C7FF1F9387FB
:106D3000E75B984383C747003AC42306F100EFE0BE
:106D40009F8B500085450545EFC0AFC810089305DF
:106D5000700F0945EFC0EFC730029305700F0D4566
:106D6000EFC02FC7300095451145EFC08FC6C167F2
:106D700017C7FF1F1307475FF9171CC3232207001C
:106D800017C5FF1F1305C555EFC08FC38327C41D4B
:106D900017C5FF1F1305855C82973C480345090012
:106DA000854582978320C1210324812183244121A9
:106DB000032901218329C1201301012282800111AD
:106DC000C16726CA06CEAA8422CC17C5FF1F035569
:106DD000A559F9176306F50437E4040083278412E4
:106DE0002E862315B10001478146ED4582977C44EC
:106DF0000356A1002AC6A68582972C0017C5FF1F3F
:106E000003558556EFC08FC801CD175501001305F6
:106E10006583EF10717C8327C412ED4528008297AB
:106E2000F2406244D24405618280011106CE22CC38
:106E30002DC9854717C7FF1FA307F72297C7FF1F55
:106E40002384072237E40400832784179305F10085
:106E50001305503082978347F100A9CBA3070100A7
:106E6000832744171306F100854513055030829798
:106E70008327441717C6FF1F1306461EB545130583
:106E8000603082978547A307F100832744171306D4
:106E9000F1008545130550308297F2406244056148
:106EA000828097C7FF1FA380071C49BF8327441711
:106EB00017C6FF1F1306861AB54513056030E9BFD4
:106EC000C16717C5FF1F0355254AF9176307F5006A
:106ED000B7E7040003A3C717028382800111854727
:106EE000A307010017C7FF1F230EF746B7E70400EB
:106EF00083A7471706CE1306F100854513055030CA
:106F00008297F24005618280EFA29FE12A840845C2
:106F10002E89B28909C900C1970500009385C574FF
:106F20006105EF00810181447D5AEF10C00963C300
:106F3000A4048144EF10200A63C6A40497F7FF1F3E
:106F4000938707C19C43DC47B307F940918723022D
:106F5000F400638109048327C900B307F4409587CF
:106F6000A302F4001C4C89C79C4799C322858297D1
:106F70006FA05FDE5C44139714008504BA972390DA
:106F8000470165B71C48139714008504BA972390EE
:106F900007004DB7832789000547B307F44095875D
:106FA000A302F40083570400638EE7028DC30947F0
:106FB0006384E7040D47E397E7FA97570100938747
:106FC00027CA1CCC97570100938787CA11A89757E7
:106FD0000100938767901CCC975701009387C79057
:106FE0005CC849B7974701009387077C1CCC97473B
:106FF00001009387677CEDB797570100938707CB14
:107000001CCC97570100938767CBD9BF85E1EFA2CE
:10701000DFD2004618448347940075839D8B631527
:10702000F700EF00501C48C46FA07FD38280EFA20E
:107030003FCF13893500C16442094111AA89014437
:10704000F11413590901054A2EC6EF00D077B24555
:107050006346A400014541016FA0DFCF83A709006B
:1070600013171400BA9783D707006388B700639497
:10707000970063742A010504C1BF0545E9BFEFA26B
:107080005FC9AA892E89328BB6843A8ABE8AEF807C
:10709000204C55C12685EF1030368D4763E5A7009B
:1070A0007D556FA09FCA83DB4400EF00D0772A8410
:1070B000EF00B0789307740031443305850263C54F
:1070C000A702EF005076EF0010762A84EF00F076EA
:1070D0009307740031443305850263CDA702EF00A6
:1070E00090749307450019A8EF00307533058502A9
:1070F0001307F0179307C017E357A7FC2D55E3C2FA
:1071000077FB63000B02D6865286A6854A85EFE0A0
:10711000106341BFEF007072330585029307C5FF0E
:10712000F1BF832749001385C90083D52700EFF0FD
:107130001FF071F9B5B76955ADB797F7FF1F239BDE
:10714000A7A097F7FF1F9387A7A0904381470C46FE
:107150003307F500420741836393B70082805446AA
:10716000139847008507C2962390E600D5B797F796
:10717000FF1F9387E79D9C4303C58700828017F517
:10718000FF1F0355259D8280EFA23FBBC167138778
:10719000D7FF6307E5026368A700F117630EF500E8
:1071A00001456FA0DFBB1387E7FF630EE500FD1706
:1071B0001D8D13351500F5B7EF40003D7D15D5BF8A
:1071C000EF40801AE5BFEF40E018CDBFEFA2FFB659
:1071D0004111AA8401442EC6EF00F05FB245634618
:1071E000A400014541016FA09FB79C4813151400EE
:1071F0003E9583570500E387B7FE0504E9BF0348C2
:107200005500814693F7F60F63E5070181473E85F8
:107210008280584593975600BA9703D72700631684
:10722000B70003D70700E304C7FE8506E1BF834626
:10723000450001479377F70F63E4D700814711A812
:107240001C45131657000507B29703D60700E31332
:10725000B6FE3E858280EFA2BFAC93170501C187C1
:1072600097FAFF1F938ACA8E6355F00883A70A0016
:10727000C0479C4703570400198D4205418163664E
:10728000F500014422856FA0FFAC12052A94DDBFF2
:10729000DC4713944900014A3E948347440063410C
:1072A000FA02014A834754006347FA028509C2097A
:1072B00093D9090183A70A009847E3EBE9FCD1B70A
:1072C0001C4413195A00A6853E994A85EFF01FF019
:1072D00011ED050AD9B75C4413195A00A6853E99E9
:1072E0004A85EFF0BFEE19E1050A6DBFE30009FC26
:1072F00051BFAA8481497DBFEFA23FA41C452A84C7
:1073000081E79307C5001CC51C44231204001CC060
:107310009307F00F63E9B70093F5F50F2285EF109F
:10732000B0136FA0DFA393940501C167C18063F719
:10733000F500A6852285EF10D015E5B7C18193F53C
:10734000F50F2285EF105011A6852285EF1010123F
:10735000C9BF97E7FF1F9387A77F884382801C459B
:1073600099C797E7FF1F23A5A77E014582807D551A
:10737000828097E7FF1F9387A77D98438347450047
:10738000484792073E958280EFA23F9B617100457E
:107390001C183EC6B70780013EC81C183ECA83575A
:1073A000440002CE02D002CC231EF10083478400A9
:1073B0002A8902D22301F1023C083ED402D6EFF022
:1073C0005FFB835705002316F102EF30706B230734
:1073D000A1025C4003556400F18313F71700834753
:1073E000F10252055181F99BD98FA307F102EFE019
:1073F000702639C5AA8403550500EF80401683D74F
:1074000004002AD26800231CF10083D72400231D26
:10741000F1001C4803D647008C43EF10100283474D
:10742000B400CA8617460100130686318117A305EA
:10743000F4006C004810EFE090305D616FA03F9267
:107440002155E5BF1C45B1CF03C5A7008946135799
:107450006500630BD7028D46630ED7028546630035
:10746000D702130740063305E50203C7B700418B77
:1074700015CB83C7B700BD8B3355F540828013759C
:10748000F5031307803EC5B709671375F5031307A6
:107490000771D1BF372709001375F5031307077C60
:1074A000D9B701458280EFA25F8903A985006305F2
:1074B00009048347B900AE8493F7070E91CF0345C3
:1074C0009900930520030D810505B305B502884495
:1074D0006105EFF0B0320DA02E85EFF0BFF62A84E3
:1074E00001CD11238325C900B307B54063F8870098
:1074F0002E94B305A440E1FD6FA07F868545C1BFF2
:10750000EFA2BF832A8403D50500011132C636C419
:107510003AC22EC002CA02CC02CEEF80400482459D
:107520002ACA22852ECCEFF0DFE403570500231E84
:10753000E100EF30F054A24632469247230FA100FB
:1075400036874C08B28622850146EFF05FB30561AD
:107550006FA0FF80EFA26FFE61711C183EC6B707D7
:1075600080013EC81C183ECA3C0800453ED4AA848F
:1075700002CC02CE02D002D202D6EFF09FDF8357B8
:10758000050035592316F102EF30904F2307A10271
:1075900009C48357440091E721594A855D616FA072
:1075A0000FFC0355640052055181EFE0B00A2A89AF
:1075B00065D58347B40093F7070E89C71305840187
:1075C000EFF0502583574400231EF10083478400C9
:1075D0002301F1025C4003550900D98313F7070822
:1075E00083471102231CA10093F7F707D98FA3004B
:1075F000F10283572900231DF1005C40F18313F74A
:1076000017008347F102F99BD98FA307F102EF70AE
:1076100010752AD251D18347940068001397570000
:107620008347B400FD8BD98FA305F4001C4803D613
:1076300047008C43EF106060A687174701001307CF
:107640002710740005464C102685EFF05FA32A89A9
:1076500029D58347B400A685FD8BA305F400EFF080
:107660009FE425BFEFA26FED832485FE2A8441119C
:107670002685EFF03FDD834734FF93F7070E9DC368
:107680002AC62685EFF05FD019C9834734FFB2457B
:10769000FD8BA309F4FE81C52285EFF03016410170
:1076A0006FA0EFEB6DDD8327C4FF2685829765F918
:1076B000834734FF93F7070E81C72285EFF09015BB
:1076C000032584FEEFF01FE9D9BFEFA20FE49C4130
:1076D00041112A8903C7070089472E849356670002
:1076E000638CF6020D466382C6049307F0076302BB
:1076F000F7022E85EF10A060AA848149C16B130C9C
:10770000490097E7FF1F9387A7449C43984763EC82
:10771000E90241016FA02FE303D745008547E3FA53
:10772000E7FE2E85EF108061C1BF03D74500E3F26D
:10773000E7FE2E85EF10A05CAA842285EF10805D05
:10774000C204C98C5DBFDC470355A900139A4900E8
:107750003E9A93170501C187635DF00083570A00C5
:107760006395A70263E574038327CA00034D5A009B
:107770001DA0A1672167A98F1307F7EFE374F7FE38
:1077800063950900EFF05FA071FD85099DBF832718
:107790008A00034D4A00835DA90003576900216AEE
:1077A000138BC7003AC6814A33CA4D01631E5D017F
:1077B00097E7FF1F9387473A9C43E1DBA2866286E7
:1077C000814526858297D1B7A1679387F7EF930C00
:1077D0004BFF63F04703B2455A85EFF05F8519CD43
:1077E00003278B00104719CA10436380C402310776
:1077F000D5BFEE856685EFF07F9D71FD93861A00FB
:1078000093FAF60F130B0B0255B7835644005C43F3
:10781000E3EDF6F622853AC6EF10603DA167938747
:10782000D7042A8A035D4400324763E89700834700
:10783000D90093E707F8A306F9001C47668522865E
:10784000E2858297C1670844FD17337AFA005295A2
:1078500008C02312A40115BF97E7FF1F9387472F86
:107860009843814715C31447814763FFD500939719
:1078700045004C47BE9519C903C75500814763753C
:10788000E600DC451606B2973E85828003C74500B8
:107890008147E37BE6FE16069C45F5B7EFA24FC88D
:1078A000AA892E8A814497EAFF1F938A6A2A83A7AE
:1078B0000A00984763E4E4006FA0CFC9DC47139443
:1078C000440001493E9413BB140083474400634BBA
:1078D000F900014913BB140083475400634FF900BA
:1078E0008504F1B70844931759005287DA86014698
:1078F000A2853E9582990509C9BF4844931759004E
:107900005287DA860546A2853E9582990509E9B730
:10791000EFA2AFC2814517F5FFFF1305255F97E77B
:10792000FF1F23990722EFF07FF76FA04FC397E760
:10793000FF1F9387E7219C4381CFEFA20FC08145B2
:1079400017F5FFFF1305855CEFF05FF56FA02FC102
:107950008280EFA2EFBC37E4040083278412411138
:107960002315E100AE893289368A3A86814601477D
:10797000ED45AA8482972AC621C50356A100D28567
:10798000EF1061258327C413CE852685829705894C
:1079900015C58327440D2314210101462C0026859B
:1079A00082972A8401C9B7E7040083A7C712ED456F
:1079B00028008297228541016FA0CFB94944E5B7DD
:1079C0006554CDBF5C41FD175CC18280EFA2EFB66C
:1079D000B7E70400FC5F829795473305F5028145C0
:1079E0000D816FA0CFB7EFA24FB5B7E70400FC5FE2
:1079F000829795473305F5020D816FA04FB6EFA230
:107A0000CFB3B7E7040083A7870B03550500829720
:107A10006FA0EFB4EFA26FB2035505003287AE86B8
:107A200017B6FF1F0356A66B97E5FF1F9385051337
:107A3000EFF03FF26FA0AFB2EFA22FB0B7E70400B4
:107A400083A7C71782976FA08FB1EFA20FAFB7E7D9
:107A5000040083A7871397E5FF1F9385251082975E
:107A600001456FA0CFAFEFA24FADB7E7040083A7EA
:107A7000C71F814517B5FF1F0355656282976FA029
:107A80000FAEEFA28FABB7E7040083A7871397E58C
:107A9000FF1F9385A50D829701456FA04FACEFA204
:107AA000CFA9B7E7040083A7C71F814517B5FF1FFC
:107AB0000355E56482976FA08FAAEFA20FA82E85C9
:107AC000EF600055EF60900D6FA06FA9EFA2EFA6D9
:107AD000EF60D0176FA0AFA85C49E1175CC95CC527
:107AE00083572501A1072319F50083570501A10735
:107AF0002318F5008280F1473305F50297E7FF1F51
:107B00009387C7089C433E9582808D476317F6068E
:107B100003D74600854763F2E706EFA20FA236853A
:107B200036842E89EF10A01D39C183574400931469
:107B30000501C18063ED97022285EF10401CFD1402
:107B4000231294009307A002630EF5009307B0027E
:107B50006301F50293079002631BF5002285EFC0D5
:107B6000B07E31A00146CA852285EF80000F6FA04C
:107B70000F9F2285EF001059DDBF828097E6FF1F1F
:107B8000938606019C42014599CF9843D44217E65B
:107B9000FF1F232FE6FE6396D70097E6FF1F23AB58
:107BA000E6FE1385C7FE8280EFA22F99E926714475
:107BB000330585029145EF70606201E565556FA060
:107BC0000F9A97E7FF1F23A1A7FC752633058502AF
:107BD0009145EF70A0607DD197E7FF1F23A8A7FA1A
:107BE000592E97E7FF1F239BA7F8712697E7FF1FE2
:107BF0002397A7F8974701009387C7B917E7FF1F97
:107C00002322F7F897070000938747ED17E7FF1F38
:107C10002328F7F6014565B7EFA22F92AA8517E54D
:107C2000FF1F1305A5F5EF1060216FA04F93EFA282
:107C3000CF90EFF07FFEEF10E02197E7FF1F9387D3
:107C400027F59C4381CF1387C7FE09CB83D5C7FF98
:107C500017E5FF1F130545F4EFF0403A6FA02F9092
:107C6000EFA2AF8DEFF09FF119C9834785002A84F9
:107C700093F7070499E70355E500EFF05FFB6FA06A
:107C80000F8E8347C5009304450117E9FF1F1309B1
:107C900029F085E3832709005CC997E7FF1F23A923
:107CA00097EE83274900E1FF97E7FF1F23A497EE94
:107CB000F9B7FD172306F5006105EF60E07E830745
:107CC000840063CB07048347840093E707F8230409
:107CD000F400B7E704009C5F82974205A947418101
:107CE0003375F5028347840093F707FCC98F23049B
:107CF000F4008347D4003E951C402318A40089CF8C
:107D0000984319CB8347C40050408145850733050C
:107D1000F502420541810297832709005CC897E775
:107D2000FF1F23A797E68327490089E797E7FF1FEF
:107D300023A297E68347C400B9D38355040117E50E
:107D4000FF1F130565E5EFF0602B15BFEF92FFFEF7
:107D500097E7FF1F938787099C4701448583858B9D
:107D600081EFAE84B2853A86EF1020142A8409C5CB
:107D7000EF10200B829408CC22856F905FFEEF926B
:107D80003FFA41112E8932C6AA89712C3247130657
:107D90000502CA8697050000938525D617E5FF1FC3
:107DA0001305C5DDEFF09FFA2A8429CD9304C500A1
:107DB00065261946AA852685EF0030688545268503
:107DC000EF001065174501001305859A4E95834510
:107DD00005002685EF0050685C4831468145A107C3
:107DE0005CC85CC483572401E1172319F40083574E
:107DF0000401E1172318F4001C4C3E85EF90FFF6B8
:107E0000A3042501228541016F90DFF4EF92FFF278
:107E10004111AA842EC632C4EF100003004DB245B2
:107E20002246834784000CC050C093F7F70393E7C2
:107E300007042304F400231804002685EF00707E55
:107E400083479400A9462317A40013D737000507DA
:107E50003307D7029D8B85072306F400A306E400B1
:107E600083C70401D8488507230FF7FE17E7FF1FD4
:107E7000130707D25843232A0400930744011DEB3C
:107E800017E7FF1F2328F7D017E7FF1F2322F7D09C
:107E900017E4FF1F130444D02285EFF0A00B1C440D
:107EA000858B5D8D09E581452285EFF02015410127
:107EB0006F90FFEA1CC317E7FF1F232DF7CCC9BF44
:107EC000EF92BFE797050000938565C40145EFF089
:107ED000DFBE01456F90BFE8EF923FE6EFF01FBFB6
:107EE0006F90FFE78347C500A1E7EF921FE52A8463
:107EF0000355E500EFF05FD215C98347840093F77F
:107F0000F7FB2304F4001C4091C7DC4381C74C40BD
:107F100001458297EFF09FC617E5FF1F1305C5C700
:107F2000EFF0400F0355E400EFF07FD06F903FE398
:107F30008280EF929FE097E7FF1F938767C59705C1
:107F40000000938525D217E5FF1F1305E5C423A084
:107F5000070023A20700EFE0507E6F905FE01C4D0A
:107F600091CBDC4381CBEF925FDD834507008297A5
:107F70006F90FFDE828097E7FF1F938727C49C43A3
:107F800003C50700828097E7FF1F938727C39C43A1
:107F900003C51700828097E7FF1F938727C29C4382
:107FA00003C52700828097E7FF1F938727C19C4363
:107FB00003C54700828097E7FF1F938727C09C4334
:107FC00003C53700828097E7FF1F938727BF9C4335
:107FD00003C55700828097E7FF1F938727BE9C4306
:107FE00003C56700828097E7FF1F938727BD9C43E7
:107FF00003C57700828097E7FF1F938727BC9C43C8
:1080000003C58700828097E7FF1F938727BB9C43A8
:1080100003C59700828097E7FF1F938727BA9C4389
:1080200003C5A700828097E7FF1F938727B99C436A
:1080300003C5B70011E11D45828097E7FF1F9387B5
:10804000E7B79C4303C5C700828097E7FF1F93876C
:10805000E7B69C4303C5D700828097E7FF1F93874D
:10806000E7B59C4303C5E700828097E7FF1F93872E
:10807000E7B49C4303D50701828097E7FF1F9387EE
:10808000E7B39C4303C52701828097E7FF1F9387CF
:10809000E7B29C4303D54701828097E7FF1F938790
:1080A000E7B19C4303D56701828097E7FF1F938761
:1080B000E7B09C4303D58701828097E7FF1F938732
:1080C000E7AF9C4303C5A701828097E7FF1F938713
:1080D000E7AE9C4303C5B701828097E7FF1F9387F4
:1080E000E7AD9C4303C5C701828097E7FF1F9387D5
:1080F000E7AC9C4303C5D701828097E7FF1F9387B6
:10810000E7AB9C438857828097E7FF1F938707ABB5
:108110009C4303D5C702828097E7FF1F938707AA76
:108120009C4303D5E70219E11305800C828097E791
:10813000FF1F9387A7A89C4303C50703828097E787
:10814000FF1F9387A7A79C43C85B828097E7FF1F09
:10815000938747A68843828097E7FF1F9387C7A529
:108160008843828019E17D558280F5DE984265DF83
:10817000FDD917E7FF1F130767C71847AA8771556F
:10818000058B6319072203C507001547E37DA7FC8C
:1081900003C737001305F0057D171377F70FE36466
:1081A000E5FC03C35700E30003FC83C86700E38CCE
:1081B00008FA03C77700494579171377F70FE36487
:1081C000E5FA03C7A70011481305F7FF1375F50F6C
:1081D000E36BA8F803CE97000D481305FEFF137557
:1081E000F50FE362A8F803C8B70063090800651833
:1081F0001378F80F1305600DE36705F703C5C70093
:10820000794879151375F50FE36FA8F403C8D70003
:108210000D457D181378F80FE36705F503D80701BE
:10822000930E40175118420813580801E3ED0EF35E
:1082300003C8E7007D181378F80FE36605F303C859
:1082400027017D181378F80FE36F05F103C8870045
:10825000C54E75181378F80FE3E70EF103D86701E0
:10826000856E938EBEE06D18420813580801E3EC4A
:108270000EEF03D847016D18420813580801E3E4D4
:108280000EEF03D887017918420813580801E36CF0
:1082900005ED03C8A7017D181378F80FE36505ED18
:1082A00003C5B7011D487D151375F50FE36DA8EAE9
:1082B00003C5D701714879151375F50FE365A8EA71
:1082C00003D5E7011308E00F7D1542054181E36CFA
:1082D000A8E803C50702494879151375F50FE3644B
:1082E000A8E8C85301C937C834005915130858BF46
:1082F000E36BA8E603A8870237C53400130555BF12
:108300005918E36205E717E5FF1F2327C58A03C64F
:10831000050117E5FF1F2323F58A0545E375C5E42D
:1083200003D82501D04933760603E31E06E203C6CF
:108330001501E30A06E217E6FF1F232DB68683C563
:10834000270001466387A50003C61700F1453306E1
:10835000B60283C707039305C00272971A07130773
:10836000C70516031A9796084697B387B702415573
:108370003E97329742074183636EE802EF92FF9B7C
:108380003685EF60D06FEFD0B0212A84EF80B01D2A
:108390002A94EFC090252A94EF7040072A94EFF0BA
:1083A000BF802A94EF2050632A94EF5040662295B4
:1083B0006F90FF9A8280EF925F984111A307A1000E
:1083C000EF80801E9305F10017050000130565B9C5
:1083D000EFF0CFCC014541016F907F98EF927F93F2
:1083E00017E4FF1F130484A00328840079599368BD
:1083F000180097E4FF1F23AF149F13781800631E23
:108400000800BA84BE89368B328A2E89AA8AEFE0A8
:108410001FD67D15269509E531594A856F90FF9243
:10842000EFE0FFD47D152695A167E357F5FE97E7AA
:10843000FF1F9387A7D298433E8C814B11C70145FC
:10844000EFC0B03E933B15004A85DA865686D2854A
:10845000EF7070372A8911CD1C44F99B17E7FF1F75
:10846000232AF79883270C00CDDBE3880BFA829749
:108470006DB7268597E7FF1F23AC0796EFE0FFCB8C
:108480004146CE8517E5FF1F1305C59FEF00A17478
:10849000EFA070080325040BEFA0700A0545EFA0BC
:1084A00070100545EFF03FF18DBF97E7FF1F9387F1
:1084B000E7939C47858BD5C7EF923F8817E5FF1F51
:1084C0001305859A97E7FF1F23A2079297E7FF1FDF
:1084D00023A0079297E7FF1F23AE0790EFE09033AA
:1084E000EF40C002EFE0F00AEFE0700F97E7FF1FE8
:1084F0009387478E9C4381C70545EF60B03397D77C
:10850000FF1F9387E7769C4389C741657D15EF5030
:10851000A06BEFC0703AEFA0F00097E7FF1F9387C2
:10852000E7A19C431397170163540700EFC0A045D0
:1085300097E7FF1F23A8079497E7FF1F23A6079439
:1085400097E7FF1F23A4079497E7FF1F23A2079431
:10855000EFF09F984923EFF0AFBBEFC080676F90BB
:108560001F80828097E7FF1F938747888843828018
:10857000EF92AFFCEF60B07EEF7080006F902FFE47
:10858000EF920FFA2A849304140201112E85B28906
:10859000A685214636C63A89EF0081611DE1B246C3
:1085A00038082686CE8513059404EF4060432146A3
:1085B0002C084A85EF00C15F1335150005616F90E7
:1085C0006FF90145E5BFEF924FF79305450617D5C3
:1085D000FF1F1305E55EEFE070226F904FF8EF92FA
:1085E000CFF541112EC6EFF00FC0B24588C1410151
:1085F0006F90EFF6EF92CFF2AA842E84EF6050785E
:10860000AA8985452285892D83C7E40113899408A9
:1086100099E313890403CE8522853D2D21469305D8
:1086200019022285192D97D7FF1F9387277C8C432A
:108630002285EF00E0682146938584022285F52B90
:108640006F904FF1EF92EFEC3971EFC0E04E930570
:10865000400645EDEF60D06F630E051097D7FF1F02
:1086600083C7C75713B7170097D6FF1F2388E6564F
:10867000014489CFC16417D9FF1F130929779309D2
:10868000400EFD14EFF03F986348A408EFF0AFB53B
:108690004169B7290900096AFD7A2A8B81447D194D
:1086A0009389F97B130A0A71938A8AC7EFF0BF9501
:1086B00063D5A4041304400EB387840217D7FF1FA9
:1086C0001307C7720324070B3E948357C4016386C4
:1086D000270918403307EB4063EAE9008347440069
:1086E0008507B3874703D6976369F7060146814537
:1086F0000945EFF0CFE8AA8B29E1EF20105A854712
:10870000631FF50489659385057117D5FF1F130550
:10871000254BEFE0B00EA1A8B30734030327090BE4
:10872000BA9703D7C7016308970003C75700A3820E
:1087300007002382E7000504B1B79305C500228531
:10874000EFF05FEB5E852286973501009385850308
:10875000EFF0CFEB5E85EF00E06F850481BF97D728
:10876000FF1F9387A7689C478D83858BC1FF21617D
:108770006F90AFDD01468545094502D002D202D493
:1087800002D6EFF0CFDFAA847DD1EFC0203A138963
:10879000C4002A8481454A85C1210C4041464A854E
:1087A000692983294400638809084E8502D802DAC2
:1087B00002DC02DEEF00816A2ACE141005462C0886
:1087C00008184ECCEF4060191375F50F2DE5835551
:1087D000840093E525004A856D2911460C104A85D1
:1087E000A929014697350100938545FA2685EFF0C2
:1087F000EFE12685EF0000665C40B5DB014685456C
:108800000D45EFF0CFD7AA843DD148401389C4006D
:10881000EF00C1642AC64A85C5263246636AC50090
:108820004C404A851929014681452685EFF00FDE27
:1088300026850D252DBF8355840071BFEF92EFCFA4
:1088400097D7FF1F9387875A9C4719CD93E78700D7
:1088500017D5FF1F1305C53617D7FF1F232CF75851
:10886000EFE060786F90AFCFDD9B17D7FF1F23231A
:10887000F758EF2090427DF517D5FF1F13054534BB
:10888000EFE04079C5B7EF92CFC84169AA892E8A37
:10889000B28A368BBA8B814417DCFF1F130C0C5540
:1088A000930C400E7D19EFF00FF663C4A400014451
:1088B0002DA03384940383270C0B3E948357C4016B
:1088C000638027055A87D6865286CE851305040312
:1088D000EFF01FCB11C523800B0022856F90EFC6F0
:1088E0008347F40191CF5A87D6865286CE851305E9
:1088F0009408EFF0FFC809C585472380FB00F1BF4E
:10890000850455B783574500638D0716EF924FC115
:1089100001112A84ED2619C58547630AF50405610E
:108920006F904FC3EFC040217DF983574400494702
:10893000ED9BE396E7FEC14522854524AA84228566
:10894000F52E0357440002CE91472A896317F7009A
:10895000228539293C082ACC3ECEEFC0201D5C552B
:10896000DDDF74084A86A685054582974DBF03570B
:108970004400D147E3F5E7FA032A0400C16901493D
:1089800097DAFF1F938A8A46130B400EFD19EFF00A
:108990008FE76344A90C2285032A04008D26A14594
:1089A0002A8922851D2CAA842285D92614402A864C
:1089B000AA8978082685CA85EFF0FFECAA8425D11C
:1089C00003C7F40189476315F7008347C101A1DBA1
:1089D0005546D28513856400EF00E11F0145EF6025
:1089E000103801C583D7C401B1EB97D7FF1F938718
:1089F000E73F9C4793551900858913D73700058BAE
:108A000011CB8983858B6397B70001452EC6EFF0A4
:108A1000FFE2B2454E85EF60703C0346C1012A84F7
:108A2000937519002685EF70703131C92685EF6086
:108A30007037268511C00145EF60D061EF20F02529
:108A40008547E31EF5EC83C754001307F00FE38856
:108A5000E7EC8507A382F400D9B5B304690383A7C3
:108A60000A0BBE9483D7C401638937015546D2856A
:108A700013856400EF00C11371D1050909BF5DDCE6
:108A80005DBF8280EF92CFA9EF60902C11CDC164C1
:108A9000014417D9FF1F130969359309400EFD14CE
:108AA000EFF06FD6634AA40017D5FF1F13054511D9
:108AB000EFE060536F900FAA330534038327090B4F
:108AC0003E958357C5016386970023120500EF602A
:108AD000702D0504F1B797D7FF1F938727319C4767
:108AE0008D83858B99EBEF924FA517D5FF1F13054B
:108AF000250DEFE020526F908FA68280EF92EFA3BA
:108B000097050000938545B417D5FF1F1305450B46
:108B1000EFE0A0426F90AFA4EF922FA28841B7E799
:108B20000400BC5B050542054181829709C5854764
:108B30002300F50005056F908FA283C7F5FF2E85F2
:108B40008507A38FF5FE828083C7F5FFFD1793F796
:108B5000F70FA38FF5FE99EBEF922F9EB7E7040076
:108B6000BC571385F5FF82976F906F9F82801C41E1
:108B7000035745008D8FBA951CC12312B5003E8561
:108B8000828093D78500A2051441DD8D835745006F
:108B90001387E6FF18C189072312F50013D6850055
:108BA0004111238FB6FEA38FC6FE4101828018417A
:108BB0009307F7FF1CC18357450085072312F50073
:108BC000A30FB7FE8280835745008D8F2312F500D7
:108BD0001C41BE950CC12E858280AA8703D7470011
:108BE00008410D8FAA952392E7008CC3828018411B
:108BF00008453305A7408280835745000357650029
:108C00001D8F1C4108453385A7403305A74082804E
:108C1000EF92AF9241112EC62A84EFF0FFFDB245CC
:108C20006373B50001A0835744000840BE9523122A
:108C3000B4003E9541016F908F92EF920F904111D9
:108C40002E84B28532C6EFF0BFFC3246A285EFF02B
:108C5000907841016F90AF90EF922F8E2E848545D2
:108C6000EFF01FFB230085006F906F8FEF92EF8C6A
:108C700041112317B1008945EFF09FF98347E100C7
:108C80002300F5008347F100A300F50041016F9038
:108C90000F8DEF928F8A93D78500A2054111DD8D4C
:108CA0002317B1008945EFF0BFF68347E1002300A9
:108CB000F5008347F100A300F50041016F902F8A72
:108CC000EF92AF871397850193D78501C16693868D
:108CD00006F0D98F13D78500758FD98FA205370776
:108CE000FF00F98D4111DD8D2EC69145EFF05FF249
:108CF0006C001146EFF0306E41016F904F86EF929D
:108D0000CF831C41854503C40700EFF0DFEB2285CC
:108D10006F90EF84EF926F821C414111894503C728
:108D2000070083C717002307E100A307F100EFF056
:108D30009FE90355E10041016F906F82EF82FFFFD1
:108D40001C414111894503C7070083C7170023074A
:108D5000E100A307F100EFF01FE78357E1004101B5
:108D600013D58700A2075D8D420541816F803FFFCB
:108D7000EF82BFFC0C4141112A8411466800EFF0DC
:108D8000906591452285EFF01FE4B247C166938656
:108D900006F01397870113D58701598D13D78700E4
:108DA000758F598DA2073707FF00F98F5D8D41013F
:108DB0006F80FFFA1C45BE950CC18280AE8794433C
:108DC00091E6584101EF0CC15CC1828003C7570096
:108DD00013671700A382E700B687D5B70CC3EDB7BA
:108DE000AA87084119CD1841D44398C36313D5000D
:108DF000D8C32A87034657009376160081E62320BE
:108E000007008280944381CA8C4203A847008CC328
:108E100063930601CCC3799A14C3A302C7003687B3
:108E2000D1BF1C45DC471D8DB777DBB6938777DB59
:108E300009853305F502420541818280F147B385FA
:108E4000F50248452E958280834745008507230219
:108E5000F5008280EF827FEE2A8419E06F803FF078
:108E600083474400E5DFFD1793F7F70F2302F40073
:108E7000F5F71C4403D7270005072391E700DC43DF
:108E800099C3228582974C4889CD83475400898BAA
:108E900099E71C4422859C479C439C478297232A40
:108EA00004000040232004004DBFEF821FE98357D8
:108EB000250041112EC691E70144228541016F80B2
:108EC0001FEA035705008147F146E307F7FEB38524
:108ED000D702404585072E948345440008C4F5F524
:108EE000B247AA8481E7232A040009A81C456C0024
:108EF00022859C439C43829748C85DDD85472312A9
:108F0000F400B24723200400231804002319F400BE
:108F10005C485CC483D72400FD172391F40071BF23
:108F2000EF82BFE197D7FF1F938787CB8843232624
:108F30000500232405004105EFE0C00D6F803FE2EE
:108F4000EF82BFDF17D4FF1F130484C91C404111F7
:108F500089CF9C472300B5002AC65CC1EFF05FFCB7
:108F60001C40DC4399C33245829741016F803FDF4B
:108F7000034745001DEB584DAA877D550DCBEF8269
:108F8000DFDB1CC3DC4797D6FF1F23ABE6C4F156DB
:108F9000130507012390D7009705000093858501ED
:108FA000EFD0B07901456F809FDB7D558280828054
:108FB000EF82BFD80111614681452800EF80FFDABA
:108FC00097D7FF1F9387C7C19C4328009305F00FD5
:108FD000DC473EC6EFF0DFF605616F805FD897D7BC
:108FE000FF1F9387E7BF9C43D847A1679387C702BA
:108FF0006312F70A397106DE22DC26DA80004AD8CD
:109000004ED652D456D23285B284EFF05FCFAA89C1
:109010002685EFF03FD02318A4FC2685EFF09FCFE4
:109020002319A4FC2685EFF0FFCE83D744000A8ADB
:10903000231AA4FC858393F7F70F230EF4FC86070D
:10904000BD0793F7073F3301F1408A8A01498347FF
:10905000C4FD6365F902CE85130584FC232C54FD01
:10906000EFF01FEE5281130104FCF2506254D2540F
:109070004259B259225A925A216182802685EFF0D4
:109080007FC993171900D69705092390A700137974
:10909000F90F75BF828097D7FF1F938767B49C43F2
:1090A000D847A1679387A7026310F70A397106DED4
:1090B00022DC26DA80004AD84ED652D456D23285E7
:1090C000B284EFF0DFC3AA892685EFF0BFC4FD5755
:1090D0002318A4FC26852319F4FCEFF0BFC383D723
:1090E00044000A8A231AA4FC858393F7F70F230E02
:1090F000F4FC8607BD0793F7073F3301F1408A8AE6
:1091000001498347C4FD6365F902CE85130584FCDC
:10911000232C54FDEFF0DFE25281130104FCF250E6
:109120006254D2544259B259225A925A21618280D1
:109130002685EFF03FBE93171900D69705092390B7
:10914000A7001379F90F75BF828097D7FF1F938708
:1091500027A99C43D847A16789076318F708397185
:1091600006DE22DC26DA80004AD84ED652D456D209
:1091700032853289EFF0BFB8AA894A85EFF09FB9EE
:10918000835749000A8A2318A4FC858393F7F70FB5
:10919000230CF4FC8607BD0793F7073F3301F1402A
:1091A0008A8A8144834784FD63E5F402CE851305F2
:1091B00084FC232A54FDEFF0BFD85281130104FC34
:1091C000F2506254D2544259B259225A925A2161F1
:1091D00082804A85EFF01FB493971400D6978504D8
:1091E0002390A70093F4F40F75BF828097D7FF1FD9
:1091F0009387079F9C43D847A1679387E70463122F
:10920000F70A397106DE22DC26DA80004AD84ED60B
:1092100052D456D23285B284EFF07FAEAA89268529
:10922000EFF05FAF2318A4FC2685EFF0BFAE231A42
:10923000A4FC2685EFF01FAE83D744000A8A2319C9
:10924000A4FC858393F7F70F230EF4FC8607BD0774
:1092500093F7073F3301F1408A8A01498347C4FDF0
:109260006365F902CE85130584FC232C54FDEFF0D1
:109270003FCD5281130104FCF2506254D254425942
:10928000B259225A925A216182802685EFF09FA816
:1092900093171900D69705092390A7001379F90FA2
:1092A00075BF828097D7FF1F938787939C43D847CA
:1092B000A1679387C7046310F70A397106DE22DCC1
:1092C00026DA80004AD84ED652D456D23285B2849D
:1092D000EFF0FFA2AA892685EFF0DFA3FD57231840
:1092E000A4FC2685231AF4FCEFF0DFA283D7440008
:1092F0000A8A2319A4FC858393F7F70F230EF4FC45
:109300008607BD0793F7073F3301F1408A8A014979
:109310008347C4FD6365F902CE85130584FC232CC5
:1093200054FDEFF0FFC15281130104FCF25062546E
:10933000D2544259B259225A925A216182802685CA
:10934000EFF05F9D93171900D69705092390A700AA
:109350001379F90F75BF828097D7FF1F93874788CE
:109360009C43D847A167DD07631BF702EF82FF9C90
:10937000797132853284EFF09F982AC62285EFF00A
:109380007F992311A1022285EFF07F97B245230038
:10939000A1022808EFF0DFBA45616F805F9C8280F0
:1093A00097D7FF1F9387C7839C43D847A1679387AD
:1093B0008704631BF702EF825F98797132853284EC
:1093C000EFF0FF932AC62285EFF0DF942311A1026C
:1093D0002285EFF0DF92B2452300A1022808EFF0CA
:1093E0003FB645616F80BF97828097C7FF1F938705
:1093F000277F9C43D847A1679387A704631CF70086
:10940000EF82BF93011128008145EFF07FB3056122
:109410006F80FF94828097C7FF1F9387677C9C4370
:10942000D847A167938757026311F702EF82FF9035
:1094300001113285EFF0BF8C2308A100814528007F
:10944000EFF01FB005616F809F91828097C7FF1F6B
:10945000938707799C43D847A1679387E702631FE7
:10946000F702EF829F8D011132853284EFF09F8ADF
:10947000AA842285EFF01F8A854719E52285EFF03F
:109480001F884205B337A0002800814523189100AA
:109490003ECAEFF0FFAA05616F807F8C828097C77C
:1094A000FF1F9387E7739C43D8479947631FF704CF
:1094B000EF82BF88797132853284EFF05F842AC6EB
:1094C0002285EFF03F852310A1022285EFF03F8334
:1094D0002301A1022285EFF09F82A301A102228530
:1094E000EFF0FF812302A1022285EFF05F812313B9
:1094F000A1022285EFF0BF80B2452314A102280803
:10950000EFF01FA445616F809F85828097C7FF1F82
:109510009387076D9C43D847A1679387C703631F51
:10952000F704EF829F81797132853284EFF02FFD4D
:109530002AC62285EFF00FFE2310A1022285EFF04C
:109540006FFD2311A1022285EFF06FFB2302A10220
:109550002285EFF0CFFAA302A1022285EFF02FFAC5
:109560002303A1022285EFF08FF9B245A303A102E4
:109570002808EFF0FF9C45616F806FFE8280EF82CC
:10958000CFFB01112A84EFF08FF7AA842285EFF038
:109590006FF82285EFF00FF8035744008D4763F50D
:1095A000E7002285EFF00FF72285EFF0AFF62800F5
:1095B000A685EFF0FF9805616F806FFA97C7FF1FD0
:1095C000938707629C43D847A167FD076319F7009B
:1095D000EF82AFF63285EFF09FFA6F804FF882800E
:1095E00097C7FF1F9387C75F9C43D847A167E507CD
:1095F0006311F706EF826FF4797132853284EFF0F0
:109600000FF02AC62285EFF0EFF02285EFF08FF001
:109610002310A1022285EFF0EFEF520551812311B3
:10962000A102228523020102EFF06FEDA302A10245
:109630002285EFF0CFEC2303A1022285EFF02FEC7F
:10964000B245A303A1022808EFF09F8F45616F8008
:109650000FF1828097C7FF1F938787589C43D84795
:10966000A1679387E7036319F700EF820FED328557
:10967000EFF0FFF06F80AFEE828097C7FF1F9387F8
:1096800027569C43D847A167938747046314F70282
:10969000EF82AFEA797132853284EFF04FE62AC665
:1096A0002285EFF02FE7B2452808EFF07F8945616A
:1096B0006F80EFEA828097C7FF1F938767529C43B2
:1096C000D847A167938787026316F702EF82EFE618
:1096D000797132853284EFF08FE22AC62285EFF06D
:1096E0000FE2B2452300A1022808EFF07F85456113
:1096F0006F80EFE68280EF824FE40111EFF02FE000
:10970000AA852800EFF0DF8305616F804FE597C7DA
:10971000FF1F9387E74C9C43D847A167D107631984
:10972000F700EF828FE13285EFF0FFFC6F802FE3CF
:10973000828097C7FF1F9387A74A9C43D847A1679A
:10974000C5076319F700EF824FDF3285EFF0BFFAEC
:109750006F80EFE0828097C7FF1F938767489C4325
:10976000D847A167B9076319F700EF820FDD32858B
:10977000EFF07FF86F80AFDE828097C7FF1F93877F
:1097800027469C43D847A167AD076319F700EF82CE
:10979000CFDA3285EFF03FF66F806FDC828097C7BB
:1097A000FF1F9387E7439C43D84789476310F7021D
:1097B000EF82AFD80111328532C8EFF04FD4AA85BD
:1097C0002800EFF0EFF705616F806FD9828097C7AF
:1097D000FF1F9387E7409C43D847A1678D07631716
:1097E000F702EF828FD5011132853284EFF02FD14D
:1097F00013066100AA844C002285EF20D00C2800BB
:10980000A685EFF0EFF305616F806FD5828097C773
:10981000FF1F9387273D9C4381CBDC4391C7EF8299
:10982000CFD182976F80AFD38280EF820FD17971D1
:109830003C08AE843ED2A165B7070A002A843ED414
:1098400048103C08DD053ED636C432C63AC2EFD0D9
:10985000BFAA12474810BA85EFF00FC03246481031
:10986000B285EFF0AFC0A2464810B685EFF0CFBE8C
:10987000501001478146A6852285EFD07FC84561FB
:109880006F80EFCDEF826FCB01117C000329C50102
:10989000AE843ECAA165B70707002A843ECC4808BB
:1098A0007C00C5053ECEEFD03FA58345D9004808D2
:1098B000EFF08FBA500801478146A6852285EFD088
:1098C0003FC405616F80AFC9EF822FC783C7950082
:1098D00093F7F707A384F500EFF0DFFA6F802FC846
:1098E000EF82AFC579713C08AE843ED2A165B7075F
:1098F00009002A843ED448103C08938545043ED68E
:1099000032C636C4EFD05F9FA2464810B685EFF04E
:10991000AFB432464810B285EFF04FB55010014752
:109920008146A6852285EFD0BFBD45616F802FC3DC
:10993000EF82AFC083C7950041112A8493F7F707E0
:10994000A384F50032852EC6EFF0CFBC85672AC40C
:10995000637CF500EF50B0402246B24509E911475B
:1099600081462285EFF07FEC41016F804FBF0147B8
:109970008346F501FDB7EF82AFBA01113C003ECA44
:10998000B7070A003ECC3C003ECE83C79500AA89AB
:10999000328593F7F707A384F5002E84EFF08FB795
:1099A00085676371F504A165AA84938585044808D9
:1099B000EFD09F942685EF50903A2A891DE5914576
:1099C0004808EFF06FA9A6854808EFF02FAACA85CE
:1099D0004808EFF06FA8014781465008A2854E85E0
:1099E000EFD01FB205616F80EFB681454808EFF0F8
:1099F000AFA603490902C1BFEF828FB279711C1073
:109A00003ECAB7070F003ECC404D1C10AA84AE8959
:109A10004808994532C636893ECEEFD0FF8D324692
:109A20004808B285EFF04FA363040902A545480832
:109A3000EFF00F9E2546CA85EFF0E0195008014768
:109A40008146CE852685EFD0BFAB45616F808FB054
:109A50008355C4024808EFF06FA10355E402814525
:109A600015C185478545630FF500C167FD1793054F
:109A7000F00F6309F5007D15EF5020749305150074
:109A800093F5F50F4808EFF02F9D83450403480830
:109A9000EFF08F9C834514034808EFF0EF9B83554C
:109AA00024034808EFF08F9C835544034808EFF0E7
:109AB000EF9B69B7EF826FA883C795008146014687
:109AC00093F7F707A384F500EFF01FF36F802FA93A
:109AD000EF82AFA679713E841C103ECA2E89B7076B
:109AE0000F00A1653ECCFD051C10AA84480842C0A9
:109AF0003AC23ECE36C432C6EFD01F803246480846
:109B0000B285EFF06F95A2464808B685EFF00F9644
:109B100012474808BA85EFF06F95024863040802BF
:109B200091454808EFF0CF8E1146A285EFF0A00ACC
:109B3000500801478146CA852685EFD07F9C456144
:109B40006F80EFA189454808EFF08F8C83470400B0
:109B50002300F50083471400A300F500D1BFEF8276
:109B60002F9C83C7950001112A8A93F7F707A384D6
:109B7000F5003285AE8432C6EFF0CF9932462A899D
:109B80003285EFF0CF978567637FF900AA894A8510
:109B9000EF50F01C2A8419E9114781464A86A685B0
:109BA0005285EFF09FC805616F80CF9A9387E9FFD8
:109BB00093F7F70F0547E368F7FE8347F50195E74D
:109BC0008947E382F9FE8346F401528501474A86BC
:109BD000A685EFF09FC5A167D90748083ECC230AA8
:109BE000010002CEEFF0BFC27DBF639CE700894752
:109BF000639CF90093071020231FF500EF50901A83
:109C0000D9B70947E391E7FC8D47E39EF9FA22852E
:109C1000EF50D03B97C7FF1F9387C71B9C4399E723
:109C200097C7FF1F9387C7049C4389C703D50400C8
:109C3000EF60300C231F04002285C9B7EF82EF8F3D
:109C400001113C003ECAB7070B003ECC3C003ECEA3
:109C500083C795002A89328593F7F707A384F50017
:109C6000AE84EFF02F8B93170501C187635EF0047C
:109C7000A1652A849385E5024808EFD0EFE7A28525
:109C80004808EFE0BFFE97C7FF1F938767FE9C431E
:109C90009DEF01449375F40F4808EFE0FFFB9355E7
:109CA000844093F5F50F4808EFE01FFB93550441FE
:109CB00093F5F50F4808EFE03FFA01478146500859
:109CC000A6854A85EFD0DF8305616F804F894165A6
:109CD00085460546A2857D15EF3070675DD9510533
:109CE000EFD04027130440063344850265B7EF8266
:109CF000CF840111B70706003EC683C795002164D3
:109D00002A8993F7F707A384F500AE84280093050A
:109D1000A4040AC40AC8EFD02FDE300001478146F0
:109D2000A6854A85EFD0CFFDEFE02FF81304940409
:109D3000480822CC230A010002CEEFF05FAD056196
:109D40006F80EF81EF72DFFDC1642A89014497C9FA
:109D5000FF1F9389A909130A8002FD14EFE0AFAB3E
:109D60006345A40001456F70FFFEB307440303A7DA
:109D7000C90ABA9703D707006306970083D727005D
:109D8000638427010504D9BF0545F1BFEF725FF970
:109D90002A8A2E8999C123A005008149814497CA46
:109DA000FF1F938A6AE4614BEFE02FAD63C5A40007
:109DB0004E856F703FFA3384640383A70A003E9494
:109DC0008357040099E76304090023208900850470
:109DD000E1BF4146D28513054400EFE0705D65F9AF
:109DE000A289F5B7EF72DFF339717C083ED4B7076B
:109DF0000A003ED67C083ED883C795002A8A328561
:109E000093F7F707A384F5002E8932C6EFE09FF0A1
:109E100085676373F5063246AA843285EFE03FEE2C
:109E20008547AA8963EAA704A1659385850428105C
:109E3000EFD08FCC2685EF5080722A8429E191459E
:109E40002810EFE07FE1A6852810EFE03FE2CE8505
:109E50002810EFE07FE0014781463010CA85528527
:109E6000EFD00FEAA1679387770448183EDC230AF6
:109E7000010202DEEFF0BF9921616F70BFED8145F5
:109E80002810EFE07FDDA6852810EFE03FDE97C7C2
:109E9000FF1F9387672C9C4391C722856387090026
:109EA000EFB0600C8345040265B7EFB0200BDDBF57
:109EB000EF721FE783C795004111AA8993F7F7074F
:109EC000A384F5003285AE84328AEFE0BFE4856773
:109ED000637BF5022A89EF5080682A84914621C16C
:109EE0008347F50105476383E70291C70D47636E1A
:109EF000F702AD462DA09305050303250A00414650
:109F0000EFE0104B1DE141016F70DFE49305950810
:109F100003250A004146EFE0B049814679F94A86B7
:109F2000A6854E85EFF0DF9BF9BF83250A00130558
:109F30009408EF60600119C1C146D5B797C7FF1FEC
:109F4000938747E99C4399E797C7FF1F938747D2B9
:109F50009C4389C72285EF60A05479FD8547A30FF4
:109F6000F4002285EF80B05D2285EF50A0634E851E
:109F700081464A86A685EFF0BF96A167938757046E
:109F800048003EC42302010002C6EFF05F88A5BF6F
:109F9000EF723FD883C795004111AA8993F7F7075D
:109FA000A384F50032852E89B28AEFE0BFD685679B
:109FB0006370F50CAA84EF50805A2A841DE9416B26
:109FC000014A97CBFF1F938B6BE2130C400E7D1B56
:109FD00019A833048A0383A70B0B3E948357C4014B
:109FE000638D6703050AEFE00F82E344AAFE9546FE
:109FF00039A88357C501639297029305050303A50A
:10A000000A004146EFE0D03A994611E181462686A2
:10A01000CA854E85EFF0DF8CA1A883A50A00130541
:10A020000403EF507072C1467DF12285231E940017
:10A03000EF80F0502285EF50E05697C7FF1F9387BF
:10A04000A7119C438DCB230004022285EFA09061D1
:10A050004E8581462686CA85EFF09F88A167938743
:10A06000070448003EC42302010002C6EFF02FFAA5
:10A0700041016F709FCD89472300F402D1BF397130
:10A0800006DE22DC4AD8800052D456D25AD026DAD4
:10A090004ED65ECE2E8A32892A8BEFD0DFF30605AC
:10A0A000710541998A8A3301A140232224FC23149B
:10A0B00004FCEFD05FF283479A000605350593F75D
:10A0C000F7072315A4FCA304FA004A85232624FCE1
:10A0D000EFE05FC493170501C1876340F00256812A
:10A0E000130104FCF2506254D2544259B259225A1C
:10A0F000925A025BF24B21618280AA844A85EFE08A
:10A100007FC1AA894A85EFE0FFC0A1659385C5029A
:10A110002A89130544FCEFD02F9E2685EFD0AF93FC
:10A12000854501C94A86CE85EFD06F8DAA8B15ED86
:10A130008945130544FCEFE03FB2A685130544FCB6
:10A14000EFE0DFB2CE85130544FCEFE03FB2CA85F5
:10A15000130544FCEFE09FB101478146130644FC20
:10A16000D2855A85EFD0CFB99DBF8145130544FCF8
:10A17000EFE09FAEA685130544FCEFE03FAFCE8530
:10A18000130544FCEFE09FAECA85130544FCEFE0E5
:10A19000FFAD8144EFD03FE4E3D0A4FC83A70B01E3
:10A1A00013971400BA9783D5070089C5130544FC9B
:10A1B000EFE0DFAB8504F9BF797106D622D44AD02F
:10A1C00000184ECE52CC56CA26D25AC8AE89328911
:10A1D000AA8AEFD05FE00605690541990A8A330132
:10A1E000A140232A24FC231C04FCEFD0DFDE83C71C
:10A1F000990006052D0593F7F707231DA4FCA384FA
:10A20000F9004A85232E24FCEFE0DFB09317050107
:10A21000C187634FF0005281130104FDB2502254F4
:10A2200092540259F249624AD24A424B45618280B5
:10A23000AA844A85EFE01FAEA1659385A5022A890D
:10A24000130544FDEFD04F8B2685EFD0CF80854599
:10A2500019C5CA85EFC0BFFD2A8B0DE989451305D5
:10A2600044FDEFE07F9FA685130544FDEFE01FA0AE
:10A27000CA85130544FDEFE07F9F01478146130621
:10A2800044FDCE855685EFD0AFA771B78145130544
:10A2900044FDEFE07F9CA685130544FDEFE01F9D84
:10A2A000CA85130544FDEFE07F9C8144EFD0BFD207
:10A2B000E3D5A4FC83270B0113971400BA9783D529
:10A2C000070089C5130544FDEFE05F9A8504F9BFD7
:10A2D000EF72BFA683474500404DD5E7FD574DC0FF
:10A2E000834694000947636DD7080346B40085464A
:10A2F00063E8C6088306E40063C406085C45F956B3
:10A300002390D70097C7FF1F83C7478E99E3A30405
:10A31000E40097C7FF1F9387A7959C4381E7894770
:10A32000A306F40097C7FF1F938707E39C4381E7C9
:10A3300089472306F4009705000093854505AA8404
:10A3400013050401EFC0703FFD57231AF402814743
:10A350001CDC014897C7FF1F23A6878897C7FF1FEC
:10A3600093878788232E040304C08043EFD0FFD057
:10A3700061463306C50281452285EF701F9F8147E4
:10A380003E856F70DF9DFD57E5BFEF721F9B2A84EE
:10A3900003554502EF50A01C09E5231E04006F7011
:10A3A0001F9C8357E401E5DF930504FF17150100A7
:10A3B00013058577EFB01063DDB7EF721F982E8914
:10A3C000A16541119385E5032A8436C432C6BE8453
:10A3D0003AC2EFC07FF212472285BA85EFE0DF87ED
:10A3E00032462285B285EFE07F88A2462285B68577
:10A3F000EFE0DF87630D090091452285EFE05F8183
:10A400001146A685EFE0207D41016F705F9589457B
:10A410002285EFE0EFFF83C704002300F50083C728
:10A420001400A300F500CDB7EF723F9183C79500EC
:10A43000444D054793F7F707A384F5001C424111EB
:10A4400083C70700636DF7042E842A8985CC03C770
:10A45000D4006309F70217C7FF1F1307678118436A
:10A4600001CFA386F400EF80902B83C7D40089E747
:10A4700041657D15EF30407583D72403918B99C3D7
:10A48000EFB0B0624A85A285EFF0CFBFA167C107E8
:10A4900048003EC42302010002C6EFF04FB741015D
:10A4A0006F70FF8BEF727F8903D745008D47AA84B9
:10A4B00041112E8432892E8563EDE700EFE09F8500
:10A4C000AA85230009002685EFC07FD641016F7061
:10A4D0001F89EFE03F842AC62285EFE0BF83B245A3
:10A4E00085472A862300F9002685EFC05FD1F9BF92
:10A4F000397106DE22DC26DA80004ED652D456D2DE
:10A500004AD85AD05ECEAE89B284AA8AEFD0BFAB09
:10A5100006051305250241990A8A3301A140232229
:10A5200024FC231404FCEFD01FAA83C7990006055E
:10A530004D0593F7F7072315A4FCA384F90026859E
:10A54000232624FCEFE00FFD93170501C18763402C
:10A55000F0025281130104FCF2506254D254425969
:10A56000B259225A925A025BF24B21618280AA8B25
:10A5700003AB0400EFC03FCE35E983D74400014967
:10A580008544F11793B71700A301F4FC834734FC0B
:10A59000A165BDC79385E504130544FCEFC0DFD575
:10A5A000A685130544FCEFE02FEBDE85130544FC84
:10A5B000EFE0CFEB834734FC114691E30946DA859F
:10A5C000130544FCEFE06FE7814463080900416B29
:10A5D0007D1BEFD05F9F63C8A4020147814613062D
:10A5E00044FCCE855685EFC0BFF1A5B7A6851306FE
:10A5F00034FCEFF03FEB933415002A89860479B7D9
:10A600009385C50451BF8327C90013971400BA97D7
:10A6100083D5070063866501130544FCEFE00FE571
:10A62000850445BFEF72EFEE79711C103EC4B70789
:10A630000F003EC61C103EC883C79500AA8A32850B
:10A6400093F7F707A384F500AE893284EFE08FEC2F
:10A6500093170501C1876350F0062A8A2285EFE02F
:10A660006FEB2A895285032B0400EFC0DFBE39E56A
:10A670008357440081440544F11793B71700A3039F
:10A68000F10083457100DA872287CA865286280046
:10A69000EFF0BFD2014781463000CE855685EFC02E
:10A6A0003FE6A1679387D70348083ECC230A810081
:10A6B00026CEEFF0CF9545616F702FE9A285130686
:10A6C0007100EFF03FDEAA84094445DD3544E30A1A
:10A6D00055FB4A85EFF00FE70D4445D50144EFD017
:10A6E0009F8E634BA400C16B0144FD1BEFD0BF8D57
:10A6F000634EA400154471B7DC4413171400BA97D5
:10A7000083D70700638127030504D1BFD84493177B
:10A710001400BA9703D70700631977012390270124
:10A720002685EF80C0540144A9BF0504C1B7EF726C
:10A730002FDF83C7950041112A8A93F7F707A38477
:10A74000F50032852E893284EFE0CFDC93170501C6
:10A75000C187635BF004AA892285EFE0AFDB231198
:10A76000A1004E85832A0400EFC0FFAE29E1835784
:10A77000440085440144F11793B71700A300F1008A
:10A780000348110003572100D6875285CE862686BE
:10A79000CA85EFF0EFB3A167F10748003EC423027A
:10A7A000910022C6EFF0AF8641016F70AFDAA2854B
:10A7B00013061100EFF01FCF2A84894471D183570B
:10A7C000210011678544BA97C2071167C183130737
:10A7D000F7EFE367F7FA97B7FF1F9387A75F9C43ED
:10A7E00091C7854513052100EF40300E83552100A8
:10A7F00022858144EFC09F9D41D52310050022850D
:10A80000EF808048B5BFEF72CFD083C7950041116C
:10A810002A8B93F7F707A384F50032852E8A3284BA
:10A82000EFE04FCF93170501C1876359F004AA8A5F
:10A830002285EFE02FCE2A895685832B0400EFC0B6
:10A840009FA121E18357440081440544F11793B748
:10A850001700A301F10003483100DE875A854A87BB
:10A86000D6862286D285EFF0AFA6A167ED07480015
:10A870003EC42302810026C6EFE07FF941016F70DC
:10A88000CFCCA28513063100EFF0DFC1AA840944C2
:10A8900079D19167CA97C2071167C1831307F7EF90
:10A8A0000544E36AF7FACA85EFC05F92014445F5B3
:10A8B0008149EFD04FF263DBA900984893971900C4
:10A8C000BA9703D7070015E723902701EFD0AFF021
:10A8D0001544E382A9F82685EF80003B97B7FF1F58
:10A8E0009387474F9C430144BDD74A85EF4040764C
:10A8F0009DB785097DBFEF72AFC279713E847C0838
:10A900003EC82E8AB7071400A1653ECAE5057C083B
:10A91000AA89080836C4428932C6BA8AC6843ECC9F
:10A92000EFC09F9DCA850808EFE00FB332460808C4
:10A93000B285EFE0AFB3A246630E09029D45080859
:10A94000EFE00FAD1D468145EF702FC263870A0609
:10A9500091450808EFE0CFAB1146A685EFE0A027B0
:10A96000100801478146D2854E85EFC07FB9456109
:10A970006F704FBEB6850808EFE04FAF1C40080867
:10A98000D8439355C701858912075183B205D98DE4
:10A99000EFE0CFAD1C40080883C58700EFE0CFABE8
:10A9A0001C40080883C5A700EFE00FAB1C40080857
:10A9B00083C59700EFE04FAA51BF89450808EFE033
:10A9C0002FA583C704002300F50083C71400A3004C
:10A9D000F50079B7EF72CFB483C795004111AA890A
:10A9E00093F7F707A384F5003285AE843284EFE055
:10A9F0006FB293170501C1876357F0042A89032AB0
:10AA00000400EFC05F8519E9835744000548F1173A
:10AA100093B71700A307F100814621A81306F100A0
:10AA2000A285EFF03FA81DC11C459DC383D64700FA
:10AA300001480347F10093078500D2884A86A6851E
:10AA40004E85EFF05FEB41016F70CFB00948E9B779
:10AA50001D48D9B7EF72CFAC65715C083EC4B7072B
:10AA60007B013EC65C083EC883C795002A8A3285B2
:10AA700093F7F707A384F500AE89EFE04FA883575B
:10AA8000E100C5C389452800EFC01F878145280024
:10AA9000EFE08F9CEFC0FF8B97B7FF1F9387C76BCB
:10AAA0009C4317B4FF1F03446414AA84333480000A
:10AAB00099C31364240097B7FF1F9387671B9C43B8
:10AAC00099C31364440097B7FF1F9387A7309C4333
:10AAD00099C31364840083D5040028000149EFE082
:10AAE000EF9883D524002800EFE04F9883D54400E9
:10AAF0002800EFE0AF97EFD00FC993150501C18192
:10AB00002800EFE0AF96A2852800EFE02F969C4446
:10AB1000636CF900014781463000CE855285EFC055
:10AB20003F9E59616F700FA3DC4413144900280045
:10AB30003E94EFE06F8C834744000347540089073D
:10AB40000607BA978607E36EF5FC835524002800B4
:10AB5000814AEFE0AF91834544002800EFE0CF8FBA
:10AB6000834554002800EFE02F8F8347440063C9DA
:10AB7000FA00814A8347540063CFFA00050941BFB8
:10AB80001C4413975A002800BA9783D50700850AFA
:10AB9000EFE0CF8DD9BF032BC40093975A00280054
:10ABA0003E9B83552B00850AEFE04F8C83550B00AD
:10ABB0002800EFE0AF8B7DBFEF722F985C4993E7E1
:10ABC00017005CC9EF8020336F706F99EF72EF96BA
:10ABD0002E848145EFF08F9B05C183570500FD173B
:10ABE0002310F50009C4835725002310F400EFF06B
:10ABF000BFFC01456F70AF9631456DDC231004003A
:10AC0000D5BFEF72EF9183C7950041112A8A93F760
:10AC1000F707A384F50032852E893284EFE08F8F09
:10AC200093170501C187635EF004AA89C145228597
:10AC3000EFD0BFFA2A8B4E85832A0400EFC0AFE124
:10AC400021E583574400231101000544F11793B710
:10AC50001700A300F10081440348110003572100AD
:10AC6000D6875285CE862286CA85EFE07FE6A16729
:10AC70009387170248003EC42302810026C6EFE0F6
:10AC80001FB941016F700F8D13061100A285EFF0FF
:10AC90007F81AA8409E523110100094475BF93054A
:10ACA00021005A85EFF09FF2835721002A84CDD7E7
:10ACB00097B7FF1F938707129C4391C785451305DC
:10ACC0002100EF4080408355210026853144EFC0AC
:10ACD000EFCF59D1231005002685EF70F07A01449B
:10ACE000A5BFEF728F8541112E896C00AA8402C620
:10ACF000EFF0CF8909CD0357050005072310E500C4
:10AD0000EFF09FEB81473E8541016F704F853247E1
:10AD1000954775DBCA852685EF20D008C147E344F7
:10AD200005FE3244854741462310F400835709004D
:10AD3000A685130544002311F400EFD0D0692285C5
:10AD4000C1B7EF62FFFD83C795004111AA8A93F74F
:10AD5000F707A384F5003285AE893284EFD09FFBDC
:10AD600093170501C187635EF0042A8AC1452285D5
:10AD7000EFD0BFE6AA845285032B0400EFC0AFCD0D
:10AD800021E583574400231101008544F11793B74F
:10AD90001700A300F10001440348110003572100EC
:10ADA000DA875685D2862686CE85EFE07FD2A167E8
:10ADB0009387070248003EC42302910022C6EFE0B9
:10ADC0001FA541016F601FF9A28513061100EFF066
:10ADD0006FED2A8409E523110100894475BF26859A
:10ADE00093052100EFF0FFEFAA845DF58355210064
:10ADF0002285EFC0AFBD4DF10149EFD0CF9D635D1E
:10AE0000A900184893171900BA9703D707001DE740
:10AE1000035721002390E700EFD0EF9B6302250347
:10AE200097B7FF1F938707FB9C4389C703552100F2
:10AE3000EF4000222285EF703065B9BF050975BF6C
:10AE4000954499BF05C19307F00F630FF500C547FF
:10AE5000630CF5009307F5FF05453315F500420532
:10AE6000418182800145828041657D158280B9E102
:10AE7000EF62BFEC034506033284EFF0BFFC93059D
:10AE8000803EB305B502C205C18191C90357E402F2
:10AE9000854763F6E70013050401EFC020168357CA
:10AEA000E40241677D176385E700FD172317F4026D
:10AEB0006F60FFEA8280EF62DFE5004283C79500A2
:10AEC000444D0349140093F7F707A384F500834723
:10AED0000400220911673369F900A167B347F9003B
:10AEE00041112A8BAE8A63ECE70C834724001307D9
:10AEF000C00EB91793F7F70F6371F70E03473400CD
:10AF0000C14763ECE70C834744001307E00793C78E
:10AF100007086373F70A8349840083477400A20912
:10AF2000B3E9F900856763F9F908034A64008347C8
:10AF300054004E85220A336AFA00EF40406245C150
:10AF400023962403834B3400137AFA00239A3403A4
:10AF5000238874032399440393890401631A090025
:10AF600023A60402239804024E85EFC0A00A1DA068
:10AF7000034924004A85EFF0FFEC2397A40283479E
:10AF800044004E85A388F402E3810BFEE30F09FC25
:10AF9000EFC06005EF70907981460146D6855A85ED
:10AFA000EFE09FA5A167938797033EC423020100AA
:10AFB000480002C6EFE0BF8541016F601FD985449C
:10AFC000A2862686D6855A85EFE01FA3A1679387C0
:10AFD00097033EC423029100E1BFBD44D5B791441D
:10AFE000C5B7EF62FFD301111C08404D3EC2B70741
:10AFF0000F003EC41C083EC62A89AE89EFC01F9DC3
:10B00000585C1C5C634CB70A6394E50063E8A70ACC
:10B010003385A740B3B7A700B305B7401306803EFA
:10B0200081469D8DEFD0407B93140501C180A165C1
:10B030009385C5034800EFC02FAC81454800EFD091
:10B04000BFC1835504044800EFD05FC28355240478
:10B050004800EFD0BFC1814599C8C167FD1793056E
:10B06000F00F6386F4002685EF402015AA8548007E
:10B07000EFD09FBE03554404814511C9C167FD1738
:10B080009305F00F6305F500EF402013AA854800F3
:10B09000EFD09FBC834564044800EFD0FFBB8345DD
:10B0A00074044800EFD05FBB500001478146CE8555
:10B0B0004A85EFC0EFC405616F60DFC9814485BF79
:10B0C000EF62BFC783C7950093F7F707A384F50026
:10B0D000EFF03FF16F60BFC8EF629FC483C7950078
:10B0E0004111404D93F7F707A384F5002A8A328572
:10B0F000B284AE89EFD01FC22A8B2685EFD09FC1C4
:10B100002A892685EFD0BFBF93170B0163CA0702B8
:10B11000E177CA97C207C183116763E3E702930728
:10B120000910C207C1831307B00F637BF7009317A1
:10B130000901C187AA8A6348F000C54763FA57012D
:10B1400041016F603FC1EFC08F83E31B25FFF5B75F
:10B1500063060B0263040902814463870A02B7078E
:10B160007F0023106405231124057CC05685EFF071
:10B170007FCD9304803EB304950239A0B7077F00CA
:10B18000232004047CC0814403552404EFB0101034
:10B1900095CCEFC0BF83269593D7F4413337950004
:10B1A000AE97BA9708DC5CDCCE855285EFF07FE382
:10B1B00099E023220404A1679387B70348003EC4A3
:10B1C0002302010002C6EFE08FE49DBF81470148E2
:10B1D0001CDC232E0403C9BFEF623FB6EFC0FFE9BA
:10B1E000E1473305F5029145EF30507FE55711C532
:10B1F00097B7FF1F23AAA79E81473E856F603FB682
:10B20000854717B7FF1F2303F79E8280EF62FFB2C7
:10B2100097B7FF1F9387079D80432DC08357040472
:10B22000639EA70483572404639AB7043689B284C3
:10B23000EFC0CFF95C5C63C3B7046395B7001C5CD7
:10B2400063EEA7028347640463F3F400A687230335
:10B25000F4048347740463F39700A687A303F404FC
:10B260008357440441677D176385E70085072312F0
:10B27000F4043C4481C7CA85268582976F603FAE3F
:10B2800097B7FF1F938707969C43014599C303C552
:10B2900087008280EF627FAA0111B70707003EC6D0
:10B2A00083C79500584D0AC493F7F7070AC8A384CB
:10B2B000F5002A89AE8401CB1C4283C70700230412
:10B2C000F700EF70D0452164930554022800EFC0C9
:10B2D000AF82EFF0FFFAAA852800EFD0FF97300089
:10B2E00001478146A6854A85EFC08FA11304440219
:10B2F000480822CC230A010002CEEFE04FD10561BD
:10B300006F60FFA5EF627FA301117C003ECAB70703
:10B3100007003ECC7C003ECE83C795002E84AA84D5
:10B3200093F7F707A384F500A165938555024808B4
:10B33000EFB09FFCEFF0DFF4AA854808EFD0DF9173
:10B34000500801478146A2852685EFC06F9B0561A5
:10B350006F60FFA097B7FF1F9387C7889C4309457D
:10B3600099C303C59700828097B7FF1F938787878C
:10B370009C43094599C303C5D700828097B7FF1F37
:10B38000938747869C43014599C303C5A7008280E4
:10B39000EF621F990111B70708003EC683C79500E9
:10B3A000404D0AC493F7F7070AC8A384F5002A8919
:10B3B000AE8429C01442854703C7060063EEE70642
:10B3C0008347940009468149638EC700B307F7405D
:10B3D000A304E400B339F00083C716002305F4008A
:10B3E000EF70F03303572403058B09C7638409000A
:10B3F000EFA0B06B2164930584022800EFB0DFEF6B
:10B40000EFF05FF5AA852800EFD01F85EFF01FF75A
:10B41000AA852800EFD05F84014781463000A685C9
:10B420004A85EFC0EF8D13047402480822CC230A2A
:10B43000010002CEEFE0AFBD05616F60BF91EF622A
:10B44000DF8F01117C003ECAB70708003ECC7C00AC
:10B450003ECE83C795002E84AA8493F7F707A38472
:10B46000F500A165938585024808EFB0FFE8EFF08D
:10B470007FEEAA854808EFD02FFEEFF03FF0AA85B7
:10B480004808EFD06FFD500801478146A285268508
:10B49000EFC00F8705616F609F8C97A7FF1F938791
:10B4A00067749C43014599C303C5B7008280EF626E
:10B4B000DF880111B70707003EC683C79500404DDE
:10B4C0000AC493F7F7070AC8A384F5002A89AE8453
:10B4D00005C41C42054783C70700636AF704034796
:10B4E000B400630BF700A305F400EF70502383470B
:10B4F000B400A9C3EFD00FD921649305B40028008C
:10B50000EFB09FDFEFF07FF9AA852800EFD0CFF4EE
:10B51000014781463000A6854A85EFB07FFE2904A9
:10B52000480822CC230A010002CEEFE04FAE0561AD
:10B530006F60FF82EFD02FDAC1B7EF621F80011179
:10B540007C003ECAB70707003ECC7C003ECE83C7D6
:10B5500095002E84AA8493F7F707A384F500A165CC
:10B56000AD054808EFB05FD9EFF03FF3AA85480872
:10B57000EFD08FEE500801478146A2852685EFB0B7
:10B580003FF805616F60AFFD97A7FF1F9387876541
:10B590009C43094599C303C5C7008280EF62EFF958
:10B5A00001117C00AE843ECAA165B70707002A845A
:10B5B0003ECCD1057C0048083ECEEFB0FFD3EFF083
:10B5C000BFFCAA854808EFD02FE950080147814603
:10B5D000A6852285EFB0DFF205616F604FF8EF625C
:10B5E000CFF583C7950093F7F707A384F500EFF035
:10B5F000FFFA6F60CFF6EF62AFF283C795000329C1
:10B60000C501411193F7F707A384F5001C4283C9D4
:10B610000700854763EC370597B7FF1F9387C7B3CC
:10B620009C432E84AA8495C7EFF01FF689476302D6
:10B63000F502630009028347C900638C37012306C2
:10B640003901EF70D00D83572903898B99C3EFA07F
:10B65000D0452685A285EFF07FF4A167CD0748008D
:10B660003EC42302010002C6EFE06F9A41016F6001
:10B670006FEE97A7FF1F9387E7569C431D4599C31D
:10B6800003C5E7008280EF624FEB0111B7070700A7
:10B690003EC683C79500584D0AC493F7F7070AC8FA
:10B6A000A384F5002A89AE8405C71C4283C707001E
:10B6B00093968701E18663C8060485466385D704AF
:10B6C0008346E7006386F6002307F700EF70300536
:10B6D00021649305E4002800EFB01FC2EFF07FF96A
:10B6E000AA852800EFD04FD7014781463000A685B4
:10B6F0004A85EFB0FFE03504480822CC230A010058
:10B7000002CEEFE0CF9005616F606FE5EF62EFE290
:10B7100001117C003ECAB70707003ECC7C003ECE3C
:10B7200083C795002E84AA8493F7F707A384F500B6
:10B73000A165B9054808EFB03FBCEFF09FF3AA85BB
:10B740004808EFD06FD1500801478146A285268571
:10B75000EFB01FDB05616F608FE0EF626FDCAA84E2
:10B76000014417A9FF1F13092948E149EFC0FF90C1
:10B770006344A400014519A8330534038327090055
:10B780003E95835725006395970011056F608FDC08
:10B790000504E9BF032E850063040E1017A3FF1FE5
:10B7A0001303436303230300631503002943639AD0
:10B7B000060E03234E01631503001D436393070E1A
:10B7C000EF622FD5C689428A3E89BA8AB684328B07
:10B7D000AE8B2A84A1E903554E0009E501431A8581
:10B7E0006F60AFD6A167A98F116763F7E700EFF02D
:10B7F000DFF68145EFF08FBD0844B70700E0584100
:10B80000F98F18455CC1B707001FF98F1CC55C494B
:10B8100081C76105EFB01000E38209FC2285EF705B
:10B82000606E6DBF3285EFA0E0620D434DD91C44C0
:10B83000116703D54700A167A98F63F7E700EFF011
:10B84000DFF18145EFF08FB80323840093164B019D
:10B85000D1828347B300035663008588FD8BA3051F
:10B86000F300FD777D8E558EFD76FD16B204F18EC8
:10B8700083274301C58E231273012313D3002304AE
:10B88000530123052301A3044301D9D72285EFB037
:10B890007FBBAA850844B5DD6105EFB02076ADBF5A
:10B8A0001D431A858280EF62AFC70569AA84AE89FD
:10B8B000328A0144FD5A7D19EFC0EFF06345A400C0
:10B8C00001456F602FC9D84493171400BA9703D766
:10B8D0000700631B37032390570163050A00268581
:10B8E000EF70E0389C448DC383D76700B3F727011E
:10B8F000639C3701D2880148814701478146014650
:10B9000081452685EFF01FE905047DB7EF624FC141
:10B9100079711C103EC4B7070F003EC61C103EC80C
:10B9200083C79500AA8A328593F7F707A384F500A9
:10B930002E893284EFD00FBE93170501C187635063
:10B94000F006AA892285EFD0EFBC2A8A4E85032B08
:10B950000400EFB05F9039E583574400814405440B
:10B96000F11793B71700A303F10083457100DA873D
:10B970002287D2864E862800EFE03FA40147814609
:10B980003000CA855685EFB0BFB7A1679387F7032C
:10B9900048083ECC230A810026CEEFD05FE7456100
:10B9A0006F604FBBA28513067100EFE0BFAFAA84A2
:10B9B000094445DD5285EFE0EFB80D445DD50546FD
:10B9C000D2852685EFF03FEE2A8445B7EF62EFB6C9
:10B9D000835507000346270041112A842E8532C66D
:10B9E0002EC4EFE02FB611C53246A2452285EFF0F6
:10B9F0009FEB41016F60AFB6EF62AFB183C79500B7
:10BA00004111AA8A93F7F707A384F5003285AE891E
:10BA10003284EFD02FB093170501C1876357F00828
:10BA2000C1452A8A2285EFD04F9B2A8D2285EFD0EF
:10BA30006FAE2A892285EFD08FAC930705F893F774
:10BA4000F70F1307E007AA8B6371F7062285EFD083
:10BA50000FAB2A8C2285EFD08FAAAA8C5285032B9C
:10BA60000400EFB04FFF29E5835744002311010084
:10BA70008144F11793B71700A300F1000544034771
:10BA8000110083562100938784005685DA88228826
:10BA90005286CE85EFE03FE6A167E90748003EC445
:10BAA0002302810026C6EFD09FD641016F60EFA927
:10BAB00013061100A285EFE0FF9EAA8409E5231179
:10BAC000010009446DBF930521006A85EFF06FA165
:10BAD0002A8455F5835521009356C9001316490150
:10BAE00085486688E2875E87858A51822685EFF0E1
:10BAF0007FCA2A8469B7EF62CFA183C7950041113D
:10BB00002A8B93F7F707A384F5003285AE89328438
:10BB1000EFD04FA093170501C1876352F0082A8A1E
:10BB20002285EFD02F9FAA8A2285EFD0AF9E2A8947
:10BB30002285EFD0CF9C930705F893F7F70F1307F3
:10BB4000E0072A8C637DF7042285EFD04F9BAA8CF7
:10BB50002285EFD0CF9A2A8D5285832B0400EFB037
:10BB60008FEF29E18357440085440144F11793B7CF
:10BB70001700A301F10003473100930784005A85A1
:10BB8000DE882688D6865286CE85EFE0DFD68D47C2
:10BB900048003EC42302910022C6EFD05FC7410196
:10BBA0006F60AF9AA28513063100EFE0BF8F2A8441
:10BBB000894471D19356C9001316490185486A8892
:10BBC000E6876287858A5182D685EFF0BFBCAA845A
:10BBD0005DB7EF62EF942A8981440144617A916AEA
:10BBE00017ABFF1F130B0B1FEFC0EFBE63C5A40005
:10BBF00022856F602F968327090093991400CE97B2
:10BC000003D50700330745014207418363625703A9
:10BC100011CD03270B0009C785453E85EF30E04A6B
:10BC2000832709000504CE972390070085046DBF84
:10BC3000EFF0BFB2832709000504CE9723900700D9
:10BC400075D58145EFE09FF8D5B7EF626F8D83C75B
:10BC5000950041112A8A93F7F707A384F5003285EE
:10BC60002E893284EFD00F8B93170501C18763545F
:10BC7000F004AA89832A0400EFB0EFDD21E18357A5
:10BC8000440085440144F11793B71700A301F10064
:10BC900003483100D68752850147CE862686CA855D
:10BCA000EFD01FE3A167F50748003EC423029100CF
:10BCB00022C6EFD0DFB541016F60CF89A2851306A0
:10BCC0003100EFE02FFE2A84894479D197A7FF1F26
:10BCD000938747109C4381CB0449EFC0CFAFAA851F
:10BCE0002685EF30803E13050401EFF09FEE22859C
:10BCF000EF609079814469BFEF62AF8183C795009F
:10BD00004111AA8A93F7F707A384F5003285AE891B
:10BD1000328423110100EFC0FFFF93170501C18793
:10BD2000635CF0042A8AC1452285EFC01FEBAA8B11
:10BD30005285032B0400EFB00FD231E1835744004A
:10BD400085440144F11793B71700A300F10003489D
:10BD5000110003572100DA875685D2862686CE85C4
:10BD6000EFD01FD7A1679387270248003EC4230264
:10BD7000910022C6EFD0BFA941016F501FFDA285DF
:10BD800013061100EFE00FF22A84894469D197A7C6
:10BD9000FF1F9387270498433E8901CB0449EFC0D6
:10BDA0008FA3AA852685EF30403213050401EFF0FA
:10BDB0005FE2EFC04FA2954459D9930521005E85FB
:10BDC000EFE03FF2AA8441F51C4803572100228589
:10BDD0002390E700EF60506B83270900ADDB03552C
:10BDE0002100EF30E026A5B7EF52BFF283C79500E0
:10BDF0004111AA8A93F7F707A384F5003285AE892B
:10BE00003284EFC03FF193170501C1876359F004F5
:10BE10002A8A2285EFC01FF02A895285032B04004D
:10BE2000EFB06FC321E18357440085440144F1170B
:10BE300093B71700A301F10003483100DA87568554
:10BE40004A87D2862686CE85EFD09FC8A167F9079C
:10BE500048003EC42302910022C6EFD05F9B4101FF
:10BE60006F50BFEEA28513063100EFE0AFE32A84E6
:10BE7000894479D19167CA97C2071167C1831307B3
:10BE8000F7EF8544E36AF7FA97A7FF1F938787F4D4
:10BE90009843BE8B01CB0449EFC0EF93AA8526855A
:10BEA000EF30A02213050401EFF0BFD2EFC0AF9234
:10BEB000954459D11C482285814423902701EF6085
:10BEC000B05C83A70B00ADDB4A85EF306018ADB7DF
:10BED000EF52BFE62A844105B284EFF09FCF01C53F
:10BEE0002285EF60705A81460146A6852285EF7053
:10BEF000C00B1C4C89C7DC4799C3228582976F50C1
:10BF00001FE697A7FF1F9387E7CD9C43014599C381
:10BF100013850701828097A7FF1F9387A7CC8843CB
:10BF20008280EF529FE19317C600DD8DC20541115B
:10BF3000C1812A8432C6EFC07FD332462285118266
:10BF40009375F60FEFC05FD141016F505FE1EF5283
:10BF50003FDD79713C083ED2B7070C003ED43C0867
:10BF60003ED683C79500AE842A8993F7F707A3844A
:10BF7000F500A165938535044810EFB0EFB7C165B2
:10BF8000FD15014417AAFF1F130A4AE6930A400E43
:10BF9000AE892E8B2EC6EFC00F8742059317040182
:10BFA0004181C183B24563E3A702C167FD17638581
:10BFB000F5004810EFC09FCB501001478146A68581
:10BFC0004A85EFB0EFD345616F50DFD83307540394
:10BFD00083270A0BBA9703D6C70163083601638823
:10BFE00035014810EFF0FFF3DA85050465B7B28537
:10BFF000EDBFEF521FD279717C083EC8B707110020
:10C000003ECA7C083ECC83C79500AA89328593F747
:10C01000F707A384F5002E89EFC0DFCF8567637E25
:10C02000F502A165AA8489050808EFB0EFAC268562
:10C03000EF30E052133415000A04A2850808EFC05F
:10C04000BFC1A6850808EFC07FC235C00147814641
:10C050001008CA854E85EFB0AFCA45616F50FFCE5C
:10C06000B30754030327CA0ABA9703D70700631A12
:10C07000970003D62700638A65030808EFF07FEA7C
:10C08000DE8505042EC6EFB01FF9420593170401A3
:10C090004181C183B245E3E5A7FCC167FD17E38792
:10C0A000F5FA0808EFC09FBC55B7B285D9BFC16586
:10C0B000FD15014417AAFF1F130A4AD3930A8002F1
:10C0C0002E8BAE8BC1B7EF525FC718418347170065
:10C0D00083460700A207D58FD207D1832390F500AE
:10C0E00083472700034717008D45A207D98F918307
:10C0F0002310F600EFC03FAD6F507FC6EF525FC216
:10C10000C164014417A9FF1F130949CE9309800296
:10C11000FD14EFB05FF06345A40001456F509FC36D
:10C12000330534038327C90A3E9583570500E38707
:10C1300097FE0504F9BFEF52BFBE2A8AAE89B284CA
:10C14000B68AEF30C04109E591473E856F509FC0E8
:10C150002A894E85EF9010502A84638A0A048D47FD
:10C160006DD503570500C547E31147FF0347F901A4
:10C170008546AD47E31BD7FC8347450091CB41463D
:10C18000A6855D05EFC0D022814761D1AD4775BF5F
:10C19000130965012302E500CA852685EF10202DCD
:10C1A00015CDA547E3830AFA2302040079BF11CD18
:10C1B00083570500E39A47F94146A6851905EFC064
:10C1C000301F814759D1994749B74E85EFF01FF38A
:10C1D0002A8495473DD9130955007DBF4146A68560
:10C1E000231044012311340113051900EFC0B01EC0
:10C1F0002285EF60B03C814789BFEF521FB479714F
:10C200007C003ECCB7070A003ECE7C003ED083C700
:10C210009500B2842E8493F7F707A384F5001306E4
:10C22000A1002A892C002685EFF0FFE9A1652808E6
:10C230008D05EFB06F8C90408355A10003558100B0
:10C240008546EFF05FEFAA84AA852808EFC0DFA03B
:10C250000356A100835581002808EFF09FCC3008D9
:10C2600001478146A2854A85EFB08FA985474810CE
:10C270003ED42302910202D6EFD06FD945616F50B0
:10C280001FAEEF529FAB79717C003ECCB7070A001E
:10C290003ECE7C003ED083C79500B2842E8493F7B7
:10C2A000F707A384F5001306A1002A892C00268530
:10C2B000EFF07FE1A16528088D05EFB0EF83904096
:10C2C0008355A100035581008146EFF0DFE6AA8483
:10C2D000AA852808EFC05F980356A1008355810006
:10C2E0002808EFF01FC4300801478146A2854A851F
:10C2F000EFB00FA148102302910202D402D6EFD072
:10C300000FD145616F50BFA5EF523FA3EFF0BFE2E1
:10C310006F50FFA497A7FF1F9387078D88438280E4
:10C32000EF52BFA1835725004111AE842A84230711
:10C33000B10017F5FFFF1305A5696C002316F10086
:10C34000EFB0CFD581C42285EF60B02DFD5723100B
:10C35000F40013062002814513055400EF50FFA09E
:10C3600041016F50DF9FEF52BF9B79717C003ECC43
:10C37000B7070A003ECE7C003ED083C79500AA894D
:10C38000AE8493F7F7073285A384F5001306A10066
:10C390002C00EFF05FD3035581001144EF30201CD7
:10C3A00015C10355A1000144EF90D02A01CD0357D8
:10C3B00005008357810045446316F7008545EFF07B
:10C3C0003FF601442169930539002808EFA0DFF208
:10C3D000A2852808EFC05F880356A100835581001D
:10C3E0002808EFF01FB4300801478146A6854E8526
:10C3F000EFB00F9148104AD42302810202D6EFD049
:10C400000FC145616F501F95EF529F919797FF1F86
:10C410009387477D2A8488432E8915C10357450396
:10C420008357C401631DF700232605022318050264
:10C430004105EFA0303E63040900EF60302F8144D6
:10C4400097A9FF1F9389899A130A8002EFB0BFBC96
:10C4500063CCA40297A7FF1F938787819C4389C75A
:10C460000355C401EF104076630509002285EF6093
:10C4700050031306400E81452285EF501F8FFD5754
:10C48000231EF4006F501F8D3385440383A7C90A10
:10C490003E95035705008357C4016315F700CA850D
:10C4A000EFF01FE885045DB7EF529F8783C79500C3
:10C4B0004111AA8993F7F707A384F5003285AE846A
:10C4C000EFC05F8585676370F5042A89EF30200926
:10C4D000014411C983D7040031446386270185458F
:10C4E000EFF09FF201444E85A2864A86A685EFD0E2
:10C4F0002FBFA1679387170448003EC42302810021
:10C5000002C6EFD0CFB041016F50DF84EF525F81A0
:10C510009797FF1F9387076D80431DCC0145EFA0C0
:10C52000E05681470148C1641CDC232E040323200C
:10C53000040417A9FF1F1309698B01449309400ED6
:10C54000FD14EFB05FAC634BA400814517050000FC
:10C5500013054598EFB08FB46F50CFFF3305340308
:10C560008327090B3E958357C50163859700854551
:10C57000EFF09FE90504F1B79357050113D7870042
:10C58000A380F50093170501C183A1832380E500F3
:10C590002381F500A381A5008280EF520FFA2300CA
:10C5A000050083C71500A300F50083C725002301FC
:10C5B000F50083C73500A301F50083C745002302BA
:10C5C000F50083C75500A302F50083C765009305F6
:10C5D0009500A30305002303F5002304050032851D
:10C5E000EFF09FF96F50AFF7EF528FF34111E9541D
:10C5F0001DC995C993F9C5FF2E842A89AA84338A57
:10C60000A900B7EA040063149A020D88854401CC9E
:10C61000B7E704009C5F82972AC622866C00330528
:10C620003901EFC0405B268541016F50AFF283A70F
:10C630008A039104829793170501C183A183A38E76
:10C64000F4FE93570501238FF4FEA183238EA4FEED
:10C65000A38FF4FE4DBF63E0D502EF520FEEB28719
:10C6600041113686BE8536C6EFC0E056B24641015E
:10C6700036856F50CFEE81463685828083870500F0
:10C680001387F5003D05FD8793F77708834607007C
:10C690007D158606B58FA300F5006307B7007D17EB
:10C6A000834717009D83DDB78280EF520FE9B7E71C
:10C6B000040083A7070932872A863A8582971335B3
:10C6C00015006F50CFE901CD814799C9EF52EFE6D0
:10C6D0004146EFC0405085473E856F504FE8814747
:10C6E0003E8582801DC5EF524FE5414681452A8433
:10C6F000EF50AFE74146814513050403EF50EFE6E5
:10C700000147C1672322040438C87CC805456F501F
:10C710000FE501458280814729CDA1CDEF52EFE1A0
:10C72000B2842E891306800581452A84EF50EFE3F9
:10C73000CA8524C42685EFF01FF94146814522852C
:10C74000EF50AFE23044A2852285EFF01FF693044C
:10C750000401A2852685EFF07FF2A6851305040269
:10C76000EFF0DFF12285EFF0FFF785473E856F5050
:10C770000FDF3E858280EF52AFDA4111E9541DC9C7
:10C7800095C993F9C5FF2E842A89AA84338AA90002
:10C79000B7EA0400639444030D88814401CCB7E7F1
:10C7A00004009C5F82972AC622866C0033053901FB
:10C7B000EFC06042268541016F50CFD983A78A031D
:10C7C0009104829793170501C183A183A38EF4FE80
:10C7D00093570501238FF4FEA183238EA4FEA38F1C
:10C7E000F4FE4DBF71CDEF52AFD3B28401E60545E3
:10C7F0006F504FD62A842E890145FDD93C48784890
:10C80000B3E6E700F5D69386F7FFB3B7F6007D17DA
:10C81000032A4404BA9734C87CC8630F0A04C14988
:10C8200013050A03B38949412295637B3601B28619
:10C830002E86A685EFF03FE27C40BE9464C045BFE3
:10C84000CE862E86CE85EFF01FE1C114D2944E998C
:10C8500023220404A2879306040103C7070003C62A
:10C8600007038507318FA38FE7FEE398F6FE304478
:10C87000A2852285EFF07FE32699C14933069940CE
:10C8800063EA9900ADD4A686A68513050403EFF0EC
:10C890009FDC6DB78147B306F4003307F60003470A
:10C8A000070083C5060085072D8F2380E600E394EB
:10C8B00037FF3044A2852285EFF03FDFC1147DBFF2
:10C8C0000145828019C9EF524FC713068005814583
:10C8D000EF50AFC905456F508FC801458280814731
:10C8E0003DC9B5C9EF526FC5FC4141462E84AA84AB
:10C8F0006393C70413860501A2878146C14503C718
:10C90000070003C507038507298F3305D6000345B4
:10C9100005008506298FA38FE7FEE392B6FE30441B
:10C92000A2852685EFF07FD82285EFF0BFF98547F5
:10C930003E856F50CFC2138507031D8E814522951A
:10C94000EF50AFC27C40130700F813060402A29711
:10C950002388E70255B73E858280EF520FBE6D7186
:10C960002E84B284AA85901028003689EFF0BFDAB1
:10C9700019E9D55705A050400C402800EFF09FE67C
:10C980006DD9FD142104E5F82C004A85EFF03FF540
:10C99000814765D13E8551616F506FBCEF52EFB951
:10C9A00041112EC432C62C000546EFF01FFB410199
:10C9B0006F50EFBAEF526FB801112A842EC602C829
:10C9C00002CA02CC02CEEFC06049B2462A86A285D6
:10C9D0000808EFF0BFFC1375F50F05616F502FB815
:10C9E000EF52AFB57971B2872A8421462308B1008E
:10C9F00013051101BE853AC436C6EFC0C01DB2464C
:10CA0000930591013685EFF03FB722851410354626
:10CA10000C08EFF0BFF82A84224711E521460C10DC
:10CA20003A85EFC0401B228545616F504FB3EF52EE
:10CA3000CFB07171AE84AA850A853284EFF0BFC889
:10CA400001C90A86A6852285EFF03FC6814711E11C
:10CA5000C5473E854D616F508FB0EF520FAB1D71D2
:10CA60002A8AB289BE8435468547130511012E8C6A
:10CA7000B68A3A8BC28C468D2308F100EFC0A01510
:10CA800010100C085285231F0100EFF05FFA2A8472
:10CA90002DE9A147631BFD069307900591E0E5474B
:10CAA0003546E2851305110113990A012308F100A7
:10CAB00013590901EFC020121357890093978A0078
:10CAC000D98F90080C085285231FF100EFF03FF634
:10CAD0002A8405E9A1E09387FA0091831379F9008C
:10CAE0003EC6631309004149668B8144C14B854DA5
:10CAF000B2476397970C6A868C0033855C01EFC060
:10CB0000800D228525616F500FA493079004C9F80A
:10CB1000A54779B7834701050947C14B2308F100B1
:10CB200083471105A58FA308F10093872400814452
:10CB300063EFFB02014714083386E6008C08B386D6
:10CB4000E400BA95DA9683C6060083C5050005079A
:10CB5000AD8E2300D600E390E7FE41476398E704DB
:10CB600090080C085285EFF09FEC35D535A8B30638
:10CB70009B00BA871008B305F60090083E9603C5DF
:10CB800006000346060085078506298E2380C5001A
:10CB9000E39277FF998F90080C085285BE94EFF0CE
:10CBA0001FE98947014749D52A84A1BF90083E96CD
:10CBB000034606001408BE962380C600850779BF89
:10CBC000B2478504638B971281471808B306F700B4
:10CBD00098083E973386F90003470700034606008E
:10CBE0008507318F2380E600E39177FF90080C08DA
:10CBF0005285EFF0DFE34DF93546E285130511016B
:10CC00002308B101EFB0307D13970401418393975E
:10CC100084002183D98F10180C085285231FF1003E
:10CC2000EFF0FFE051F1814710183387F9003E968D
:10CC30000347070003460600B306FB008507318F54
:10CC40002380E600E39277FF75A01808B306F7008B
:10CC500098083E973386F90003470700034606000D
:10CC60008507318F2380E600E3E127FFCA876398B9
:10CC7000770990080C085285EFF07FDB15F58147A6
:10CC80009800B306F700900818103E973E960347A9
:10CC90000700034606008507318F2380E600E391F5
:10CCA00077FF3546E285130511012308B101EFB086
:10CCB0009072139704014183939784002183D98F45
:10CCC00010180C085285231FF100EFF05FD6E31D0A
:10CCD00005EC814710183387F9003E96034707009B
:10CCE00003460600B306FB008507318F2380E6006C
:10CCF000E3E227FFC109410BE5BB8147B5B79408C3
:10CD0000BE9683C6060018083E972300D700850705
:10CD1000B9BF638E062CEF425FFF59712A84BE892A
:10CD2000B28B85473546130511022E8B468C4289FE
:10CD3000BA8A368A2300F102EFB0F06910180C109D
:10CD4000228523170102EFF09FCE631E0510A14735
:10CD50006319FC069307900563930900E547354680
:10CD6000DA851305110293140A012300F102C18030
:10CD7000EFB0706693178A0013D78400D98F90089C
:10CD80000C1022852317F102EFF07FCA69ED639042
:10CD900009049307FA00BD88918391E0C144C2075A
:10CDA000C183DE8C814A3EC6414DB24763EAFA0C2C
:10CDB0006286B3854B018810EFB0905F4DC53D553D
:10CDC0005DA093079004E39C09F8A54749BF8347FA
:10CDD00001050947C14C2300F10283471105B3C780
:10CDE000F900A300F10293872900814963EFFC0257
:10CDF000814618103306D7008C083387D900B695C2
:10CE000056970347070083C5050085062D8F23002D
:10CE1000E600E390D7FE4147639AE70490080C10C0
:10CE20002285EFF0DFC035D53DA8B3863A01BA8739
:10CE30001010B305F60090083E9603C506000346A1
:10CE4000060085078506298E2380C500E39297FF9B
:10CE50003387EC4090080C102285BA99EFF03FBD63
:10CE60008947014741D565616F40FFED90083E96C7
:10CE7000034606001410BE962380C600850769BFCE
:10CE8000B247850A93990A01939D8A0093D90901B3
:10CE90006399570D85473546DA851305110223003E
:10CEA000F10293D98900EFB01053B3ED3D0190002A
:10CEB0000C1022852317B103EFF07FB74DF58147A2
:10CEC000A68963E6970626860C084A85EFB0B0501F
:10CED00081471810B306F700100898083E973E9651
:10CEE00003470700034606008507318F2380E600CD
:10CEF000E3E197FE639DA90590080C102285EFF0F1
:10CF00001FB335F181479810B306F7009008181841
:10CF10003E973E9603470700034606008507318F7C
:10CF20002380E600E391A7FF4109C10CBDBD1808AD
:10CF30009000B306F7003E963387FC0003470700D6
:10CF4000034606008507318F2380E60095BF9808C9
:10CF50004E97034707001C10CE972380E7008509F2
:10CF600051BF85473546DA85130511022300F102CA
:10CF700093D98900EFB03046B3ED3D0190000C101D
:10CF800022852317B103EFF09FAAE31E05EC81472A
:10CF900018089000B306F7003E963387FC0003475D
:10CFA0000700034606008507318F2380E600E391E2
:10CFB000A7FF41460C084A85EFB0F04181471810A1
:10CFC000B306F700100898083E973E9603470700FF
:10CFD000034606008507318F2380E600E391A7FF13
:10CFE00090080C102285EFF09FA41DDDADBD7D558E
:10CFF0008280EF429FD401112A842E85930551002F
:10D00000328902C002C202C402C693047400EFF067
:10D01000AFD61D46A68513059100EFB0D03B100892
:10D020008A854A85EFF0BFA019ED93071400180810
:10D0300083C607000346070085070507B18EA38F47
:10D04000D7FEE397F4FE05616F407FD1EF425FCDDD
:10D050002E848C414111AA8983871500328991441D
:10D0600063D30700A1449797FF1F9387E70E9C4364
:10D07000B1C3B5CE8D472310F10083C725004A8583
:10D080002301F10083C73500A301F10083C74500E8
:10D090002302F10083C75500A302F10083C7650096
:10D0A00093059100A30301002303F1002304010071
:10D0B000EFF08FCC0C404A860A85EFF00FCE0328A4
:10D0C000040083564400A6881D0881470147E516E1
:10D0D00042868A854E85EFF05F982A8909E5A68504
:10D0E0002285EFB0FFB24A8541016F40BFC64A8634
:10D0F0000A85EFF08FCA7DBFEF429FC22E848C411C
:10D100004111AA89838715003289914463D30700AE
:10D11000A1449797FF1F938727049C43B1C3A5CED3
:10D120008D472310F10083C725004A852301F100B4
:10D1300083C73500A301F10083C745002302F10036
:10D1400083C75500A302F10083C7650093059100D2
:10D15000A30301002303F10023040100EFF0CFC17A
:10D160000C404A860A85EFF04FC3835644000328DB
:10D1700004008A85858EC2061D08C1822312D40050
:10D18000A68881470147E51642864E85EFF07FB8B5
:10D1900041016F403FBC4A860A85EFF00FC0C9B716
:10D1A000EF42BFB9B335B000011185052A891315C7
:10D1B000F601336515012308B1009305110136848A
:10D1C0003AC632C03EC442C2EFF00FBBA24712487B
:10D1D000425593D68700230BF10093059101935795
:10D1E0008800A30AD100A30BF100230C0101EFF08A
:10D1F000AFB83247024603280400B337E000835635
:10D2000044009207914411C2A1444A85A6884286EF
:10D210000C08EFF09F842A8909E5A6852285EFB0E6
:10D220003F9F4A8505616F409FB3EF427FAF011179
:10D230003EC68647B335B0008505AA891315F601A9
:10D240005D8D2308B1009305110136843A89B284BB
:10D2500042C446C2EFF04FB2224892481645935757
:10D260008800A30AF1009305910193D78800230B4E
:10D270000101A30BF100230C1101EFF0EFAF3247D6
:10D28000104083564400B337E0009207032809009A
:10D29000914891C0A1480C084E85EFF09FA7AA8441
:10D2A00011E5835544004A85EFB09F9626850561B8
:10D2B0006F405FAAAA959307F00F17F700001307B6
:10D2C000278A6317B50013C5F7FF1375F50F828022
:10D2D00005058346F5FFB58FBA9783C70700D5B715
:10D2E0000357450014419307F00F17F6000013068B
:10D2F0002687369742074183139506014181631BB8
:10D30000E500AD8FB29703C50700130515F313357C
:10D3100015008280850603C5F6FFA98FB29783C7E3
:10D320000700D9BFEF427FA1B28736842E86BA8626
:10D33000AA853E85BA84EFF06FE6634B050022852F
:10D34000EFB0D0312A86A686A2852685EFF00FE5BC
:10D350006F40FFA0EF42DF9C5D712A8BAE8A17E51C
:10D3600000001305657D2C00B284368ABA893E8997
:10D37000EFF04FE42A8459E534104146DA8528005D
:10D38000EFF0CFE12A843DED8547A303F100A6C26B
:10D39000930771002408BEC4A68685470D462C1845
:10D3A000281002DC02DED6C0BEC6EFF00FDB2A84F6
:10D3B00031E983477102A6860D4693F7F7072300EC
:10D3C000FA00C1473EDE2C188947281026DCA3034B
:10D3D000F100EFF08FD82A8415E54146A6854E85E9
:10D3E000EFB0607F8D47A6860D462C182810A3034A
:10D3F000F100EFF08FD62A8411E54146A6854A85D3
:10D40000EFB0607D228561616F40DF94EF42FF9253
:10D4100097D700009387070C984383C7470079711B
:10D420002A89AE8417E50000130585710C083AC4FB
:10D430002306F100EFF00FD82A8415E514104146B9
:10D44000CA850808EFF08FD52A8411ED1408154617
:10D450002C000810EFF08FD42A8411E521462C0807
:10D460002685EFB04077228545616F405F8FEF42A0
:10D47000DF8C97D700009387E7059C477971AA84D2
:10D480002E8417E500001305256C0C083EC6EFF04E
:10D490006FD20DE514104146A6850808EFF00FD0B5
:10D4A00011ED140811466C000810EFF02FCF19E5AC
:10D4B0008347F10193F7F7032300F40045616F40C0
:10D4C0001F8AEF429F873688A14881470147E5467A
:10D4D000EFF0AFD86F40BF88EF423F863688A14853
:10D4E00081470147E546EFF0DF826F405F87EF42FB
:10D4F000DF8401112A842E850C0832C6EFF08FCB11
:10D5000019E9324797E60000938686621008C14504
:10D510002285EFF03FE105616F407F84EF42FF819C
:10D520004111C1472EC032C48A8509463EC23EC65B
:10D53000EFF0AFC241016F409F82EF421F80411167
:10D54000AE8613061009AA850A8502C002C202C46B
:10D5500002C6EFF0AFC441016F407F80EF42EFFDA4
:10D56000328797E600009386A65E2E86930500021A
:10D57000EFF05FDB6F40AFFEEF422FFC7971C147E8
:10D580002ACC2ED032D42C080D4628003ECE3ED2D6
:10D590003ED602C402C602C802CAEFF00FBC456103
:10D5A0006F40EFFBEF426FF90111AA842E8417E55B
:10D5B00000001305655A8A85EFF0CFBF05E5140812
:10D5C0004146A6850A85EFF06FBD09ED8347E1016D
:10D5D0000347F101A207D98FCA07C9836177D98FA1
:10D5E0002310F40005616F408FF705C9EF42EFF497
:10D5F0009787FF1F9387C76390439785FF1F938586
:10D6000065631785FF1F1305A55EEFB080091785B9
:10D61000FF1F1305E55D6F408FF41785FF1F13058E
:10D62000255D82809DC5EF424FF19787FF1F93874D
:10D630002760944301112E840A869785FF1F9385E6
:10D64000655FEFB0800A0A850294014505616F406D
:10D650000FF17D558280EF424FEEEFB08014978737
:10D66000FF1F23A7A75C17F5FFFF130525F8EF9011
:10D67000D0406F40CFEE1787FF1F1307A75D9317AA
:10D68000150008433E95FD572310F5008280EF42B8
:10D69000CFEA2A84084019E16F406FEC1C415840E2
:10D6A0001CC06313E5005CC08347550023200500C0
:10D6B000F99BA302F500EFB0EFF9E9BFEF424FE6A7
:10D6C0009787FF1F9387075B98432A8411CB834773
:10D6D000350093F7070289C703550500894502976E
:10D6E00013054401EF901013835504000355E40023
:10D6F000EF20701B485809C5EFB0CFF5232A04026C
:10D7000013058403EFF0BFF88144B149EFA0FF9AFD
:10D7100063C5A402834734002320040493F727FC45
:10D72000A301F4000048EFA05F9A1316150081458D
:10D730002285EF408FE36F40EFE1B3873403032985
:10D74000040385043E994A85EFF07FF42304090021
:10D7500075BF8347350093F7070299E3014582803F
:10D760008357E500E39CB7FEC167FD176316F6001B
:10D77000054582800545B9A0EF422FDC93170601CD
:10D78000C187B2842A8401496359F0028357050096
:10D790008DCB01456367F600034584003E95332534
:10D7A000A6001375F50F39A81C4813171900BA976E
:10D7B00083D70700E38097FC0509EFA01F91E3459D
:10D7C000A9FE01456F40AFD9EF428FD5AE89AA843B
:10D7D000EFA07F852A84EFD0BFAAAA86014713064F
:10D7E000840197050000938545E91785FF1F130500
:10D7F000A546EFA0AFD52A8921CD8C441304C500DE
:10D8000022859E0593F50508EFB00FC5CC408387B0
:10D810007400E18163D1070493E505082285EFB028
:10D82000AFC30D46938544002285EFB00FC183D569
:10D8300004002285EFB0EFC583D524002285EFB028
:10D840004FC503D6490083A509002285EFB0EFBE7E
:10D850004A856F402FD093F5F507C9B7EF42EFCD5A
:10D8600001112A84328532C6EFB06FB4EF903F9138
:10D87000835704001787FF1F130747573246231BA0
:10D88000F100930700F8A30DF1001C471843231A79
:10D89000A1008983858BB307F740B28548083ECE47
:10D8A000231C0100230D0100EFF01FF205616F4002
:10D8B0000FCBEF42EFC60041014529CC9304C400D1
:10D8C00026853289AE89EFB08FB295452A8A2685A2
:10D8D000035B0401EFB02FAF2685EFB02FC68D4557
:10D8E000AA8A2685EFB02FAE2685EFB02FC55C48FB
:10D8F000420A135A0A01D2975CC423186401814773
:10D9000063983A0146054D81330625419337160049
:10D9100013F5F70F6F400FC4EF42AFBF89692A8B31
:10D92000AE8B328AB68A81440144314CFD19EFA096
:10D93000CFF863C9A400EFA04FFB018D33B5AA0057
:10D940006F40AFC03389840383270B003E99631770
:10D950000A008347890085043E94D1BF03560A001C
:10D96000DE854A8533F6C900EFF0BFF47DD1054569
:10D97000C1BFEF428FBC01112A847C000355E50032
:10D980003ECAB70707003ECC7C003ECEEF10303DCC
:10D990002A8985454808EFB0EFC199454808EFB09E
:10D9A0002FA7AA844A85EF10B03D2380A400978753
:10D9B000FF1F9387A7439C434166130606F0939687
:10D9C000870113D78701558F93D68700F18E558F26
:10D9D000A207B706FF00F58FD98F11462C001385DB
:10D9E00014003EC4EFB0201F5008A38204008945F4
:10D9F0002285EFF0BFE609C9AA8513058403EFB0BD
:10DA0000EFBB3C4085073CC005616F404FB5EF421E
:10DA1000CFB2EFA08FED2A840504EFA00FEC330501
:10DA2000A402F14791453305F502EF10207B01E593
:10DA300065556F40CFB29787FF1F23A5A722EFA0A0
:10DA4000CFEA2A840504EFA04FE93305A4028945F3
:10DA50000605EF10A07869DD9787FF1F23ACA71E8E
:10DA6000EFA0AFE82A840504EFA02FE73304A40257
:10DA70009787FF1F2392871EEFA02FE72A84EFA02E
:10DA8000CFE5930714003385A7029787FF1F2396DE
:10DA9000A71C97E700009387E7CF1787FF1F232175
:10DAA000F71C014579B7EF42AFA7AA842E8901443C
:10DAB0009789FF1F93898933130A8006EFA0EFE14E
:10DAC0006345A40001456F40EFA83305440383A7D5
:10DAD00009024A86A6853E95EFF0BFC719E1050405
:10DAE000F1BF0545CDB7EF42CFA2AA8A2E8BB28BEC
:10DAF000368C3A8A814401448149978CFF1F938C6C
:10DB0000EC2E130D8006EFA04FDD63C7A40011E0DB
:10DB100085494E856F406FA33389A40383A70C0208
:10DB20005E86D6853E994A85EFF0BFC219CDEFA03B
:10DB3000CFDB0544636B4501D2866286DA85130527
:10DB40000903EFF07FDD11C1854985046DBFEF4208
:10DB50002F9DC16441112A8901449789FF1F938930
:10DB6000E928130A8006FD1436C632C42EC2EFA07F
:10DB7000CFD692452246B2466346A40001454101F4
:10DB80006F404F9D3305440383A709023E9509C6A4
:10DB900083473500C18B9DC791C68347350093F7F6
:10DBA00007028DC3630699008357E500639C270134
:10DBB0000357050001CB63E7E50083478500BA976B
:10DBC000E3CFF5FA05044DB7EF428F95C1642A897A
:10DBD00001449789FF1F93896921130A8006FD1468
:10DBE000EFA0AFCF6344A4006F40CF96330544034A
:10DBF00083A709023E958357E50063889700630475
:10DC0000990063942701EFF07FAB0504D1BFEF4289
:10DC1000CF8F89692A8AAE8A328BB68B8144178C62
:10DC2000FF1F130CAC1C930C8006314DFD19EFA0A7
:10DC3000CFCA63C4A4006F400F9133899403832734
:10DC40000C028355CA015A863E994A85EFF07FB08F
:10DC500005CD814D05A03384AD038327090303D689
:10DC60000B00D68533F6C9003E942285EFF07FC4C1
:10DC700019E5850DEFA06FC4E3CFADFC31A022857F
:10DC8000EFF0FFA023040400850455B7EF426F882E
:10DC90004169AA8A014A178BFF1F130B2B157D19A7
:10DCA000C14B054CEFA06FC36344AA006F40EF89DE
:10DCB00093098006B3073A0383290B02BE9983D7E1
:10DCC000E900638C270163842A016398570103A448
:10DCD000890311E44E85EFF0DFC9050AE1B78357E8
:10DCE0000401639977079304C4002685EFA03FF0F1
:10DCF00085452A8D2685835C0401EFA0DFEC26850F
:10DD0000EFA0FFFF62056185635F05028D452685F3
:10DD1000EFA07FEB89452685EFA0FFEA89452685A0
:10DD2000EFA07FEA85452685EFA03FEB83470500FE
:10DD3000094793F7F7076398E70099452685EFA011
:10DD4000DFE9A30285014848337D2D0123189401A2
:10DD50006A9548C40040B5BFEF323FFE37E4040087
:10DD60008327041D82979787FF1F83C727F51755C1
:10DD7000FF1F1305253EA300F5008327441C82974F
:10DD80008327841C81461306F00F81450145829745
:10DD90006F30FFFC1787FF1F130747E21843978573
:10DDA000FF1F83C5A5F19787FF1F9387A7EF8346C2
:10DDB0008703034697036397D5009787FF1F238F39
:10DDC000C7EE828083C587010347A7036317B600A8
:10DDD0009787FF1F2384E7EE828003C687016317BE
:10DDE000C7009787FF1F238BD7EC828083C68701EC
:10DDF000130750026319D700930760021787FF1FAC
:10DE0000230EF7EA828083C687011306600263153A
:10DE1000D60093077002DDB783C7870155BF978788
:10DE2000FF1F938727E8D44B09476385E608EF3245
:10DE3000DFF01789FF1F130929E43E848347090097
:10DE4000918B9DCFB7E4040083A7041D829783A71D
:10DE5000441C1785FF1F1305A5E2829783A7841C26
:10DE600081461786FF1F0346A6E381450145829739
:10DE700021C183470900ED9B1787FF1F230EF7DEA3
:10DE80008347040093F7F70F85C791471787FF1F54
:10DE90002324F7E2EFF05FECEFF0DFEFB7E70400E9
:10DEA000BC4F414691451785FF1F034525E08297EA
:10DEB0006F30FFEA8280EF325FE88D4741116304E3
:10DEC000F504C5476306F50285476310F502978799
:10DED000FF1F2387A7DEB7E70400BC4B93050010A4
:10DEE0001785FF1F034585DC829741016F303FE7AF
:10DEF00085471787FF1F2305F7DCB7E70400BC4BF6
:10DF000093050020F1BF9787FF1F9387A7D9D44BB4
:10DF10001147638DE600B7E7040083A7071D8297CA
:10DF2000B7E70400BC4B930500045DBF05491787A4
:10DF3000FF1F232327D983C7070032C62E8493F7F8
:10DF4000F70FC5D7B7E4040083A7041D7D1413742D
:10DF5000F40F8297E37689FCB245994703C6150012
:10DF6000E3F0C7FCFC4409061785FF1F130585D5A0
:10DF70008297BC48930500081785FF1F034505D30A
:10DF8000829779BFEF327FDB1787FF1F130787D197
:10DF90004047184B1C409786FF1F23ABF6D06316F3
:10DFA000E4001787FF1F2327F7D0130584FEEF90A7
:10DFB0007FF3035564FFEF903FC6EFA0BFE96F30DA
:10DFC0001FDAEF329FD79787FF1F9387A7CDD84BD4
:10DFD000DC4799C3EFF01FFB85471787FF1F232DF1
:10DFE000F7CC9787FF1F938767BD9C43930500027B
:10DFF0001785FF1F034585CB83C787031787FF1F3F
:10E00000230EF7CAB7E70400BC4B82976F303FD5A9
:10E010009787FF1F23AAA7C88280EF327FD037E4FB
:10E0200004007C4CA1451785FF1F034525C8829736
:10E030007C48A1451785FF1F034545C79784FF1FEF
:10E04000938444C68297DC4489E7EFF05FDD6F304C
:10E050007FD003D567FFEF903FBCAA897DD5D84814
:10E0600091476310F7027C4C91451785FF1F0345CC
:10E07000E5C382977C4891451785FF1F034505C37B
:10E08000829703A9490103D409018947B7E904002C
:10E090001787FF1F2322F7C283A7091D210442040B
:10E0A000829783C784011755FF1F1305A50A6119BD
:10E0B0001757FF1FA300F70A83A7491C41808297C7
:10E0C0009787FF1F238E07BE83A7C91C8146094679
:10E0D0009375F40F4A85829711E99787FF1F83C7CD
:10E0E00067CE89C79740FF1FE7808078B7E70400B5
:10E0F000BC4F2146A1451785FF1F034525BB8297CD
:10E10000B9B7EF329FC393F7052001112E8481CB5D
:10E11000EFF03FEB1345042005616F305FC493F7C8
:10E120000510A9CB9784FF1F9384C4B7DC48EFF098
:10E130007FC61787FF1F130767A8184383C784018B
:10E14000034787036316F700DC4499C3EFF09FE3AE
:10E1500085471787FF1F2321F7B6B7E70400BC4B9D
:10E16000930500021785FF1F034545B482971345A9
:10E1700004105DB793F70508ADC79787FF1F83C7E6
:10E1800077B4E91719469785FF1F9385C5B3130523
:10E19000D10093F4F70F1789FF1F0349A9B2EFA02D
:10E1A000902393970401C1831787FF1F130707B2BA
:10E1B000231DF100231CF1009787FF1F938787AE73
:10E1C0003ACE3ACAD8432306010009CBDC43931563
:10E1D000890154080D46E1856800829713450408BB
:10E1E00025BF93F72500B1CF9787FF1F938787AB94
:10E1F000D84B89476306F7029787FF1F83C7C7A7D6
:10E2000013F7270011EF918B99CFB7E70400BC4FAC
:10E210001306000A89451785FF1F034525A9829724
:10E2200013452400D5BD9787FF1F938727999C43EB
:10E2300083C787031787FF1F2302F7A8EFF0FFDDCF
:10E24000C5B793F7050291C7EFF03FDD1345040210
:10E25000E1B593F7850091C7EFF0BFD61345840071
:10E2600065BD93F7150091C7EFF07FBB1345140010
:10E2700065B593F7450091C7EFF07FBA13454400A9
:10E2800061BD93F7050485C39787FF1F83C787A1E7
:10E2900081CBEFF07FAC91471787FF1F232EF7A0AC
:10E2A0001345040495BD93F705010145E38607E690
:10E2B0009787FF1F9387079FD84B91476310F704F9
:10E2C0009787FF1F9387479B9C4313D7270085831E
:10E2D000D98F858B91E7B7E7040083A7071D829745
:10E2E000B7E70400FC4F91451785FF1F0345059CC8
:10E2F000829785471787FF1F2320F79C134504014A
:10E3000021BD9787FF1F238FA7AA8280EF32FFA22C
:10E310009787FF1F23AE07989787FF1F23AC0798A7
:10E3200085471784FF1F130464891787FF1F232560
:10E33000F7981C4083C787031787FF1F2300F798B0
:10E34000EF90FFDF39C19757FF1F23A9A7E01C40BB
:10E3500017050000130525DB83C787031787FF1FF9
:10E36000230EF7941757FF1FA306F7DE9787FF1FAB
:10E37000A38A0792B7E7040083A7070882979787C5
:10E38000FF1F2385A7926F309F9DB7C7898E938704
:10E3900067ED1757FF1F2323F7DC55BF1787FF1FB4
:10E3A00003474790795555E39787FF1F9387878FDA
:10E3B00003C7170005079786FF1FA385E68E03C7CF
:10E3C00017008D463377D7029786FF1FA38CE68C04
:10E3D00083C617001777FF1F1307477E184393F66E
:10E3E000F60FA9EA834787031787FF1F2308F78CD7
:10E3F00085471787FF1F2307F78A9787FF1F938794
:10E40000A7879C430145998BA9E3EF321F9337E41B
:10E4100004007C48C1451785FF1F03452589829765
:10E420003C4885451785FF1F034545888297014570
:10E430006F30FF9283C7170085466395F6008347C8
:10E4400097035DB78347A70345B782809787FF1F70
:10E4500083C74785A1CBEF325F8E37E404009787EF
:10E46000FF1F238107847C4885451785FF1F0345CF
:10E47000E58382977C4C91451785FF1F03450583F3
:10E4800082977C4891451785FF1F03452582829717
:10E490003C48C1451785FF1F0345458182970145CB
:10E4A0006F30FF8B79558280EF323F892A84035584
:10E4B00065FFEF906FF69777FF1F9387A77ED8478A
:10E4C000BE841DEBEFA05F989C48232004008DEBD9
:10E4D0009777FF1F23A0877E9777FF1F23AA877C4C
:10E4E000B7E70400BC4B89451775FF1F0345057C42
:10E4F000829701456F30BF86630A87001843D1B702
:10E5000080C39777FF1F23A7877AD9BF7955DDB7D7
:10E51000EF32BF829787FF1F9387078B884323269D
:10E520000500232405005105EF80D02E6F303F8376
:10E53000EF32BF801784FF1F130404891C40411170
:10E5400089CF9C472302B5002AC61CC1EFF05FFCAF
:10E550001C409C4B99C33245829741016F303F80EC
:10E56000EF32AFFD4111444D328532842EC6EFA00B
:10E570000FF92AC42285EFA0EFF903A84400630C29
:10E580000800B245835744001840224683D5450011
:10E59000AA862685029841016F306FFCEF32EFF9B1
:10E5A000404D1DC408C0970500009385E502130582
:10E5B0004401EF8090189787FF1F9387E7809C4363
:10E5C000014589E79787FF1F23A087806F302FF9C8
:10E5D0007D55EDBFEF326FF6011168009305F00F26
:10E5E00002C602C802CA02CC02CEEFF07FF4056177
:10E5F0006F30EFF69777FF1F9387077D9C43D847CF
:10E60000A1679D076311F702EF322FF301113285E5
:10E61000EFA0EFEE230AA10081456800EFF05FF163
:10E6200005616F30CFF382809777FF1F9387C7799B
:10E630009C43D847A167938777036311F702EF32B2
:10E64000CFEF01113285EFA08FEB230AA1008145A6
:10E650006800EFF0FFED05616F306FF08280977713
:10E66000FF1F938767769C43D8479547631CF70243
:10E67000EF32AFEC011132853284EFA04FE8230A6C
:10E68000A1002285EFA00FE983574400231BA100BE
:10E6900081453ECC1C4068003ECEEFF07FE905612D
:10E6A0006F30EFEB8280930785FF89CF8327C5FF0B
:10E6B00091CBDC4B81CBEF324FE8032585FF82976E
:10E6C0006F30EFE98280EF324FE72A843285EFA086
:10E6D0000FE3BD4763EBA70018449377F5000345AC
:10E6E000B70041995D8DA305A7006F304FE7EF326A
:10E6F000CFE401117C003ECAB70707003ECC7C0086
:10E700003ECE5C4D8DCF2A8413858700AE84EF808A
:10E710007004A1652A899D054808EF80FFBD930517
:10E72000803EB345B902480893F5F50FEFA0CFD26C
:10E73000014781465008A6852285EF807FDC056170
:10E740006F30EFE1EF326FDFEFF07FFA6F302FE1E4
:10E75000EF32AFDE01117C00AE843ECAA165B7077F
:10E7600007002A843ECC48087C00938575033ECE82
:10E77000EF809FB81C44480883C5B700BD89EFA04F
:10E78000AFCD500801478146A6852285EF805FD72F
:10E7900005616F30CFDCEF324FDA2A84AE84EFF0C0
:10E7A0009FF2A6852285EFF0BFFA6F304FDBEF3284
:10E7B000CFD8EFF0FFF96F308FDAEF320FD803299F
:10E7C000C5014111630409022A843285B284EFA095
:10E7D0000FD32AC62685EFA0EFD3832749002A86C8
:10E7E00091C7DC4781C7B2452285829741016F30CE
:10E7F0000FD7EF328FD4444D81CC2A843285EFA0DD
:10E800006FD1DC40AA8589C79C4799C3228582972E
:10E810006F30EFD4EF32CFD0032AC501411163032B
:10E820000A062E89AA84954532853284EF80DFACB2
:10E8300085452285EFA0CFBDAA89CA852285EFA094
:10E84000EFC283274A009DC7DC438DC72285EFA016
:10E85000AFBA83274A00104083564400DC43711549
:10E86000A307A100B2961307F1004E86CA8526853C
:10E87000829701C52380090031A08345F1002285DC
:10E88000EFA00FB941016F30EFCCEF320FCB6571C4
:10E890001C083EC2B70780013EC41C0832893EC630
:10E8A0002A84AE84EFF07FF14A85EFA0AFC683578C
:10E8B000A10089CFAA8550002285EFF0BFF501475E
:10E8C00081465000A6852285EF809FC359616F3035
:10E8D0000FC9EF32EFC465711C088329C5013EC220
:10E8E000B70780013EC41C082A84AE8432893EC624
:10E8F000EFF03FF0638409024A85EFA0AFC1835770
:10E90000A100AA8581CF50002285EFF0BFF001471A
:10E9100081465000A6852285EF809FBE59616F30E9
:10E920006FC3EF328FC165711C083EC2B70780010B
:10E930003EC42A841C0832853EC6AE84EFA08FBD3B
:10E940008357A10089CFAA8550002285EFF09FEC64
:10E95000014781465000A6852285EF807FBA596124
:10E960006F30EFBFEF326FBD444D91E883474500F4
:10E9700093B71700B307F0403E856F304FBE184580
:10E98000FD577DDB97070000938707032A845CCB44
:10E9900097050000938565D113858400EF80E059C9
:10E9A00080C003474400814761FB1777FF1F232F77
:10E9B0009740D9B7EF32CFB68329C501411103295A
:10E9C00085008147638B09080324090191452A8A40
:10E9D0002285EF807F9285452285EFA06FA3894530
:10E9E000AA8A2285EFA0CFA2AA84EF809F9683A750
:10E9F00049002A8B9DC79C438DC72285EFA0CF9FDE
:10EA000083A74900A306A1001040835644009C43FD
:10EA10001307D100B296D6851306E100528582977E
:10EA200009CD83570B002380F400A183A380F40059
:10EA300023800A00A306010029A88357E10022854C
:10EA40002380F4008345D100A183A380F400EFA0CC
:10EA50002F9C8347D100B337F0000347B9009207DA
:10EA600001453D9BD98FA305F90041016F308FAE61
:10EA7000EF32AFAC41111DE99777FF1F9387073540
:10EA8000804305C80440130984009DC55C4099C7B4
:10EA90009C4B89C726852EC68297B2459307803E38
:10EAA000B385F5024A85EF80605521A0404DAA84C8
:10EAB00079F841016F30AFAA4A85EF80A0555C40DC
:10EAC000EDDBDC4BFDD726858297E5B7EF32EFA66D
:10EAD0002A843285EFA0AFA2AA852285EFF05FF9E4
:10EAE0006F30EFA7EF326FA52A84AE84EFF01FFEE0
:10EAF000A6852285EFF0BFBF6F306FA60841335562
:10EB0000B50005898280EF324FA31774FF1F1304ED
:10EB1000E42D1C5C0111231701008D83858BA30359
:10EB2000F1008327040B231801002319010003D7E8
:10EB3000C7013ECA3C002314E1007D572315E100C4
:10EB40000357C4023ECC02CE2316E100EF802FE330
:10EB50008357E101231EA10093F707E093E7171005
:10EB6000231FF1009777FF1F83C7E72A85C3054757
:10EB70000145638AE7008347840393E727001777FB
:10EB8000FF1F2301F72A05616F306F9D814717D75B
:10EB900000001307271C85461306710085454808A9
:10EBA000EF70E04B6DF183478403F59B1777FF1FF0
:10EBB000230AF72685471777FF1F230EF724E1B7AF
:10EBC000EF32AF94977DFF1F938D4D2203A6CD06A4
:10EBD00039712A8981478144930600023357F60030
:10EBE000058B01C7850493F4F40F8507E398D7FEDE
:10EBF00083A70D0B231701022318010203D7C701B6
:10EC00003EDA3C102314E1027D572315E10203D7BD
:10EC1000CD023EDC231901022316E10202DEEF8061
:10EC20000FD68357E103231EA102014593F707E0A6
:10EC300093E71710231FF1029777FF1F83C7A71DC4
:10EC4000A9EF9777FF1F83C7F71D3EC69779FF1F70
:10EC50009389C9190144014D9D4A054B954B177C79
:10EC6000FF1F130CEC1F977CFF1F938CEC1E03DA25
:10EC7000C90563090A00EA85631459036685EFF044
:10EC8000FFE71DC1050DA1478909E312FDFE2DE037
:10EC90009777FF1F23A4071C014521616F30AF8ABE
:10ECA0006285EFF0BFE579DD3247B3878400E3F09A
:10ECB000E7FE9C001306140006043E9413178A0016
:10ECC00093578A00D98FC207C183A30EF4FCA18396
:10ECD000230FF4FC03A70D07B317AB01D98F1777E8
:10ECE000FF1F232DF71663047601328461BF15449C
:10ECF0009777FF1F83C70712138717009776FF1FA9
:10ED0000238AE61093161400230EF10017D7000093
:10ED100013074704814785067008CA854818EF70B5
:10ED20000034E34705F68347C10105451777FF1F08
:10ED3000A302F70E9777FF1F238F270DB9BFEF228E
:10ED40003FFE0111AA892E84EFD0EF9C2A89977487
:10ED5000FF1F9384A4096399090A9C5C414793F7B8
:10ED600007036393E70A1777FF1F0347170B8947CA
:10ED700063ECE70883A7040B2317010023180100A5
:10ED800003D7C7013ECA3C002314E1007D57231579
:10ED9000E10003D7C4023ECC231901002316E10091
:10EDA00002CEEF80CFBD231EA100EFC06FCD8357F1
:10EDB000C101230FA100914613D78700A207D98F65
:10EDC0002312F1009777FF1F83D7E70513D787003A
:10EDD000A207D98F2313F10017D70000130707F7F5
:10EDE0008147500095454808EF70602705889317C4
:10EDF000240003C484036D985D8C9777FF1F2383E1
:10EE0000870205616F201FF5EF70B0781775FF1F3F
:10EE10001305C501EF80002083A7040B9775FF1F22
:10EE200083D585FF03D5C701EF10E0279777FF1F34
:10EE300083C747FF93F60702014789E61777FF1F4D
:10EE4000035787FD9776FF1F2390E6FE1777FF1F76
:10EE5000130787F8184309CBC18B99C789451775E4
:10EE6000FF1F035565FB02979777FF1F23A607FA3D
:10EE70009777FF1F238107FA9777FF1F23AE07FCC1
:10EE80009777FF1F23AC07FC9777FF1F23AA07FC88
:10EE900083D7840393F7270C93E717001777FF1F97
:10EEA0002312F7F883572903A18B99C3EF70E03F32
:10EEB00011C49777FF1F23AD07F4A1B78D471777CC
:10EEC000FF1F2327F7F4EF902FA59305803EB3058E
:10EED000B5021775FF1F130565F5EF80201215B7F2
:10EEE0009777FF1F938787F0D85325C791C99777E6
:10EEF000FF1F238207F29777FF1F23A107F6828067
:10EF0000EF22BFE383C7F70241112EC685071777AB
:10EF1000FF1FA304F7F09777FF1F2398A7F09D47E3
:10EF20001777FF1F2326F7EEEF900F9E2A84EF90AE
:10EF3000AF9DB24501E5EF902F9DAA85B305B44082
:10EF40001775FF1F130585EEEF80400B41016F2001
:10EF50001FE182809777FF1F938747E9D85331C716
:10EF6000EF22BFDD03C7F70205079776FF1FA386D1
:10EF7000E6EA11CD8C5F0D47014589818589977639
:10EF8000FF1F23A7E6E8EFF09FDB6F205FDD8547DB
:10EF90009305C0441775FF1F130545E91777FF1F39
:10EFA0002328F7E6EF808005CDB78280EF22FFD8D7
:10EFB0001777FF1F034727E68547631EF7009777FC
:10EFC000FF1F9387A7E283C7870393C7870017773D
:10EFD000FF1F2309F7E41775FF1F130525E5EF80D1
:10EFE0006003EF807FEF99471777FF1F2322F7E237
:10EFF0009777FF1FA38307E29777FF1F238D07E013
:10F00000EF90AF8F930740063305F5029777FF1F08
:10F0100023A6A7E06F20BFD49777FF1F83C787E0A1
:10F02000C18B99C7EF227FD1EFF0FFAD6F203FD3A7
:10F03000695582809777FF1F938747DBDC5381CB2D
:10F04000EF22BFCF8545EFF09FCF6F205FD1828049
:10F050001777FF1F130787D901468146BA852148D4
:10F06000631E06019DCA2390A60083C7850393E70C
:10F0700017001777FF1F2307F7DA05A08357C70587
:10F08000631DF502F8598547B397C70093C7F7FF8B
:10F09000F98F1777FF1F2325F7DC9C5D9183858B04
:10F0A00085C79777FF1F83C707D799EFEF22FFC860
:10F0B0001D45EFF0FFB06F209FCA81E699E39306EC
:10F0C000C7050506090769BF8280EF229FC4860530
:10F0D000AA84B309B500977AFF1F938AEAD7054B34
:10F0E000977BFF1F938B8BD7214C639434039777C7
:10F0F000FF1F9387A7CF9C5F9183858B89CB9777E1
:10F10000FF1F83C747D181E72145EFF07FAB6F2019
:10F11000DFC303DA0400630B0A041779FF1F130926
:10F12000E9CC0144CA8C8357C905639D4703A28576
:10F130005685EFF0BF9C11E5A2855E85EFF01F9C20
:10F1400005C903A74C07B3178B00D98F1777FF1F8B
:10F150002328F7D083C78C0393E717001777FF1F87
:10F160002302F7CC05040909E31F84FB8904B5BF1A
:10F17000231E0904C5BF1777FF1F0347C7C985476B
:10F18000631AF700EF227FBBEFF05FE2EFF0BF976B
:10F190006F20FFBC8280814785451306000293865D
:10F1A0001700B397F500E98F13F7F60F89E7B687D5
:10F1B000E397C6FE01473A858280FD4785457D5627
:10F1C000B396F50013871700E98E1377F70F89E6DA
:10F1D000FD17E397C7FE01473A85828089E9014719
:10F1E0003A85828001473A8541016F205FB7EF225F
:10F1F000DFB441112AC62E852EC4EFF0DFF9A245F7
:10F200007D158547B397A700E39EF5FC32469377BB
:10F21000360099C3719A11069777FF1F9387C7BC71
:10F2200094433E871778FF1F130848BB89EA83275A
:10F2300008009107F19B9776FF1F23A7F6BA0325D5
:10F2400088001843B307A700B3F7B702B387F540A8
:10F25000FD15FD8D83274800AA95B306B600E3F39C
:10F26000F6F8E371D5F82E979777FF1F23ACD7B642
:10F270003DDB3A858145EF205FAF2A87ADB7184166
:10F280009777FF1F938787B523A4070098C358413A
:10F29000D8C39777FF1F23A907B48280EF225FA806
:10F2A000AA8401441779FF1F130949B49309400E3A
:10F2B000EF807FD56345A40001456F20BFA93305CA
:10F2C00034038327090B3E958357C501E38797FED7
:10F2D0000504F9BFEF22FFA39779FF1F938909B1B6
:10F2E0003E84BA848347060003A7090041119D8329
:10F2F000058B3D8F83C74401AE8A2A89F99BD98F3C
:10F30000238AF4001C44B685231204001CC0228505
:10F31000328A36C6EF90DF8FB246D2853686EF90BE
:10F32000900BDC4883A509000840858B56869D8D8F
:10F33000EFD03FCC61E918407D5583475700034724
:10F340006700A207D98FC207C1872394F4006358CE
:10F35000F00A83C7440193F70703B5CBD0489377EE
:10F36000160003A609001D8E9777FF1F9387C7DE3F
:10F370009C43ADEB814641A003A70B0093172A00E5
:10F38000BA9718409443834757008345670033F684
:10F390005601A207CD8F6311F6028347370003465B
:10F3A000470003472700A207D18F4207D98FBD82AC
:10F3B000B3F76701638AF604050AEF80DFC34205ED
:10F3C00093170A014181C183E3E8A7FA41BFA16A0B
:10F3D000370B0200014A977BFF1F938BEBAEFD1AA0
:10F3E0007D1BE1BF83C7440113070003854693F7E4
:10F3F0000703E391E7F8A2854A85EFD0FFCF4101EB
:10F400006F20BF946155E5BF7955D5BFEF225F915D
:10F410009774FF1F9384C4859C40D9EF9777FF1F93
:10F420009387479B9C436399070CEF80DFBE93074C
:10F4300080023305F5028945EFF05FDA41C997771D
:10F44000FF1F23ABA7A4EF801FBC9307400E33051B
:10F45000F5029145EFF09FD835C99777FF1F23AF8D
:10F46000A7A2EF805FB201CDEF80FFB191450E05FD
:10F47000EFF0DFD621CD9777FF1F23A3A7A2EF8060
:10F480001FCB11CDEF80BFCAD9473305F50289459F
:10F49000EFF0DFD405CD9777FF1F23ADA79EEF8058
:10F4A0009FB591450A05EFF07FD30DC19777FF1FF8
:10F4B00023ACA7A0014521A8EF803FC29307800697
:10F4C0003305F5029145EFF07FD101E565556F20D9
:10F4D0007F889777FF1F23ABA7920144130A80060A
:10F4E0001779FF1F13098990B14AEF801FBF63642A
:10F4F000A4029C40E38407F2EF803FBE9307A00480
:10F500003305F5028945EFF07FCD69D19777FF1F6D
:10F5100023A0A79C19BFEF805FBB89450605EFF0CC
:10F52000FFCB4DD5B3094403032709024E9708CBFF
:10F53000EF80BFB8330555039145EFF03FCA59D569
:10F540008327090205041374F40FCE9788DB71BF7B
:10F550009777FF1F93878789884705898280C167CE
:10F56000FD176319F5009777FF1F9387278803A579
:10F57000070B8280EF226FFCEFF05FD26F202FFE2F
:10F58000814709C58347E501B337F0001777FF1FAF
:10F590001307C78518470983058B19C393E727000D
:10F5A0003E858280EF226FF92A84EFF07FFD83474A
:10F5B000E401AA851305940899E3130504039776DB
:10F5C000FF1F9386A6829442130615021307840236
:10F5D00013059504EFD0CFC06F206FF8EF224FF4E2
:10F5E0009774FF1F9384848098442A892E8409830A
:10F5F000058B9C4019C76314F5006380050E014418
:10F6000001A2E3FEA7FE1387A702E36AA7FE850710
:10F6100063FCA70883A9440BEF80FF9613163500FF
:10F6200081454E85EF206FF49767FF1F23A0277D4C
:10F630009767FF1F23AE077A49CC9C4493E74700A6
:10F640001767FF1F2328F77A9777FF1F238C078000
:10F65000630F040C9767FF1F23AA2779014405490C
:10F66000EF807F926341A40AEF80FF949305000628
:10F67000B3C5A502B7F73600938707E81765FF1FE4
:10F680001305857E416901449309400E7D19B385B8
:10F69000F502EF70B016EF801F97634FA408014585
:10F6A000EF3040700544A9A86398A7029DE583A99F
:10F6B000440BEF805F8D1316350081454E85EF209A
:10F6C000CFEA9767FF1F23A327739767FF1F23A125
:10F6D00007729C44ED9BADB785C51767FF1F0347B5
:10F6E00067789307F005E3FCE7F021F8EF60F03C62
:10F6F0006DD19C4493E707021767FF1F232CF76E19
:10F7000022856F202FE583A7440B131534003E9507
:10F710008357050081CB8347250099C72146814542
:10F72000EF20AFE405042DBF23012501E5BF976756
:10F73000FF1F23AF076A0DBF3305340383A7040BF4
:10F740003E958357C50163842701EFF0BFE50504AB
:10F7500099B7EF228FDEEF801F8613040006334532
:10F76000A4029764FF1F9384646883C784073E954F
:10F770001375F50F9767FF1F2386A76E9307F00594
:10F7800063E7A7020545EF30E061EF80DF82334594
:10F79000A402B7F53600938505E8B305B5021765F1
:10F7A000FF1F1305656CEF7070056F204FDB9C44E5
:10F7B00005458983858B81CBEF904F8888408145B3
:10F7C000EFF0DFE1DDB7EF30E05DC5B7EF224FD5F9
:10F7D000130495082A8913069005A28513050503CD
:10F7E000EF90603F1306900581452285EF20EFD70B
:10F7F0004A85EF30C0548144176AFF1F130A0A5F1D
:10F80000930A8002EF803F8163C4A4006F208FD4ED
:10F81000338454038327CA0A3E9403570400835752
:10F82000C9016317F702834744009DC3930964012C
:10F830004546CE8513055400EF90E0394546814595
:10F840004E85EF208FD2228523020400EF3000572F
:10F8500085044DBFEF226FCE9767FF1F9387474107
:10F860009C432A8491C70DC50355C501EFE00FC223
:10F870009777FF1F9387478E9C4389CBEFB0DFD0EC
:10F8800085476315F5002285EF50C05D6F202FCDB1
:10F8900041657D15E1BFEF224FCA1764FF1F1304B6
:10F8A000E4544440938714001767FF1F2322F75442
:10F8B000EF30605E1C448983858B9DE75840B7E735
:10F8C000B0009387075063F1E7020145EFF01F9DF9
:10F8D00001CD0545EF809FF6084085450505EFF011
:10F8E000FFCF0145EFF01FF726856F204FC7EF22AE
:10F8F0002FC3A1642A8901449769FF1F9389C95CBA
:10F90000FD14338AA500EF800FEF6344A4006F203D
:10F910006FC403A7090093172400BA979843658F13
:10F9200042074183634C2701635A47012380070044
:10F93000A380070023810700A38107000504E1B726
:10F94000EF22AFBC83594500C547411163F53731FC
:10F950000441C1E533853401834785FF034795FFA3
:10F960000348B5FFA207D98F0347A5FFC2072207A7
:10F9700033670701D98F0347C5FF0348D5FF220727
:10F98000336707010348E5FF0345F5FF42072208F7
:10F990003365A800498FB98F1767FF1F130787507A
:10F9A0001768FF1F130808523A85832807006384ED
:10F9B000172B1107E31B07FF1767FF1F130787505C
:10F9C00018431318270042951CC10507A147336748
:10F9D000F7029767FF1F23A7E74E93F735001397AA
:10F9E000470083474601C16B368993F7F7FCD98FEF
:10F9F00032842E8A230AF600814A176CFF1F130CEB
:10FA0000EC3EFD1B976CFF1F938C8C26176DFF1F20
:10FA1000130D0D4CEF802FDF63C7AA00E15426853C
:10FA200041016F204FB21308400EB3870A03032829
:10FA30000C0BB30DF800638E0D2083D7CD01638AC4
:10FA4000772183A70C00014B639707169767FF1F69
:10FA5000938747389C436390071683C7040003C706
:10FA60000D0493F7F707631BF71ACA872287CE8620
:10FA7000268693859D0613851D04EFF0BF85631FC1
:10FA8000051883D7CD01032709002320B4012312D1
:10FA9000F400FD572313F4008347170093F6F7078C
:10FAA0008347D40093F707F8D58FA306F40093F7A4
:10FAB000F707B337F000B307F0402307F40083479C
:10FAC00017009D839396370083474401DD9BD58FB4
:10FAD000230AF4008347370083464700A207D58FE7
:10FAE00083462700C206D58F1CC88347770003478B
:10FAF0008700A207D98F2315F4000D476304EA009D
:10FB0000BD5491DF93870710C207C1831307B00F5D
:10FB1000BD54E376F7F0EF800FC98144E31105F09F
:10FB20009766FF1F83C6863A938716001767FF1FE5
:10FB3000230EF7381767FF1F13070739231BD4005D
:10FB400093972600144303578400E175BE96A1677E
:10FB50001386F7FFB377C70098426D8FD98F9CC289
:10FB60001848F18F3E07D98F9CC2EF80CFC89767A6
:10FB7000FF1F83C7A73533F5A7029767FF1F2387AA
:10FB8000A73471BD9307A004B308FB0283270D00BF
:10FB9000BE9803D7080083D7CD01631DF70083C744
:10FBA000040003C7880093F7F707630BF70083C7C8
:10FBB000FD019DEB050BEF804FD2E345ABFC71BD22
:10FBC0009385980113859800CA872287CE8626865A
:10FBD00046C6EFF02FF0B24879F98347440193E726
:10FBE0004700230AF40071BD83C7040003C79802CD
:10FBF00093F7F707E310F7FCCA872287CE8626869D
:10FC00009385A8031385A802EFF0CFEC45F5834751
:10FC1000440193E72700230AF400C1B783C7FD011D
:10FC20008DCB83C7040003C79D0993F7F7076312C1
:10FC3000F702CA872287CE86268693852D0C1385E8
:10FC4000AD09EFF02FE911E58347440193E7270061
:10FC500049BF850AC1B3FD54D9B3EF228F8B7971A7
:10FC600083544500AA8B2E84B28AEF80CFBB5905FE
:10FC700063499504B7E4040003A90407EF80AFBA11
:10FC800059054205418102992A8905CD2AC62318C2
:10FC90000100EF804FB959052319A1006146814544
:10FCA00028089769FF1F938969144ACAEF20EF8BD0
:10FCB0002302810203A48900058819E4BC544A8503
:10FCC000829745616F206F8874003008D6855E8505
:10FCD000EFF01FC765F56800EF807FF1176AFF1F1F
:10FCE000130A8A4783270A00AA84035B010189CB90
:10FCF00089476397FA00835501025E85EF502030F3
:10FD000003552102EF704FC819E503552102EF702A
:10FD10008FD43334A000931764000344C1022C082D
:10FD200068001374F4FB5D8C23068102EF60B0560B
:10FD3000E9576314F5028356E1029767FF1F938723
:10FD4000A7189C43139726006176BA979843718F42
:10FD500098C39767FF1F238BD7168317210263452C
:10FD6000F00085476396FA00B25793F7070C95E7C2
:10FD7000D247C2040347C102C180BE9426C62318DD
:10FD8000610113770703C147631DF70083475102E1
:10FD9000054793F7F7076390E704B7E70400BC57FC
:10FDA00039BF92570544A18393F7F707E377F4FE31
:10FDB00015C78347C1021307000293F70703639730
:10FDC000E700EFB06FFC8547E319F5FC8347C102FC
:10FDD00093F7070389CFEFB0AFCA21A8EFB08FD751
:10FDE000E30985FCEFB04FFAE31985FAD9B7EFB014
:10FDF000EFD8AA8501460545EF707FF82A8451DDCA
:10FE00008347C102414793F707036384E702324700
:10FE10008347170093F707F8A300F700324792577C
:10FE200083461700A18393F7F707FD17D58FA3002B
:10FE3000F70003560101B245130BC4005A85EF8049
:10FE4000DFDFE24A130690058347C10283C4EA015B
:10FE5000918BB384C40213851404569595C35444FE
:10FE6000B3879A0083C7070403C70600137707F810
:10FE70002380E600584483460700D58F2300F7000F
:10FE8000B25703A609008146858B1D8EDA85EFD017
:10FE9000EF9B15E9B25783A50900484413869406E1
:10FEA000858B56969D8DEFD0CF9411ED83270A0058
:10FEB00099EFB257054791838D8B6387E7049DCFF8
:10FEC00009476389E7042285EF80DFF8F9B5EFB0D1
:10FED000AFEB85476309F5008347C102414793F7BC
:10FEE0000703E398E7FC835521025A85EF40907C95
:10FEF00069D183172102E35EF0FAF1B7EFB08FC545
:10FF00007D151335150061D1014681452285EF70BD
:10FF1000FFEF55BFEFB04FE7E5B7EF121FE2976471
:10FF2000FF1F938424EE2685EF809FEB2A8419E13E
:10FF30006F10FFE21305C40005468145EFF0FFD1C5
:10FF40002285EF803FF1C5B7EF123FDF4111AE844C
:10FF50002A8493079503130715019306F1000546BC
:10FF60006C00268523060100EFD0CFBE1DEDA685CF
:10FF700041462285EF8030468347F1009305140205
:10FF800026852308F400EFD06FC805E19767FF1FAF
:10FF90009387871C9C4389EF1306940497C5000040
:10FFA0009385C5DB2685EFD08FD441016F103FDBF1
:10FFB0001306940297C500009385C5DA2685EFD015
:10FFC0000FD379D9DDB7EF12BFD59767FF1F93879E
:10FFD000A7EF8043AE84B289368AAA8AEF80AF81C8
:10FFE0001316250081452285EF103FD89767FF1F24
:10FFF000238E07EC9767FF1F938747DF03A4070B48
:020000040001F9
:1000000013F714003E89230FE400CE8525C713059E
:100010009408EFF07FF301C555556F10BFD38947A2
:10002000A30FF4009767FF1F938707139C430327D1
:100030008900858093B7170086072300F402231EEA
:1000400054019767FF1F23A347DB85889377B7FF8A
:1000500099C0936747001767FF1F232DF7D82285A4
:10006000930700061767FF1F230EF7DEEFF08FD30D
:10007000014565B713050403EFF01FED45D569BFD2
:10008000EF12BFCBFD572310F500231105002312FB
:100090000500231305001306200481452105EF10F8
:1000A000DFCC6F10DFCBEF12BFC74111AA84014430
:1000B0001769FF1F1309C9E19309A0042EC6EF8039
:1000C000CF81B2456344A40061550DA033053403CC
:1000D000832709003E9583572500639CB70083570B
:1000E000050063989700EFF0BFF9014541016F10DB
:1000F0007FC60504E1B7EF12BFC29767FF1F938762
:1001000067CD9C434111AA842E84B28903592500EE
:10011000C1C39767FF1F83D727D0639B2707EF7063
:100120000F862A8903D5240093051002B305B40273
:1001300085472302F10093578900A302F1009357EA
:100140008500A303F10083D744002304A1002546C2
:1001500013D787002305F10083D76400A304E100CF
:100160004E8513D78700A305E1002306F10013870E
:10017000950093879501A105B386B400A6974C001E
:10018000269723032101EFD0EF9C41016F109FBC04
:10019000EF60FFFE51BFEF12BFB84111AA840144C6
:1001A0001769FF1F1309C9D29309A0043AC636C4C0
:1001B00032C22EC0EF707FF282451246A24632470D
:1001C0006344A400615599A0B307340303250900D3
:1001D000AA9703D8070003D5C4016310A80495E9C2
:1001E0001DEE91CA03C6E401930510023306B60260
:1001F00025063E9690C2014511CB83C6E401130645
:100200001002B386C602E506B6971CC341016F1003
:100210007FB403D52700E305B5FC050441BF83C5C2
:10022000E40113051002B385A502BE9583C58500C0
:100230002300B6007DB7EF12BFAE5C4141112A84A6
:1002400003DA2700C167FD17AE843289630CFA0018
:100250002685EF807F9A8D4763EDA7007D5541018C
:100260006F105FAF2E85EF803F999D47E3E2A7FEB9
:10027000F5B75C40268583D54700EF809F90835576
:1002800084002685EF80FF8F8D452685EF803F8E89
:10029000AA89EFF04FE0935705012380F9009357A7
:1002A0008500A380F9002381A9005840C167FD178C
:1002B0008345A7006314FA0093E505082685EF80BF
:1002C0001F8F9767FF1F9387E7B09C430840D9CFE4
:1002D0008347B400858BD9CB7800340013067100B6
:1002E0008145EFF05FEB1DC98347B40018409306CA
:1002F0009005F99BA305F4008347E701B387D70274
:10030000B306F70083C60604A303D100938617043F
:1003100093879706BA96BA9736C43EC61764FF1FEE
:100320001304C4AC1C440C4026858983858B9D8DA9
:10033000834771009E05DD8D93F5F50FEF803F87B4
:100340001C44104022458983858BCA861D8EA68554
:10035000EFC0DFCFE31505F01C440C403246898323
:100360008840858B9D8DEFC0DFC8D5BD8347B40025
:1003700013079005F99BA305F4008347E501B387B4
:10038000E7023307F50003470704A303E1001387DF
:100390001704938797062A973E953AC42AC6BDBF8D
:1003A000EF121F98032A45009307F00FAA84034712
:1003B000AA00AE89328436896316F700EFB06FABBE
:1003C0002305AA00938AC9000146D6852685EFF049
:1003D0009FE62A8A21E51767FF1F1307E7D718430F
:1003E000DC4039C383C6A7000547638FE60283D587
:1003F00047005685EF40102C05C9DC408397470025
:100400006354F00201CC1C4089C74A8681450145EE
:1004100082975C4081C7CA85014582974E85EF80EF
:100420007FA352856F101F93DC4003D54700EF6018
:10043000BFD501E9DC4003D54700EF60DFE181472C
:100440001DCD19C41C4089C74A8681450145829744
:100450004E85EF807F9FAA851765FF1F1305859A3C
:10046000EF80DF9511C45C4081C7CA850145829742
:100470001765FF1F13054598EF60F0368547D84094
:1004800085460346A700E30BD6F8031747006353DE
:10049000E000C9F74A86A2854E85EF703F97BDBF41
:1004A000EF121F88AA8401441769FF1F130949A28C
:1004B0009309A004130A9508EF703FC26344A40097
:1004C000014535A033053403832709003E95835742
:1004D000250099E30504CDB70357050083D7C40170
:1004E000E31AF7FE52868545EFF0FFC065D56F1021
:1004F0007F86EF12FF82AA8401441769FF1F130948
:10050000299D9309A004EF705FBD6344A4006F10A0
:100510007F8433053403832709003E9583572500E4
:1005200081CF8357050063999700930595021306C1
:1005300010022105EF80206A0504F1B7EF12EFFFEA
:100540000347E5012A848347F5016307B70089E77C
:1005500081452E856F10BF80230FB400054781C9E8
:10056000E398E7FE8947A30FF4008545DDB7638B69
:10057000E7020947E39FE7FC2285EFF02FA5976785
:10058000FF1F938727859C4399E79757FF1F938702
:10059000276E9C4389C70355C401EFF09FF5A30F55
:1005A0000400E1B755D6C9BFEF128FF7EFA0FFEEF9
:1005B00085476312F508EF80EFCC1764FF1F130423
:1005C000A4B91C4081CBEFA03FFC89476304F50030
:1005D0001C4082979757FF1F9387C77F9C43B9CFD3
:1005E00082979757FF1F9387A7689C4391C3829771
:1005F0001754FF1F1304847F8327040B83D4C70180
:10060000EF60FFB78327040BAA85144003C6E701F8
:100610001C448983858B99C313662600268541690E
:10062000EF40C03D8144D9497D19EF705FB063CA86
:10063000A4006F102FF2EF800FCA41B7EF705F88F0
:100640004DB7B38734030327840ABA9703D527002D
:100650006308250103C6470183D50700EF40A03B8F
:100660008504E1B7EF12CFEB01449754FF1F938449
:10067000E4771309400EFD59EF70FF98634FA4040F
:1006800001449754FF1F9384647613098002FD5937
:10069000EF707F98634CA40401449754FF1F938428
:1006A000E4745949FD59EF709FA8634AA40497F573
:1006B000FFFF9385450A1755FF1F1305E57AEF6085
:1006C000D00797050000938585851755FF1F1305F3
:1006D000A572EF6050056F10EFE73307240383A77F
:1006E000040B0504BA97239E370179B73307240317
:1006F00083A7C40A0504BA972390370151BF330773
:10070000240383A7840A0504BA972391370161BFA4
:10071000D4410387350085473356F5026377E600F9
:10072000A54899E7238006008280B387E702EDB7EA
:100730003358F502038735003375F502B3D7E70266
:100740001307000363DA080103C6050013077003EB
:10075000118A19E21307700585064297A38FE6FEFA
:10076000C9B718451C416376F7005C41BA972380EE
:10077000B7001C4585071CC58280EF120FDC4111B4
:10078000AA872E85B285368636C6829763480500CD
:10079000B246158D3335A0003305A04041016F10DE
:1007A0000FDCEF12EFD7056941112A8A23200600DA
:1007B00001448149975AFF1F938A0A74056B7D197A
:1007C00032C62EC4EF703F85AA84EF70DF83269572
:1007D000A24532466346A4004E8541016F108FD773
:1007E00003A70A0093171400BA9703D707003377BB
:1007F000670101E71CC20504E1B703D70700935660
:10080000D700858AE39946FF33772701E315B7FEC2
:10081000BE89D5B7EF126FD201112EC6B2843689C8
:10082000EFB02FEE2A84615501C8B24589E9232E25
:10083000040023200402014505616F104FD2A14638
:100840003008CA852685EFF05FF37DF58357810177
:100850000357A101231EF4008357C1012310E402B2
:100860002311F4028357E101D207D1832312F4024A
:100870008357E1011397370163560700FD57231F84
:10088000F4005DBF231F040045BFEF126FC917546A
:10089000FF1F1304A4558327040B03D7C701C167A7
:1008A000FD17630EF7109767FF1F9387278B9C43F5
:1008B00081C70545EF406077C1690149930A400E41
:1008C000FD19176BFF1F130B2B89EF70CFF3634BD1
:1008D000A90E1757FF1F0347E7589307F00563E476
:1008E000E702EF704FED93050006B3C5A502B7F719
:1008F0003600938707E81755FF1F1305E556B385A4
:10090000F502EF60A06F81451705000013058520F3
:10091000EF60DFF8EFB0EFDE01CD0357C50109CB83
:100920000357E50111C78347050299C3EF60A06B28
:10093000EFB06FDE31C51757FF1F0347675F97574B
:10094000FF1F9387E75E0DCF03C717002304E50061
:1009500003C72700A304E50003C737002305E5000C
:1009600003C74700A305E50003C757002306E500BA
:1009700003C7670083C77700A306E5002307F500D8
:100980001C4493E717001757FF1F2325F7465C40C9
:1009900085E7EF708FEF0DC1EF702FEF44402A898C
:1009A000EF70AFEE33F5A4025C40FD17CA97898F54
:1009B0001757FF1F232EF7420145EF70DF9F0145B8
:1009C0006F104FB9B30459038327040BBE9483D728
:1009D000C40163883703138A0403D2855285EFF07C
:1009E000AFD605E183C7F40199CF938594082E858E
:1009F000EFF08FD509C91306900581455285EF1098
:100A0000CFB60509D9B583270B00268593B7170004
:100A100086072380F402EFE0FFB8E5B7854763F867
:100A2000A7009307F5FFBE953305A040E98D2E85FD
:100A300082809841C167BA9713D707016304A70062
:100A40009CC182804207998FE5BFEF120FAF411121
:100A50002EC63284B684EFB00FCCE15701C9B2453F
:100A600091E99757FF1F2385074C81473E85410138
:100A70006F10EFAE9D461756FF1F1306764BA685E7
:100A80002285EFF09FCFAA8775F105479756FF1F84
:100A90002380E64AE1BFEF12AFA8411191E99757D1
:100AA000FF1F23A707340144228541016F108FAA3D
:100AB000B68532858D467000EFF03FCC2A846DF507
:100AC0008347D1000347E1001759FF1F130909327B
:100AD000A2074207D98F0347C100D98F1757FF1FBD
:100AE0002328F730EF706FDA61D1EF700FDA8324CB
:100AF0004900AA89EF706FD933F5A4028327490012
:100B0000FD17CE97898F1757FF1F2323F72E69BF35
:100B1000EF12AFA21C45AA8491CFD84B01CF83D747
:100B2000470089CBEF601F92AA8509C588446105FB
:100B3000EF60C04C9757FF1F9387C7299C43014420
:100B400089EF6F10CFA19C4813171400BA9703D5F3
:100B5000070019C1EFE0CFCF0504EF70CFC7E34422
:100B6000A4FEC5B7EF126F9D011185E9EF605FDA52
:100B700001449757FF1F23A707309757FF1F23A54F
:100B800007309757FF1F23A307309757FF1F23A155
:100B90000730228505616F108F9CB6873285C94664
:100BA0007000BE85EFF07FBD2A8465F54146930550
:100BB000E1001755FF1F1305E52CEF80C001035519
:100BC000C100EF608FD7F1B78DE19757FF1F23AFBB
:100BD00007209757FF1F938767219C470145ED9B8F
:100BE0001757FF1F2328F7208280EF120F9541111E
:100BF000B685328595463000EFF03FB815EDA24737
:100C00001757FF1F2324F71E9757FF1F9387071EB1
:100C10009447B24713F7B6FF13F6170019C213E74C
:100C20004600858393F7F7079756FF1F23A4E61C1A
:100C30001757FF1F2308F72241016F104F92EF1241
:100C40002F8E03841500DC412A89AE848507038733
:100C5000F7FF19C36340800C8387240091C7635555
:100C600080007D14620461849C40370700FF0907FF
:100C7000F98F3707001009076392E70A6355800070
:100C800079146204618483C70400858B95E39379AA
:100C9000F40F4E8A93178A01E187634AF008A2870E
:100CA0006353040081473384F9407D1462046184F6
:100CB0008385240081C54A85EFF0BFAA9C40370791
:100CC00000FF0907F98F370700100907639AE70645
:100CD000930500034A85EFF0DFA883C7040093055E
:100CE0008005918B99E3930580074A85EFF07FA7F4
:100CF00083C70400858B81CB1374F40F9317840191
:100D0000E1876347F004C04005048305F4FFA1E9CF
:100D10006F104F847D14620461840DBF3707000893
:100D20000907E392E7F6E35080F67D1499BF930537
:100D300000024A857D1AEFF0DFA2137AFA0F99BFFD
:100D4000370700080907E395E7FA9305000371BF29
:100D5000930500034A85EFF0DFA07D1471BF4A853B
:100D6000EFF03FA055B7EF025FFDEF70CFAA2A84E6
:100D7000EF706FA9229589450605EFE02FC6E5576C
:100D800011C59757FF1F23A9A71681473E856F00FE
:100D90001FFD930700026306F5005D15133555002E
:100DA000828005458280EF02BFF74111AA892A8916
:100DB000130419008304F4FF32C62EC42685EFF015
:100DC0005FFDA245324659E19307D0026392F408D1
:100DD000830404000548130429009377F6FEC9E74D
:100DE00093070003639FF40E830704001307800535
:100DF00093F7F7FD6399E70683041400414609045D
:100E0000B70600806314080093C6F6FFB3FEC6025F
:100E10008147254F654EFD5F33D3C602138704FD1E
:100E20006368EF06BA8463D5C408630DF5017D5588
:100E3000636AF3006394670063C69E000545B307C9
:100E4000F602A69705048304F4FFC9BF22898DB773
:100E50009307B0020148E392F4F8830404002A885F
:100E6000130429009DBF01CA8947E31BF6F89307C5
:100E70000003E397F4F8830704001307200493F7B3
:100E8000F7FD639BE70483041400094609048DBF42
:100E900013E704021307F7F9636CEE009388F4FB81
:100EA0001307700363741E0113077005998CA5BFA7
:100EB0007D576300E50263040800B307F04091C565
:100EC00019C19309F4FF23A035013E8541016F004C
:100ED0007FE8B687FDF5D5BF9304000315F22146E0
:100EE00005B719FE294629BFEF029FE3011161549E
:100EF0000DC53284AE89414681453689EFF0BFEA9F
:100F000093140501C180639E09002685EF30102BE4
:100F1000014401C58145EF205016228505616F000F
:100F20007FE32285CD467000CA85EFF01F852A84B5
:100F30006DF52685EF30902809E90356C1008345F9
:100F4000E1012685EF20500B01C941469305E100E0
:100F50001105EF705048D1B75D54C1B7EF025FDCA7
:100F60000111E15401CDB284AE89414681453689F3
:100F7000EFF07FE32A8463970900814426850561A9
:100F80006F005FDD2685D1467000CA85EFF0EFFE69
:100F9000AA846DF58357C100EDD3EF700F8E420523
:100FA000931704014181C18363F9A702EFB08FB6A3
:100FB0004204E14741803304F40241460C082A947C
:100FC00013054400EF7030418357E1002311F40012
:100FD0008357C1002310F40055B7E55445B7EF021D
:100FE0003FD47971E15415C53284AE8941468145BB
:100FF000B684EFF05FDB1319050113590901639EF5
:1010000009004A85EF401065814401C58145EFB074
:101010002FB1268545616F00FFD3A6859306300268
:1010200070002285EFF06FF5AA8465F54A85EF40E0
:1010300070622A8411E54A85EFB04F8C2A8431C54D
:101040008357C10023112401930964002310F40085
:101050008347E1009305F10041462302F4004E85E9
:10106000EF7070371309740141469305F1014A8509
:10107000EF707036930554004E85EFC04FBF930557
:1010800064014A85EFC0AFBE69B7DD5459B7EF02BE
:101090003FC9797111E5E154268545616F009FCB09
:1010A000B284AE89414681453689EFF0DFCF131A0D
:1010B0000501135A0A015285EFE06FCA2A8463982A
:1010C000090071D98145EFB02FB48144F1B726856D
:1010D000930610027000CA85EFF02FEAAA844DFD36
:1010E00031C8B2479305D1004146858B230FF400E8
:1010F000B24713050403858393F7F707A30FF400A2
:10110000EF70702D41469305D10113059408EF70DF
:10111000902C59B73304690383A70A0B3E94835775
:10112000C401638337030509EF60FFEDE344A9FEC3
:10113000DD549DB7C1690149975AFF1F938A0ACBB5
:10114000130B400EFD19CDB7231E440159BF49CDE5
:10115000EF021FBD4111B289AE8441468145368AF6
:10116000EFF07FC4931A050193DA0A010149175B76
:10117000FF1F130BABC7EF601FE1634AA9000145D6
:10118000ADCC81441759FF1F130949C681A8832795
:101190004B0B131439003E948357040063885705A2
:1011A0000509D1BF8327490B139434003E9483571C
:1011B000040085E72310540191467000D2854E85C6
:1011C000EFF0AFDB1DE9B24713978700E18321837E
:1011D000858B58C02301F4000DA08504EF60BFDAB1
:1011E000E3C2A4FC5D5511A861558280F1F421464B
:1011F00081452285EF007FB7014541016F009FB512
:101200001971D2C4130AC10686CEA2CCA6CACAC816
:10121000CEC6D6C2B6D6BAD8BEDAC2DCC6DE52C494
:1012200063810524FD151C102ACC2ECA02CE3EC8AF
:101230009304B0021549A94983050600130416005A
:101240009DE1F2465247E24763FBE620B6972380D2
:1012500007007245F6406644D6444649B649264AD8
:10126000964A09618280930750026386F500480818
:10127000EFF02FCFF5A88357C100230701000145E8
:1012800093F7C70F2316F100814501480147014636
:1012900081469308D00213030003130E30020504A5
:1012A0008307F4FF99C7638C970463C3F404638BCB
:1012B000C70501CA0346C100858A799AD18E2306E3
:1012C000D100630908008346C100098BF59A558F48
:1012D0002306E10019C12307B100138707FD137727
:1012E000F70FA54663E2E6068146A545294535A0E8
:1012F000E38717FBE39F67FA0546FD564DB70545A3
:10130000854571BF05487D5759BFB386A6020504C0
:101310008307F4FFBA96E206E18613F7F70F130688
:1013200007FD1376F60F63E5C500138707FDF1BFD0
:101330001306F7F91376F60F636EC902138797FA4F
:10134000E30537FDA306D100130790066385E70484
:10135000634BF706130780056384E70A6345F702CA
:10136000E38107EE1307500293055002E381E7F093
:101370002286D9B51307F7FB1377F70FE364E9FC6F
:10138000138797FC75BF130730066386E70A1307B8
:101390004006E39FE7FC03250A00A947A307F100E5
:1013A000930A4A00635805009307D0023305A04012
:1013B0002307F1006C00EFF0AFB56C004808EFF0C8
:1013C0001F88568A75B713073007638EE706634197
:1013D000F7021307F006638EE70413070007E3998B
:1013E000E7F80347C100136727002306E10009A8B7
:1013F00013075007638BE70213078007E39AE7F6AA
:10140000938787FA414793B71700A307E100139723
:1014100027008347C100ED9BD98F2306F100930A73
:101420004A006C0003250A0079B7A947A307F10019
:10143000FDB7A147E5BF83050A004808930A4A00A3
:10144000EFF02FB2BDBF83270A006C0048083EC8EA
:10145000EFF0EFFE1C10930A4A003EC89DB7BA9702
:10146000FDB30145C5BBEF025F8D2A8836858346F3
:101470004800BA8703475800A206D98E328717B6AC
:1014800000001306669089E517B6000013068690E3
:10149000BE85EFF0FFD66F009F8C9757FF1F938795
:1014A000A7A89C4381CFEF025F89D843B2862E86DE
:1014B0001847AA853E8502976F007F8A6155828012
:1014C000EF02BF878357050039712A84231EF1007C
:1014D000834745009305650041461305F101230F3D
:1014E000F100EF70406F9305740141461305F1025E
:1014F000EF70606E8356240017B600001306C69185
:10150000E5450A85EFF0DFCF6C08130630020A8547
:10151000EFF0BFF821616F009F84EF021F823971E5
:101520002A849305050341461305D101EF70A06A93
:101530009305940841461305D102EF70C0698347B3
:10154000E4010347F4018356C401858B0607D98F54
:1015500017B600001306068DE5450A85230EF10037
:10156000EFF01FCA6C08130610020A85EFF0FFF2B5
:1015700021616F00CFFEEF02AFFA37040001B7041C
:1015800000FF0111814A1759FF1F130929867D1495
:101590009389F4FF17BA0000130A4A8DEF60BF9ECB
:1015A00063C5AA0005616F00EFFA8327490B139703
:1015B0003A003E978347370095CF5C43A30107006D
:1015C0005286B3F687008247E5454800E58FD58F00
:1015D0003EC083462700B3F73701858AE206D58FE0
:1015E000835607003EC0EFF0BFC111468A85480010
:1015F000EFF0BFEA850A5DB7EF022FF4014681459F
:10160000EFF0BFE96F00AFF583576500638E071AEF
:101610001D71A2CCA6CACAC886CECEC6D2C4D6C2B6
:10162000DAC05EDE801013F717003289AA8431CB4E
:10163000F99B2313F500EF601F9906053D054199BD
:101640000A8BC16A3301A1408A8B8149014AFD1A84
:10165000EF607F97634CAA0C7947930604FB17A6AB
:1016600000001306A67FCA852685EFF0DFDF638FB3
:10167000090C13961900DE85130504FBEFF0FFE15A
:101680005A8183D7640013F7270021CBF59B23935E
:10169000F400EF605F9406053D0541998A8A3301A5
:1016A000A1400A8B8149014AEF60FF926345AA0A73
:1016B0006547930604FB17A600001306A67ACA85A1
:1016C0002685EFF05FDA6387090A13961900DA8539
:1016D000130504FBEFF07FDC568183D7640013F71A
:1016E000470005CBED9B2393F4006547930604FB6D
:1016F00017A6000013064677CA852685EFF0BFD6E9
:101700009C4481C703D747003DEB130504FBEFF072
:10171000BFEE130104FAF6406644D6444649B64982
:10172000264A964A064BF25B25618280DC441317F9
:101730001A00BA9703D70700630857019397190057
:10174000DE972390E7008509050A19B7130504FB06
:10175000EFF09FEA35B79C4813171A00BA9703D7E2
:10176000070019C793971900DA972390E7008509B6
:10177000050A1DBF130504FBEFF01FE8B1BF2314DA
:10178000E4FA03D767008326C4FA2146520751833F
:101790002315E4FA370700F0758F9447930584FA10
:1017A000130504FB92069182558F2326E4FA83C722
:1017B000770013F707018347F4FABD9BD98FA3077E
:1017C000F4FAEFF09FCDB1B78280EF028FD41744C7
:1017D000FF1F1304A4610444797193F7F4FB1747C6
:1017E000FF1F2329F76093F70404A1C78588A1E0B0
:1017F00097A9000093898967EF60EFF863DBA40283
:101800008327440B139934003E998356090091CEE7
:101810004E86E5454808EFF0BF9E4808EFF0DFDD53
:10182000214681454A85EF004FD48504F1B7EFF09A
:101830009FD41C4413F7F7F79746FF1F23ACE65AD3
:1018400093F707086397071E1C4413F7F7EF9746B3
:10185000FF1F23A1E65A13F707106318071E184449
:101860009377F7DF9746FF1F23A6F6589376072056
:1018700095C6058B630A072018408983858B3ACA71
:101880000347840715464C080607D98F17A50000A3
:101890001305855A230CF100EFF03FC01C4413F7E9
:1018A000F7BF9746FF1F23A7E65493F707408DC362
:1018B000835744000D464C08231AF10083576400F7
:1018C00017A5000013058557230BF100EFF0FFBCAF
:1018D0001844FD749387F47FF98F9746FF1F23AB5D
:1018E000F6509317470163DF0700EFA08FE119C996
:1018F0008356C5016391061A17A500001305855488
:10190000EFF09FCF1C447D777D177D8F9746FF1F9B
:1019100023A2E64E13973701635A0702858B63882B
:10192000071CEFA04FDF1DC118458347E5001D468A
:101930003ACA0357C5004C0817A500001305055106
:10194000231CE100230DF100EFF03FB51844F977B7
:10195000FD17F98F9746FF1F23AEF648931727010F
:1019600063D90700814517050000130525CAEF500C
:10197000FFF21844E177FD17F98F9746FF1F23AB5D
:10198000F6469317070163D30702EFA0BF982A8496
:10199000814417A900001309E94BEF600FEE9397FC
:1019A00004014205C183418163EAA71445616F00C8
:1019B000CFB983A70A0093141900BE9483D70400FB
:1019C00033F767011DCF1396170133F77701B3F68D
:1019D00037016352060417A600001306E64309E721
:1019E00017A6000013060644E5454808EFF05F819E
:1019F0004808EFF07FC083D70400B3F74701239076
:101A0000F4000509EF602FE1AA84EF60CFDF26958F
:101A1000E341A9FA15BD368519C7EF40A04361DD42
:101A2000EFF01FAAC9BFEFD09FB371D5EFF0FFAEA3
:101A3000D9B785697D7A0149974AFF1F938ACA4BB6
:101A4000056B896BFD197D1A75BF858B9DC7EF509E
:101A50000FF3231AA10041469745FF1F9385854246
:101A600013056101EF70201749464C0817A50000C7
:101A70001305053CEFF07FA2DDB317A500001305A9
:101A8000253BEFF07FB7E1BB17A500001305C53A72
:101A9000EFF09FB621B50357E501C17785073E9763
:101AA0008357A101FD14133717003207E58FD98F33
:101AB000231DF100231AD100835605020357250286
:101AC0002146231BD100231CE100035745028566F4
:101AD000FD16758FFD76F58FD98F4C0817A5000080
:101AE00013054536231DF100EFF03F9B21BD17A5DF
:101AF00000001305A535EFF03FB089BD5C4813F732
:101B0000E7FF58C8858B89CFA6864A86C9450A85CE
:101B1000EFF00FEF8357040099E70A85EFF0DFAD90
:101B2000850461049DBD231AF100835724009305A9
:101B3000440041462808231BF100EF70C0095146BC
:101B40004C080A85EFF07F95E1BFEF020F9F8547B4
:101B50003395A7009747FF1F938747299C4741115B
:101B600081455D8D9747FF1F23A6A72893770570B2
:101B700085E393576500858BA1CBC1679387078861
:101B80007D8D05EDEF606FD19305803EB305B50205
:101B90001745FF1F130585362EC6EF50A03BB245F3
:101BA00019C16349B50085C51745FF1F13050535E4
:101BB000EF50C04441016F008F9AEF600FCE2A842E
:101BC000EF60AFCEE360A4FCEF602FCE75BF0145A0
:101BD000EFF0BFBFC5B7EF024F967971AA860144F7
:101BE0001749FF1F1309892036C6EF60CFB9B246E7
:101BF000635CA4028327490B93143400BE9483D7FB
:101C000004006396D70285C617A6000013060626B1
:101C1000E5454808EFF0CFDE4808EFF0FF9D21468C
:101C200081452685EF006F9445616F004F93050451
:101C300065BF19C223200600814701C59306D00362
:101C400089E53E85828085050505838705000307B4
:101C5000050099CF6394E700E397D7FE8147D5B796
:101C60009306D0038547E30ED7FC93371700D1BF07
:101C70009307F002E316F7FE854761D6050508C213
:101C8000C9B799C123A0050081470DC11308D0032E
:101C90001306F0023307F5008306070081CA638745
:101CA00006016397C60099C1050798C13E858280E9
:101CB0008507CDB731C9EF02CF8541112E8A6C005F
:101CC0002A89368BB28A97A400009384E40DEFF042
:101CD0005FFB2A8C0144A689B14B88406286CA8585
:101CE000EF70E01801ED0E044E945C403245DA8648
:101CF0005686D285829741016F002F850504A10485
:101D0000E31D74FD6155C5BF7D55828099E5615520
:101D10008280615505616F00EF83EF026F802E8A2C
:101D20002A8401118145B28452854146BA89368997
:101D3000EFF06F8793150501C1811376F50FA1812F
:101D40002285EF507FB12A8469D552854C08EFF087
:101D50005FF3524A2A8BE30E0AFA2A8697A50000FF
:101D60009385C50F5285EF708010AA8A0DED7D5ABC
:101D7000EF606FA563C5AA0099E8014561BF5C44A7
:101D800013971A00850ABA9723904701D5B74C4498
:101D90002EC6EF604FA3B245131615004E8502996B
:101DA000E34DA0FC85BF5A8697A500009385850B5F
:101DB0005285EF70C00B0DE1032A0401EF60AFA163
:101DC0001316150081455285EFF03EFADDD40C481C
:101DD0002EC6EF604FA0C1B75A8697A50000938525
:101DE000A5085285EF70A00841E11C44A5CF81EC05
:101DF000D443370700E0758F9447D8C33707001FD7
:101E0000758F98C701BFA1463008CE854A85EFE09F
:101E1000DF96E31105F01844835781017D76231284
:101E2000F7008357A1019396470183576700D1823A
:101E3000F18FD58FF2467D767D16F182858AB206C6
:101E4000F18FD58F2313F7008347E1018356C1013A
:101E50002305F7008347B7002314D700FD8BA305A4
:101E6000F7004DBD7D557DB55A8697A50000938539
:101E700025F35285EF60B07FE31D05E81C4CE38A33
:101E800007E89C43E38707E8CE864A86A685228535
:101E9000829749B5EFF27EEA3687B2862E86AA850A
:101EA0000545EFF0BFE66FF09EEBEFF21EE93687D7
:101EB000B2862E86AA850145EFF05FE56FF03EEA17
:101EC000EFF21EE6411199C123A005009747FF1FBD
:101ED00093878704804381441DC82E89AA893114C1
:101EE0001DC40C4070004E85EFF0BFD419CD81E8C1
:101EF000A284630C0900B2472320F90039A08C406A
:101F000008400146EFF0FFD265F5404869F82685A4
:101F100041016FF03EE4184111CBEFF21EE2AE87B3
:101F20003E85B285368602976FF07EE33555828016
:101F3000EFF2BEE08357C50013D70501C205B38792
:101F4000E7021841C1814849BA95BE95EFF0BFFC40
:101F50006FF0FEE0584111CBEFF23EDEAE873E85DA
:101F6000B285368602976FF09EDF35558280184520
:101F700009CBEFF29EDCAE873E85B28502976FF00B
:101F80001EDE355582805C4599C7EFF21EDB2E853B
:101F900082976FF0DEDC35558280EFF27ED88329A0
:101FA0000500035AC5002A844849AE848145EFF0F4
:101FB0009FFD2A890DE193D50401B385450303569E
:101FC000C4004848CE95EFF09FFA2A8909E54848B1
:101FD0008545EFF05FFB4A856FF0DED7EFF25ED408
:101FE0002A890441035BC500484979712E848145E3
:101FF000B28A368AEFF03FF941E193590401B3897F
:102000006903420441802694A299034409013304E0
:1020100080403374440111CC03254901A2865686C1
:10202000CE85EFF03FF3AA8431E1330A8A40A299CA
:10203000A29A8144630C0A025286D68508080324BA
:102040004901EF605039834609011C089305F00FE0
:10205000338646413385470136C6EFF01ED1B2467E
:102060001008CE852285EFF0FFEEAA8403254901F2
:102070008545EFF05FF1268545616FF0BECDEFF24B
:10208000DECB2E864C41A1462A84EFF03FF5AA8490
:1020900003450401A145EFE07F985C403385A740EC
:1020A00048C026856FF0BECB814797A60000938677
:1020B000A6CC6393C70082803387F50003470700EF
:1020C0008507398D135745003697034707001205DA
:1020D000398D1375F50F13574500369703470700E1
:1020E0001205398D1375F50FE9B7EFF21EC52A8475
:1020F000AA851D461305F00FEFF01FFB8347740000
:102100003385A7403335A0006FF07EC5EFF2FEC2E5
:102110004111A1463000EFF0BFE109ED0357810006
:10212000C167FD1705456317F7002800EFF0FFFBB7
:102130003335A00041016FF09EC2EFF27EBEAE8447
:102140008C414111A1462A8903440501EFF05FDE6D
:10215000AA8939E9A1452285EFE05F8C9C400357AD
:10216000C9002A8AAA97939607019CC0C182098F49
:10217000639CE602C16513D70701B385B74011E739
:102180008355E900FD15C205BE958CC0A1460A869F
:102190004A85EFF0FFD9AA8901E90A85EFF0FFF43B
:1021A00001C9832749009CC04E8541016FF09EBA4A
:1021B0000357C9008357210080403307474163DB41
:1021C000E70033FA470363170A004177798C3E949E
:1021D00080C0D9BF03450901A145417AEFE01F84C2
:1021E000098CAA8A80C0337A4401417B63648A00E7
:1021F00081495DBFA1463000A2854A85EFF05FD3DB
:10220000AA895DF12800EFF05FEE11E98357A10084
:102210000357C100337A6A0180C0BA973E9A3304EB
:102220005441E9B7EFF27EB12A84AA851D46130511
:10223000F00FEFF07FE7A303A4006FF05EB2EFF2C0
:102240005EAD2A84034505015D71A145EFE00FFDF8
:102250005C402A8B0355E4004179B3F727016C00F9
:102260003EC6EFE00FFD8355C400B247A1463008DB
:10227000BE95B385654122852EC8EFF07FCBAA8439
:10228000634B05002808EFF05FE611C9B2452285CF
:10229000EFF0BFD0AA84268561616FF01EABC24704
:1022A0000357A101417C338B6741B3F72701BA97EC
:1022B0003EC810100C082285C24BEFF01FE8AA841C
:1022C00079F90810EFF07FE22DE95C403ECA30104A
:1022D0004C0822855249EFF05FE6AA844DFD035772
:1022E0008102835701026316F7002810EFF0FFDF29
:1022F00009C55840D247E31CF7FC63902B05835770
:10230000410285CF83572102B3FA8B010810BE9A90
:102310001C442311F102EFF0FFF083490401035A3A
:102320004102B309304193F90902631B0A000C1002
:102330002285EFF0DFD4AA8439FDE31C7BF7B9B71F
:102340004E8963733A015289CA861018D685228550
:10235000EFF01FBEAA8421F1630909000C44CA866C
:1023600010182285EFF09FC7AA8403450401CA858F
:10237000EFE0CFEA1C443E9508C4E39E04F0330A24
:102380002A41CA9A5DB7EFF2BE99411191E5FD5419
:10239000268541016FF01E9CC44983D725014CC995
:1023A00004C12316F50003C705012A842317E5009D
:1023B00003C5150193160701130700022308A400A3
:1023C000C182E366A7FCE1D7B3E4F402E9F08547F4
:1023D000E3FFD7FAA145EFE06FE4AA89014A01497A
:1023E0008357C400931509012285BE95B3853541F5
:1023F0002EC2EFF0BFD119ED0355E4004C00050AE1
:10240000EFE02FE39245420A2285135A0A01EFF0CA
:10241000FFCF09E905098357E4004209135909016F
:10242000E360F9FC8357E40063944701D1548DB70E
:10243000639427039245A1463000B3853541228538
:10244000EFF01FAF35E12800EFF03FCA11C503558B
:10245000E4004C00EFE0EFDD9247C17A338737416B
:1024600058C04177F98F1CC44C401C4463EEF50002
:10247000A14630002285EFF0BFAB1DE52800EFF04C
:10248000DFC6032A44001DC15C400355E4004179C6
:10249000B3F727014C003EC2EFE0AFD99245228549
:1024A000EFF0DFC6635C0502AA84DDB5124503596F
:1024B000A100035BC10033F5AA002A99034504017A
:1024C000DA85EFE0AFD54A9508C46314450163137C
:1024D0000B04330A3A412322440179B709C58547E1
:1024E000A308F40075B54C402285EFF01FAB4DFDFD
:1024F00048408357C40086093375A9003E953305CB
:10250000354148C03375250108C42285EFF03FD31B
:1025100079D559BF4D5549BF83471501C9CFEFF252
:102520004EFF2A840345050141112E8AA145BA892F
:102530003689328BEFE08FCE8357C4000605898F32
:102540007D5563E727075C4081443EC230004C0064
:102550002285924AEFF07FBE21ED835B8100639973
:102560004B012800EFF07FB801E58504C204C1806B
:1025700058409247630BF702E3FA99FC8356C10077
:1025800061559DC663E63403C175B3FABA0063733F
:10259000D900CA868355A1005A862285D695EFF0C8
:1025A0003F9919E50355C10021A06155E3884BFD12
:1025B00041016FF08EF949558280EFF20EF8014724
:1025C000EFF09FF56FF0AEF9EFF22EF73284B2869E
:1025D0002E86835545000841EFF03FFE635385008A
:1025E0002A8422856FF0AEF7EFF22EF283471501B1
:1025F0003971C954BDC7034B05012EC62A84A145B4
:102600005A853689328AEFE06FC10D473307E502FC
:102610008357C400AA8DFD54998F63E42705630492
:10262000090063000A045C403ECA30084C08228559
:10263000524DEFF09FB0AA8945ED83578101324793
:102640006397E7002808EFF05FAA6306051058407B
:10265000D247E31CF7FC8144631B090019A08144A5
:1026600099E7268521616FF00EEEE35CA0FE5A85A6
:10267000CA85EFE0AFBA014B11C5330BB501420B70
:10268000135B0B01014D7D5CC17B930C44008357B0
:10269000E4006380A70D1C4444403307FB0063EB58
:1026A000E40432472311F1020810FD572310E10220
:1026B000231221032303F102EFF0DFB663090900BF
:1026C0000C44CA8652862285EFF05F91AA890345A1
:1026D0000401CA85EFE08FB41C443E9508C4639999
:1026E00009000C102285EFF09F99AA89CA8435D978
:1026F000CE8485BF03450401A145EFE02FB2B38727
:10270000A4002311F1028357C400B3F47401231011
:102710008103BE94898C44C0081023120102EFF09B
:102720007FB00C102285EFF09F95AA840355E4003A
:10273000E685EFE00FB05C40B3F777011CC4E3928D
:1027400004F22285EFF0BFAFAA84E31C05F0050D6B
:102750003DBFC15439B78357C101E30209F0E39883
:1027600027F1C177034C0401B377FD00035DA1019C
:10277000330C8041137C0C023E9DD28ACA8CE28BC2
:1027800063F38C01E68BDE861010EA852285EFF07C
:102790002FFAAA84E31B05EC5E860C105685EF60C9
:1027A0002041AA84E31505ECB38C7C415E9DDE9A42
:1027B000E3970CFC7DB5EFF24ED881460146EFF071
:1027C000BFE26FF0CED9638C050EEFF28ED45D714F
:1027D000054D19C213BD160003590502B68B328B85
:1027E00005094209135909012E8A2A84CA89216CD4
:1027F000930A8500E15C9304F9FFC204C180638FF2
:1028000084059306A0045000A6855685EFF0FFDAF4
:102810006357050063139501A6892689E9BF9C08C3
:102820003E95230A05FA4C005285EFF08EDE75F5D1
:1028300063040D0883570402639597089387F4FF98
:102840002310F402894613060402A1655685EFF0B1
:10285000BFD96358050661616FF02ECF0145E31CB7
:102860000DFE0549B1675D55E387F9FE9165CE958B
:1028700093048400C205DE865A86C1812685EFF066
:10288000BFD6630D09005285EF60405DAA8652866F
:10289000CE852685EFF05FD5E34F05FA8357040216
:1028A00063FF370323103403894613060402A1652E
:1028B0002685EFF07FD325A0A689014965B77D5510
:1028C0008280A6855685EFF01FEFE34605F89165F7
:1028D000FD15CA95C205C1815685EFF0DFEDE35CB9
:1028E000A0F601458DBFEFF2CEC203540502916AF6
:1028F0001D71050442042A89AE894180A16B130A27
:102900008500FD1A130B05029304F4FFC204C18075
:10291000639D7405916B2164130A8900850B170C64
:102920000000130CACCA8357090293041400C204BC
:10293000C18085076383F40E5E949306A00450085B
:10294000A68552854204EFF05FC74180AA8A85467A
:1029500013067100A2855285EFF03FC62A8B6347AC
:1029600050076347A00626847DBF56949306A004B3
:102970005008A68552854204EFF03FC441802A8C5E
:10298000854613067100A2855285EFF01FC3634C84
:102990008003E351A0F883570902E39D97F69387DC
:1029A000F4FF2310F90289465A86A1655285EFF09B
:1029B000BFC3A6855285EFF01FE0A2855285EFF0D8
:1029C0009FDF268491B7E358A0FCA9B7634BA00012
:1029D000A6855285EFF03FDEA2855285EFF0BFDD80
:1029E00059B79C10BE9A238A0AFA639109022C00F7
:1029F0004808EFF0EFCC25D91C45224552C62318D4
:102A0000810074006286DA858297B1BF0146CE8567
:102A10004808EFF00FA261FDB9B7014525616FF0DD
:102A2000CEB2EFF28EB19737FF1F9387E74E804308
:102A3000814409C42A893114814401E426856FF058
:102A40000EB2631809005C4481EF404865D8311428
:102A5000EDB708400146CA85EFF0AF9D6DF5F5B7BB
:102A60008297E5F4AA84D5B7EFF22EAD9737FF1F12
:102A70009387074B8043AA8409EC2685EFF07FFA01
:102A8000AA840144EF502FD0636CA40026856FF018
:102A90000EAD5C402285A6859C4382970040E9BF2D
:102AA00005041374F40FF9BFEFF22EA90145EFF0FE
:102AB000BFFB6FF0CEAA9737FF1F9387674623A00F
:102AC000070023A207008280EFF22EA79737FF1F8F
:102AD0009387874423A0070023A20700EFF0BFFDE0
:102AE0006FF0EEA7EFF26EA54111130985002A845D
:102AF000EF50CFE5AA854A85EFF0FF88AA8419ED4B
:102B000089461306E100A1654A85EFF01FABE17726
:102B1000634405008357E1002310F4022685410138
:102B20006FF0EEA39737FF1F9387873F90430147CE
:102B3000B28691EE05E3DC4310C11737FF1F232156
:102B4000A73E85EF9737FF1F23AEA73C82803687CD
:102B50009442C5B7144385E2DC432320050091EB82
:102B60009737FF1F23A0A73C9737FF1F23AAA73A39
:102B7000828088C3C1BF14C108C38280EFF2EE9B7C
:102B80001734FF1F130404352285EFF0BFF5AA8424
:102B900005E5179900001309292722859737FF1F9C
:102BA00023AC2733EFF01FF89737FF1F23A62733F7
:102BB0009737FF1F23AA873626856FF04E9A9737DF
:102BC000FF1F83C7A736795599EFEFF20E97EFF005
:102BD000BFEFEFF0BFFA11E585471737FF1F230757
:102BE000F7346FF0CE978280EFF22E959737FF1F64
:102BF0009387873280432A89BE8419C0311415E037
